:020000040000FA
:100000000EEF00F0FFFFFFFFD3EFF7F0FFFFFFFF62
:10001000FFFFFFFFFFFFFFFF8DEF02F09AEFF8F009
:100020000001BC6F49040DE1481CBB6FBC51BB5DB6
:1000300002E2BC6902D04850BC27120EBC650ED04B
:100040000CD00001BC51485C03E3010EBC6F02D030
:100050004850BC5F080EBC6101D0BC6F486ABC51FF
:100060001200050E0001BB5D100EBC5901E3640CCB
:100070001F0EBB5D0F0EBC5901E3500C610EBB5D42
:100080000E0EBC5901E33C0CC10EBB5D0D0EBC59FC
:1000900001E3280CE50EBB5D0C0EBC5901E3140C0A
:1000A000000CB36AB46A050EB56EEC0EB16E780E34
:1000B000B06EB0506F00C4FEBBF00001BC6B6000BE
:1000C000ECF2BCF0BB6BBB110201F56F0001BC513F
:1000D0000201F66F3901A4919481010EB26E010CF8
:1000E000C75101011A150001C06FC85101011B154C
:1000F0000001C16F60001CF3C2F0600020F3C3F088
:100100001DECFFF0C051C96FC95106E00A0EA219DB
:1001100003E1010E01018F6F0001C9511200C751A7
:100120000201AA150001C06FC8510201AB15000100
:10013000C16F60001CF3C2F0600020F3C3F01DEC3F
:10014000FFF0C051C96FC95106E00A0EA21903E1C0
:10015000010E01018F6F0001C9511200BC6F4904EB
:1001600011E1481C0001BB6FBC51BB5D02E2BC69E0
:1001700002D04850BC27BC513E5C0CE26000F8F055
:10018000BCF008D048500001BC5D02E2BC6B02D05C
:100190004850BC5F486ABC5112003C0174AB04D0AB
:1001A0000001BB6BBB2B02D00001BB6B3C01010EFD
:1001B00074AB000E0101BA19010ED8B4000E000193
:1001C000BB15BC6F3C01000E74BB010E0101BA6F80
:1001D0000001BC5112009B6A9C6A020E9D6EE20EE9
:1001E000996E986A98506F0064FEBBF00001BC6B7A
:1001F0006000ECF2BCF0BB6BBB110201F36F0001BD
:10020000BC510201F46F3901A89D010E9A6E010CD8
:10021000BC6F49040FE1481C0001BB6FBC51BB5DC2
:1002200002E2BC6902D04850BC27040EBC650AD06B
:10023000BC6F08D048500001BC5D02E2BC6B02D02C
:100240004850BC5F486ABC511200C46FEC0E0001FC
:10025000C56F020EC66F600010F3ECF260000CF385
:10026000EDF2080EC361080CC351D8B4120060004F
:1002700014F3BDF0600018F3BEF0020EBF6F580E0D
:100280005CEFF2F0C46FEC0E0001C56F020EC66F9A
:10029000600010F3ECF260000CF3EDF2080EC361A5
:1002A000080CC351D8B41200600014F3BDF0600014
:1002B00018F3BEF0020EBF6F580E5CEFF2F00001B3
:1002C000BC6B010ECABE000EBD6FBD51A519BC6F3F
:1002D000BC51BD15A36FBD5103E1BB6BBB2B02D05D
:1002E0000001BB6BBC51BD19BB15A46F6000F4F2DB
:1002F000A5F01200C06F0001C26BBF5114E0010EE7
:10030000C16F03D0D890BF37C12BBFAFFBD7D890F8
:10031000C237BF51C05D03E3BF51C05FC281D890F7
:10032000BF33C12FF4D7C2511200DE6BDF6BE06B1D
:10033000E16BE46BE56BEA6BEC6BF16BF36BF46B0D
:10034000F56BF66BF76BF96BFA6BFB6BFC6B030EE3
:10035000FD6FFE6B1F0EFF6F840EF86F840C0001A3
:10036000BC6F1F0EBC6501D0BC6FBB98BB9A270E3B
:1003700081EC03F0BB8ABB9A810E81EC03F0BB8A4F
:10038000BB9A0001BC5181EC03F0BB8ABB88120010
:10039000500EBC6FFA0EBD6F0B0EBE6F010EBF6F1D
:1003A000060EC06F3F0EC16FC26B010EC36FC46BF0
:1003B000C56BC66BC76B6000D8F3C8F0B3EFEAF04B
:1003C0000101FF510FE0EA0E5824D96EDA6A010EDE
:1003D000DA22DF503D01EA6F582A150E586405D025
:1003E000586E03D039019399596A0101FF07120031
:1003F000500EBC6FFA0EBD6F0B0EBE6F010EBF6FBD
:10040000C06F3F0EC16FC26B010EC36FC46BC56B73
:10041000C66BC76B6000D8F3C8F0B3EFEAF00D0EFF
:1004200020600D0C600078F00FF060007CF010F0A0
:10043000600080F011F0000E126A136A146A166AE6
:10044000156A176A196A186A6CEFF0F0C751020151
:10045000AC150001C06FC8510201AD150001C16F9C
:1004600060001CF3C2F0600020F3C3F01DECFFF04D
:10047000C051C96FC9511200050E576F586B070E56
:10048000596F010E5A6F070E5B6F110E5C6F5D6B3B
:10049000220E5E6F5F6B9B0E566F3901AA939A8393
:1004A0009B0C0F0E3C016B6F6C6B010E6D6F270E7A
:1004B0006E6F070E6F6F260E706F190E716F290E1B
:1004C000726F160E736F830E6A6F830CBC6F080E0B
:1004D0000001BD6FBE6BD890BC35BE35BE6FD890E5
:1004E000BC37BB51BE5D02E3BB51BE5FBD2FF3D72E
:1004F000BE511200070E0001926503D0120E9265E4
:1005000004D00D0E926F92C07BF1AF5103E0030E49
:10051000AF65030C020EAF6F020C6F0060FFBAF004
:10052000390194B1A4A103D0C0EC03F005D099B176
:10053000A9A102D0F4EC03F06000EBF2D8FF1100A7
:10054000010E966E956A976A9368926AA99199814D
:10055000000E0001BB6BBC6BBD6B01EC04F0D00E58
:10056000946ED00CBB6F0001BB050AE1010EBC6F9D
:10057000120E3F6406D08F6F010E01016B6F01D028
:10058000BC6B0001BC5112000001BC6F6000ECF2BA
:10059000DCF16000ECF2FFF1390193B905D06000A5
:1005A000F3F2EAFD010E586E938912003D015DAF32
:1005B00003D05750D8B41200576A800E5E6F200ED9
:1005C0005F6F030E656F840E5D6F636B606B12006F
:1005D000B1C0B4F00001B151B1253D016F6FFE0E05
:1005E000706F010E0101B86F4F6E0001AE6F010117
:1005F000B46F010C0001BB6F0101E4510001BB1994
:1006000008E03E01F89F6000EFF2F1FEF88FF89DE0
:10061000F8810001BB511200B2A409D0B290600071
:10062000E7F2B1FF6000E3F2B0FFB28012006000B9
:10063000E7F2B1FF6000E3F2B0FF12000A0E3C01E6
:10064000756F0E0E766F050E776F786F796F020EED
:100650007A6F7B6B7C6B7D6B860E746F860C010EE4
:100660000001C96FFF0ECA6FCB6BCC6BCD6BCE6B2D
:10067000D06BCF6BD16BD36BD26B050EC1EFEDF0AE
:10068000BE6BBF6B09D0BF51BB25D96E000EBC211C
:10069000DA6EDF50BE1BBF2BBD51BF5DF4E3BE5110
:1006A0001200026E600004F0DCF1600004F0FFF163
:1006B000390193B905D060000BF0EAFD010E586EC8
:1006C00093891200046A056A09D005500124D96E85
:1006D000000E0220DA6EDF50041A052A0350055C72
:1006E000F4E304501200BC51030B3901E16F6000C8
:1006F000EFF2E0F93F0EE517E58100F000F0E3517D
:1007000012000001BB6F010E3D01126F6000EFF29D
:1007100011FD3901A2A9FDD73D01105112003E0182
:10072000F0510001BE6FBD6B3E01EF510001BD25D0
:10073000BB6F000EBE21BC6F1200200E3D01156F75
:10074000030E166F070E196F010E1C6F830E146FC8
:10075000830CD28A3901838183838387838983854C
:10076000828F8A83849189911200060EAE6EAD6AE3
:10077000AF6A610EAB6EAA6AA495C00EAC6EC00CD7
:10078000A4916000D4FBB8F06000D8FBB9F00CEC89
:1007900003F083EFE6F0C06BC16BC26BC36BC46B3D
:1007A000C56BC66BC76B1200600E3901D96FDB6B6E
:1007B000DD6B080EDF6FDE6B12000001905102E16D
:1007C0004AEFF7F04FEFEEF0BB6F6000ECF29DF0F8
:1007D0001200820E3E01C16F820C0001BB6FBB5143
:1007E0001200BE92C6921200A991596A12002020EE
:1007F000202000FFAC8E1200B2801200AA931200DB
:100800001200120001FFFFFFFFFFFFFFFFFFFFFFCE
:10081000FFFFFFFFFFFFFFFFFFFFFFFFFFFFFFFFE8
:10082000FFFFFFFFFFFFFFFFFFFFFFFFFFFFFFFFD8
:10083000FFFFFFFFFFFFFFFFFFFFFFFFFFFFFFFFC8
:10084000FFFFFFFFFFFFFFFFFFFFFFFFFFFFFFFFB8
:10B07000000000000000FE020202020202020202C0
:10B0800002020202020202020202020202020202A0
:10B090000202020202020202020202020202020290
:10B0A0000202020202020202020202020202020280
:10B0B00002020202020202FE0000FF000000000085
:10B0C0000000000000000000000000000000000080
:10B0D0000000000000000000000000000000000070
:10B0E0000000000000000000000000000000000060
:10B0F0000000000000000000000000FF0000FF0052
:10B10000000000000000000000000000000000003F
:10B11000000000000000000000000000000000002F
:10B12000000000000000000000000000000000001F
:10B13000000000000000000000000000000000FF10
:10B140000000FF0000000000000000000000000000
:10B1500000000000000000000000000000000000EF
:10B1600000000000000000000000000000000000DF
:10B1700000000000000000000000000000000000CF
:10B18000000000FF00007F40404040404040404001
:10B1900040404040404040404040404040404040AF
:10B1A000404040404040404040404040404040409F
:10B1B000404040404040404040404040404040408F
:10B1C000404040404040407F0000FE020202020238
:10B1D000020202020202020202FA32C202FA0282EF
:10B1E000424242820242FA420202FA82424282020F
:10B1F00082424282C202FA020242FA42020202027F
:10B200000202020202020202020202FE0000FF002B
:10B21000000000808000800080000000800780E047
:10B22000931700F304848403000083840400F70070
:10B230008080070003848402078003848400030461
:10B240000400000000A0008000808000000000FFDB
:10B250000000FF000000070808050F0007080804A9
:10B260000F00000F0000000F0100000F00070A0A86
:10B270000B000F0908080700070A0A0B000F01005E
:10B28000000F000000000000000F000F0100000F81
:10B29000000000FF0000FF000000000000000000B0
:10B2A0000000000000000000000000000000FF019E
:10B2B00001010101FF000000FF0101010101FF0088
:10B2C000000000000000000000000000000000007E
:10B2D00000000000000000FF00007F4040404040B0
:10B2E000404040404040404040404040404040405E
:10B2F0004040FF8080808080FF404040FF80808011
:10B300008080FF40404040404040404040404040FE
:10B3100040404040404040404040407F0000FE02EE
:10B32000020202FA02020202E29AE20202FA8242F5
:10B330002202FA82422202C2020202C20282424275
:10B34000420242FA42020282424282C202C2824265
:10B3500042820282424282FA020202FA020202FEA1
:10B360000000FF00008080058000F007808000075B
:10B3700000878182040087818204F00384840207AD
:10B38000008485058200F0030484F08304040287AE
:10B390008007008000878003040404A700800085E4
:10B3A000800000FF0000FF00070808050F000F09DC
:10B3B00008080700090A0A040007080808000F0126
:10B3C00000000F00070808050F000708080007081D
:10B3D0000800070A0A0B000F0100000F0000000F11
:10B3E000000F0100000F00FF0000FF000000000040
:10B3F0000000000000000000000000000000FF014D
:10B4000001010101FF0000FF0101010101FF000036
:10B4100000FF0101010101FF000000000000000029
:10B420000000000000000000000000FF00007F405E
:10B43000404040404040404040404040404040400C
:10B440004040FF8080808080FF4040FF808080807F
:10B4500080FF404040FF8080808080FF404040402F
:10B460004040404040404040404040404040407F9D
:10B470000000FE02020202020282424282C202FA7C
:10B48000824242820282424242028242424202FAA4
:10B49000824243820282424282C202FA020242FA9B
:10B4A0004202028242428202C2824242820202027C
:10B4B000020202FE0000FF0000000000000304047E
:10B4C0000207000704040403000405050200030446
:10B4D000040400A70080008780030404020700031F
:10B4E0000404000304040003050505000700000030
:10B4F00007000000000000FF0000FF000000000047
:10B50000000000000000000000000000000000003B
:10B51000000000000000000F000F0100000F0000FD
:10B52000000000000000000000000000000000001B
:10B530000000000000000000000000FF0000FF000D
:10B5400000000000000000000000000000000000FB
:10B55000000000000000FF0101010101FF000000E8
:10B56000FF0101010101FF000000000000000000D8
:10B57000000000000000000000000000000000FFCC
:10B5800000007F40404040404040404040404040FC
:10B5900040404040404040404040FF8080808080AC
:10B5A000FF404040FF8080808080FF40404040401E
:10B5B000404040404040404040404040404040408B
:10B5C0004040407F0000FE0202020202020202022C
:10B5D0000202020202F2628202F20202828282020B
:10B5E0000282F2820202F20282820202028282025B
:10B5F0008202F2020282F2820202020202020202CB
:10B6000002020202020202FE0000FF00000000002F
:10B610000000000000000000000F0001060F0007FE
:10B62000080808070000070808000F0100000F00C5
:10B63000070808050F0007080800070808000000B1
:10B640000000000000000000000000FF0000FF00FC
:10B6500000000000000000000070888850F80078AA
:10B66000808040F80008FE090100FF100808F00083
:10B6700070A8A8B000FF908888700070A8A8B000DB
:10B68000F8100808F000000000000000000000FFB3
:10B690000000FF008000808000009000008080801B
:10B6A00000F0008080000080F08001000000008039
:10B6B0008000008000008000F0000000008080001A
:10B6C0008000800000008000F0008080000080F09A
:10B6D000800000FF00007F404F4140404F404F40FE
:10B6E00047484848404F4140404F40404748484005
:10B6F0004040474A4A4B404F4241404047484840FB
:10B70000474848454F40474848444F404F494848BC
:10B71000474040474848407F0000FE0202C232C214
:10B72000020202828202F202820202820202828209
:10B7300002020282828202028282820292020282D9
:10B7400082020282020282028202020282028202D9
:10B750008282020202828202820202FE0000FF0056
:10B760000E0101010E00070808090F000F02010079
:10B7700000070A0A0B00090A0A0400090A0A040061
:10B780000F00070A0A0B000F020100000708080457
:10B790000F000F0100000F00072828251F0000FFE1
:10B7A0000000FF000000000000000000000000009A
:10B7B0000000000000000000F8100808F000F90088
:10B7C0007088888800FF100808F000087F888000D3
:10B7D0000000000000000000000000000000000069
:10B7E000000000FF0000FF0000000000000000005B
:10B7F000000000000000E02020C02020C000C02485
:10B800002024C000C0202040E000FC000000E40034
:10B81000C020202000FC402020C0000000000000CC
:10B8200000000000000000FF00007F40404040405A
:10B830004040404040404040404043404043404002
:10B840004340414242424140414A4A4947404142C5
:10B8500042404340414242424043404040434040D6
:10B8600040404040404040404040407F0000FE0299
:10B8700002C24242428202020202020202020202A8
:10B880000202020202020202024202020202020258
:10B89000020202020202824242020202020202C2C8
:10B8A0000202020202020202020202C2020202FEBC
:10B8B0000000FF00003F060A1221001C2222143E55
:10B8C000003E0402023C001CA2A2947E003E001C2A
:10B8D0002A2A2C003E0804020002FF02001C222239
:10B8E000143E003F0402023C003E08040200021F16
:10B8F000222000FF0000FF00000000000000000008
:10B900000000000000000000000000000000000037
:10B910000000000000000000000000000000000027
:10B920000000000000000000000000000000000017
:10B9300000000000000000FF0000FF000000000009
:10B94000000000000000000000000000000000E017
:10B950001010A0F000FE40A0100010FE100000F239
:10B960000030C000C03000000000000000000000F7
:10B970000000000000000000000000FF00007F4009
:10B9800040404040404040404040404040404040B7
:10B9900040404040414140414041404041404040A2
:10B9A0004141404140404041404040404040404093
:10B9B0004040404040404040404040404040407F48
:10B9C0000000FE020202020202020202020202025F
:10B9D0000202828282820202020202020202020247
:10B9E0000202020202020202020202020202020237
:10B9F0000202020202020202020202020202020227
:10BA0000020202FE0000FF00000000000000000033
:10BA10000000000000007F4444443B007C10080408
:10BA20000038545458007C040478040478004854C6
:10BA30005424003854545800000000000000000056
:10BA400000000000000000FF0000FF0000000000F8
:10BA500000000000000000000000000000000000E6
:10BA600000000000000000000000000000000000D6
:10BA700000000000000000000000000000000000C6
:10BA80000000000000000000000000FF0000FF00B8
:10BA900000000000000000000000000000000000A6
:10BAA000000000E01010A0F000FE40A0100010FE0A
:10BAB000100000F20030C000C030000000000000A4
:10BAC000000000000000000000000000000000FF77
:10BAD00000007F40404040404040404040404040A7
:10BAE0004040404040404040414140414041404052
:10BAF0004140404041414041404040414040404041
:10BB00004040404040404040404040404040404035
:10BB10004040407F0000FE0202020202020202C216
:10BB200032C2020282020202820282F28202020215
:10BB300082828202028282820282820202028282E5
:10BB400002820282F28202029202F2020282020265
:10BB500002020202020202FE0000FF0000000000DA
:10BB600000000E0101010E00070808040F00000785
:10BB7000C82820070808080700EF00000F00000F82
:10BB80000007080805EF0000070808000F000F0273
:10BB90000508000101010101000000FF0000FF0095
:10BBA0000000000000000000000000000000000095
:10BBB000000000017F01000E11110A1F001F020189
:10BBC000011E001F04020100010F111000000000FF
:10BBD000000000000000000000000000000000FF66
:10BBE0000000FF0000000000000000000000000056
:10BBF00000000000000000E01010A0F000FE40A0D7
:10BC0000100010FE100000F20030C000C030000034
:10BC10000000000000000000000000000000000024
:10BC2000000000FF00007F40404040404040404056
:10BC30004040404040404040404040404141404101
:10BC400040414040414040404141404140404041EE
:10BC500040404040404040404040404040404040E4
:10BC6000404040404040407F0000FE020202021A75
:10BC7000E202E21A0202C2A2A2C20202E28242224C
:10BC80000202FA422222C20202EA0202E242222214
:10BC9000C20202C2222242FA0202C2A2A2C20202CC
:10BCA000E2422222C2020202020202FE0000FFF869
:10BCB000F8F8F8F8F8FBF8F8F8F8F9FAFAFAF8F8FA
:10BCC000FBF8F8F8F8F8FBFAFAFAF9F8F8FBF8F8E4
:10BCD000FBF8F8F8FBF8F8F9FA1A1A1B1818191AF1
:10BCE0001A1A18181B1818181B181818181818FFE3
:10BCF0000000FF0303FBFBFBFBFBFBFB0303FFFF5E
:10BD0000FFFFFFFFFFFFFFFFFFFFFFFFFFFFFFFF43
:10BD1000FFFFFFFFFFFFFFFFFFFFFFFFFF0080C0F0
:10BD20004040C08000C0C04040C080004040404013
:10BD3000C0C000FF0000FFFE00E2F0FAF8FAF0E2F7
:10BD400000FEFFFFFFFFFFFFFFFFFFFFFFFFFFFF03
:10BD5000FFFFFFFFFFFFFFFFFFFFFFFFFFFFFFFFF3
:10BD6000FF000F1F10101D0D001F1F10101F0F00D0
:10BD7000181C1613111000FF00007F414054414B66
:10BD8000434B415440417F7F7F7F7F7F7F7F7F7F19
:10BD90007F7F7F7F7F7F7F7F7F7F7F7F7F7F7F7FB3
:10BDA0007F7F7F7F7F404040404040404040404058
:10BDB00040404040404040404040407F0000FE0244
:10BDC0000202020202020202020202020202020253
:10BDD000E29AE2020202FA028242020242FA4202BB
:10BDE0000202CA020282424242820202C2824242EB
:10BDF000820202020202020202020202020202FEA7
:10BE00000000FF0000000000000000000000000033
:10BE10000000000700000007000007010204000006
:10BE200000030404000007000003040404030000EE
:10BE300007000000070000000000000000000000F4
:10BE4000000000FF0000FF000000000000000000F4
:10BE500000000000000000000000F8100808F000DA
:10BE600000F90000708888880000FF100808F000C2
:10BE700000087F8880000000000000000000000033
:10BE800000000000000000FF0000FF008040408034
:10BE90000000C0008040000040F0480000804040AA
:10BEA00040800000F80000000080404080C000009A
:10BEB000C00080400000804040800000C80000803A
:10BEC0004040400000F88040408000FF00007F407C
:10BED000434545454040474140404040405F404029
:10BEE000404344444443404043444440404354540A
:10BEF000524F404047414040404043454545404007
:10BF00004740404344444440404740404047407FCE
:10BF10000000FE0202020202020202020202020209
:10BF200002020202826282020202E20202020202B1
:10BF300002E20202020222020202020202020202E1
:10BF400002020202020202020202020202020202D1
:10BF5000020202FE0000FF000000000000000000DE
:10BF6000000000000000001C0302031C00001F046E
:10BF70000A110000010F111000001F00000E111126
:10BF8000110E00001F0201011E0000000000000051
:10BF900000000000000000FF0000FF0000000000A3
:10BFA000000000000000000000C0200000000000B1
:10BFB00000000000E00000000000000000000000A1
:10BFC0000000000000000000000000002000000051
:10BFD0000000000000E00000000000FF0000FF0083
:10BFE0000E15151600001F0402010000017F01005C
:10BFF000000E1111110E00000F101000000E515113
:10C000004A3F00001F04020100000E151516000033
:10C010001F00000E11111100001F0201011E00FF80
:10C0200000007F4040404040404040404040404051
:10C030004040404040404040404040404040404000
:10C0400040404040404040404040404040404040F0
:10C0500040404040404040404040404040404040E0
:10C060004040407F0000FE02020202020202020281
:10C070000202E29AE20202C2020202C20242FA4250
:10C080000202824242428302028282820202F20A57
:10C090000A0AF20242F24A0A0242F24A0A02020280
:10C0A00002020202020202FE0000FF000000000085
:10C0B000000000000007000000070003040402075E
:10C0C00000000304040003A4048403808000000033
:10C0D0000000030404040300001F000000001F0010
:10C0E0000000000000000000000000FF0000FF0052
:10C0F0000000000000000000000000000000000040
:10C1000000000000000000000000000F000F010010
:10C11000000F000000000000000000000000000010
:10C12000000000000000000000000000000000FF10
:10C130000000FF0000000000000000000000000000
:10C1400000000000000000000000FF0101010101EB
:10C15000FF000000FF0101010101FF0000000000DD
:10C1600000000000000000000000000000000000CF
:10C17000000000FF00007F40404040404040404001
:10C180004040404040404040404040404040FF80B0
:10C1900080808080FF404040FF8080808080FF4022
:10C1A000404040404040404040404040404040408F
:10C1B000404040404040407F0000FE020202020238
:10C1C00002FA02020202824242428202FA824222BF
:10C1D0000282424282C20282424282FA02C2824207
:10C1E00042028242428202824242420282424242EF
:10C1F0000282424282020202020202FE0000FF00AC
:10C200000000000000070404840003040404830009
:10C2100007818204000384848207F0038484040776
:10C2200000878080000083850505F00405058200F5
:10C23000848505020003850505000000000000FF5D
:10C240000000FF00000000000000000001060C07D5
:10C250000C060100070A0A0B0007080808000F0176
:10C2600000000F00090A0A0400070A0A0B00070869
:10C2700008000F0100000F00000004000000000093
:10C28000000000FF0000FF000000000000000000B0
:10C2900000FF0101010101FF0000FF010101010197
:10C2A000FF0000FF0101010101FF0000FF0101018A
:10C2B0000101FF000000000000000000000000007D
:10C2C00000000000000000FF00007F4040404040B0
:10C2D0004040404040FF8080808080FF4040FF80A1
:10C2E00080808080FF4040FF8080808080FF4040D1
:10C2F000FF8080808080FF40404040404040404080
:10C3000040404040404040404040407F00000000EE
:10C31000000000000000000000000000000000001D
:10C32000000000000000000000000000000000000D
:10C3300000000000000000000000000000000000FD
:10C3400000000000000000000000000000000000ED
:10C3500000000000000000000000000000000000DD
:10C3600000000000000000000000000000000000CD
:10C3700000000000000000000000000000000000BD
:10C3800000000000000000000000000000000000AD
:10C39000000000000000FCFA060606060606060677
:10C3A000060646A62626264606060686868606062D
:10C3B000068606868606060606868606E6060606BD
:10C3C000868686060606860686860606060606060D
:10C3D000060606060606FAFC00003F5F6060606025
:10C3E000606060606060646869696A646060676A10
:10C3F0006A6A6360606F6160606F606067686865EB
:10C400006F6060676A6A6A6360606F6160606F60D6
:10C41000606060606060606060605F3F0000FCFAC8
:10C420000606E6C686060606060646A6262626460C
:10C43000060606868686060606860686860606069C
:10C4400006868606E60606068686860606068606AC
:10C4500086860606060606060686C6E60606FAFC72
:10C46000FE003F5FE0E0EFE7E3E1E0E0E0E0E4E88A
:10C47000E9E9EAE4E0E0E7EAEAEAE3E0E0EFE1E064
:10C48000E0EFE0E0E7E8E8E5EFE0E0E7EAEAEAE34A
:10C49000E0E0EFE1E0E0EFE0E0E0E0E0E1E3E7EF63
:10C4A000E0E0DFBF7FFF0305F9F9F9F9F9F9F9F9E0
:10C4B000F9F9B959D9D9D9B9F9F9F9797979F9F9EC
:10C4C000F979F97979F9F9F9F97979F919F9F9F93C
:10C4D000797979F9F9F979F97979F9F9F9F9F9F9CC
:10C4E000F9F9F9F9F9F90503FFFFC0A09F9F9F9F94
:10C4F0009F9F9F9F9F9F9B979696959B9F9F989589
:10C5000095959C9F9F909E9F9F909F9F9897979A8D
:10C51000909F9F989595959C9F9F909E9F9F909F81
:10C520009F9F9F9F9F9F9F9F9F9FA0C0FF00FCFA80
:10C53000060606060606060606060606060606069B
:10C5400006060606060606E6F63636F6E60606068B
:10C55000F6F6C6E67636060606060606060606065B
:10C560000606060606060606060606060606FAFC81
:10C5700000003F5F6060606060606060606060609D
:10C580006060606060606060606060676F6C6C6F6E
:10C59000676060606F6F63676E6C60606060606052
:10C5A000606060606060606060606060606060608B
:10C5B00060605F3F0000FCFA0606E6C686060606D7
:10C5C000060606060606060606060606060606E62B
:10C5D000F63636F6E6060606F6F6C6E676360606BB
:10C5E00006060606060606060606060606060606EB
:10C5F0000686C6E60606FAFCFE003F5FE0E0EFE7CF
:10C60000E3E1E0E0E0E0E0E0E0E0E0E0E0E0E0E026
:10C61000E0E0E0E7EFECECEFE7E0E0E0EFEFE3E7AE
:10C62000EEECE0E0E0E0E0E0E0E0E0E0E0E0E0E0F0
:10C63000E0E0E0E0E1E3E7EFE0E0DFBF7FFF0305FC
:10C64000F9F9F9F9F9F9F9F9F9F9F9F9F9F9F9F95A
:10C65000F9F9F9F9F9F9F91909C9C90919F9F9F94A
:10C660000909391989C9F9F9F9F9F9F9F9F9F9F95A
:10C67000F9F9F9F9F9F9F9F9F9F9F9F9F9F9050314
:10C68000FFFFC0A09F9F9F9F9F9F9F9F9F9F9F9FD8
:10C690009F9F9F9F9F9F9F9F9F9F9F9890939390E7
:10C6A000989F9F9F90909C9891939F9F9F9F9F9FE3
:10C6B0009F9F9F9F9F9F9F9F9F9F9F9F9F9F9F9F8A
:10C6C0009F9FA0C0FF00FCFA06060606060606C6E7
:10C6D000261626C60606F6864646860606F68646CA
:10C6E00046860606C6068646460606C6060606C6EA
:10C6F000060686464646860606F6864646860606AA
:10C70000060606060606FAFC00003F5F60606060F1
:10C710006060606F6161616F60606F6468686760CE
:10C72000606F6468686760606F61606060606067C8
:10C730006868646F6060676868686460606F6060A4
:10C74000606F60606060606060605F3F0000FCFA86
:10C750000606E6C6860606C6261626C60606F68619
:10C760004646860606F6864646860606C606864679
:10C77000460606C6060606C60606864646468606D9
:10C7800006F68646468606060686C6E60606FAFCCF
:10C79000FE003F5FE0E0EFE7E3E1E0EFE1E1E1EF42
:10C7A000E0E0EFE4E8E8E7E0E0EFE4E8E8E7E0E035
:10C7B000EFE1E0E0E0E0E0E7E8E8E4EFE0E0E7E830
:10C7C000E8E8E4E0E0EFE0E0E0EFE0E0E1E3E7EF1D
:10C7D000E0E0DFBF7FFF0305F9F9F9F9F9F9F9396D
:10C7E000D9E9D939F9F90979B9B979F9F90979B9E9
:10C7F000B979F9F939F979B9B9F9F939F9F9F939A9
:10C80000F9F979B9B9B979F9F90979B9B979F9F9C8
:10C81000F9F9F9F9F9F90503FFFFC0A09F9F9F9F60
:10C820009F9F9F909E9E9E909F9F909B9797989F63
:10C830009F909B9797989F9F909E9F9F9F9F9F9849
:10C8400097979B909F9F989797979B9F9F909F9F4D
:10C850009F909F9F9F9F9F9F9F9FA0C0FF00FE0252
:10C8600002D20202C2824242820202C2020202C218
:10C87000020282424242820202C202824242020218
:10C8800082424242820202020202020202020206C4
:10C89000FE0602826212120A0A121262820206FE68
:10C8A00000007F40404F40404F4040404F4040409C
:10C8B000434C43404040474949494940404F41402B
:10C8C0004040404044494B4A444040404040404042
:10C8D000404040607F60404146484850504848468C
:10C8E0004140607F0000FE0202D20202C282424248
:10C8F000820202C2020202C2020282424242820258
:10C9000002C2028242420202824242428202020287
:10C910000202020202020206FE0602826212120AEB
:10C920000A121262820206FEFE003F40C0CFC0C063
:10C93000CFC0C0C0CFC0C0C0C3CCC3C0C0C0C7C9B7
:10C94000C9C9C9C0C0CFC1C0C0C0C0C0C4C9CBCA9A
:10C95000C4C0C0C0C0C0C0C0C0C0C0E0FFE0C0C153
:10C96000C6C8C8D0D0C8C8C6C1C0C0BF7F00FE06F8
:10C97000FA2AFAFA3A7ABABA7AFAFA3AFAFAFA3AA7
:10C98000FAFA7ABABABA7AFAFA3AFA7ABABAFAFA87
:10C990007ABABABA7AFAFAFAFAFAFAFAFAFAFA06AB
:10C9A000FE060282E2F2F2FAFAF2F2E2820206FEF7
:10C9B00000007F605F505F5F505F5F5F505F5F5F51
:10C9C0005C535C5F5F5F58565656565F5F505E5FC4
:10C9D0005F5F5F5F5B5654555B5F5F5F5F5F5F5F8D
:10C9E0005F5F5F607F604041474F4F5F5F4F4F47E2
:10C9F0004140607F0000FE06FA2AFAFA3A7ABABA93
:10CA00007AFAFA3AFAFAFA3AFAFA7ABABABA7AFA46
:10CA1000FA3AFA7ABABAFAFA7ABABABA7AFAFAFAF6
:10CA2000FAFAFAFAFAFAFA06FE060282E2F2F2FAE2
:10CA3000FAF2F2E2820206FEFE003F60DFD0DFDFA4
:10CA4000D0DFDFDFD0DFDFDFDCD3DCDFDFDFD8D636
:10CA5000D6D6D6DFDFD0DEDFDFDFDFDFDBD6D4D533
:10CA6000DBDFDFDFDFDFDFDFDFDFDFE0FFE0C0C1F5
:10CA7000C7CFCFDFDFCFCFC7C1C0C0BF7F00FE02AF
:10CA800002F2828282F20202F292929262020232F6
:10CA90004282423202020202020202020202020246
:10CAA0000202020202020202020202020202020662
:10CAB000FE0602826212120A0A121262820206FE46
:10CAC00000007F40404F4040404F40404F41424473
:10CAD0004840404C4241424C404040404040404031
:10CAE0004040404040404040404040404040404046
:10CAF000404040607F60404146484850504848466A
:10CB00004140607F0000FE0202F2828282F2020255
:10CB1000F292929262020232428242320202020295
:10CB200002020202020202020202020202020202E5
:10CB30000202020202020206FE0602826212120AC9
:10CB40000A121262820206FEFE003F40C0CFC0C041
:10CB5000C0CFC0C0CFC1C2C4C8C0C0CCC2C1C2CC8B
:10CB6000C0C0C0C0C0C0C0C0C0C0C0C0C0C0C0C0C5
:10CB7000C0C0C0C0C0C0C0C0C0C0C0E0FFE0C0C135
:10CB8000C6C8C8D0D0C8C8C6C1C0C0BF7F00FE06D6
:10CB9000FA0A7A7A7A0AFAFA0A6A6A6A9AFAFACA85
:10CBA000BA7ABACAFAFAFAFAFAFAFAFAFAFAFAFA15
:10CBB000FAFAFAFAFAFAFAFAFAFAFAFAFAFAFA06C9
:10CBC000FE060282E2F2F2FAFAF2F2E2820206FED5
:10CBD00000007F605F505F5F5F505F5F505E5D5B36
:10CBE000575F5F535D5E5D535F5F5F5F5F5F5F5F7A
:10CBF0005F5F5F5F5F5F5F5F5F5F5F5F5F5F5F5F45
:10CC00005F5F5F607F604041474F4F5F5F4F4F47BF
:10CC10004140607F0000FE06FA0A7A7A7A0AFAFA40
:10CC20000A6A6A6A9AFAFACABA7ABACAFAFAFAFAC4
:10CC3000FAFAFAFAFAFAFAFAFAFAFAFAFAFAFAFA54
:10CC4000FAFAFAFAFAFAFA06FE060282E2F2F2FAC0
:10CC5000FAF2F2E2820206FEFE003F60DFD0DFDF82
:10CC6000DFD0DFDFD0DEDDDBD7DFDFD3DDDEDDD31E
:10CC7000DFDFDFDFDFDFDFDFDFDFDFDFDFDFDFDFC4
:10CC8000DFDFDFDFDFDFDFDFDFDFDFE0FFE0C0C1CF
:10CC9000C7CFCFDFDFCFCFC7C1C0C0BF7F00FE028D
:10CCA00002F2828282F20202F29292926202020204
:10CCB000020202028202028202028282020282F2E4
:10CCC0008202028202028202028282820202020640
:10CCD000FE0602826212120A0A121262820206FE24
:10CCE00000007F40404F4040404F40404F41424451
:10CCF00048404141414141404F42414040474A4AFA
:10CD00004B4040474848404F4241404047484848D0
:10CD1000474040607F604041464848505048484640
:10CD20004140607F0000FE0202F2828282F2020233
:10CD3000F2929292620202020202020282020282D3
:10CD400002028282020282F28202028202028202D3
:10CD50000282828202020206FE0602826212120A27
:10CD60000A121262820206FEFE003F40C0CFC0C01F
:10CD7000C0CFC0C0CFC1C2C4C8C0C1C1C1C1C1C081
:10CD8000CFC2C1C0C0C7CACACBC0C0C7C8C8C0CF45
:10CD9000C2C1C0C0C7C8C8C8C7C0C0E0FFE0C0C1EA
:10CDA000C6C8C8D0D0C8C8C6C1C0C0BF7F00FE06B4
:10CDB000FA0A7A7A7A0AFAFA0A6A6A6A9AFAFAFA33
:10CDC000FAFAFAFA7AFAFA7AFAFA7A7AFAFA7A0A33
:10CDD0007AFAFA7AFAFA7AFAFA7A7A7AFAFAFA06A7
:10CDE000FE060282E2F2F2FAFAF2F2E2820206FEB3
:10CDF00000007F605F505F5F5F505F5F505E5D5B14
:10CE0000575F5E5E5E5E5E5F505D5E5F5F5855556C
:10CE1000545F5F5857575F505D5E5F5F5857575775
:10CE2000585F5F607F604041474F4F5F5F4F4F47A4
:10CE30004140607F0000FE06FA0A7A7A7A0AFAFA1E
:10CE40000A6A6A6A9AFAFAFAFAFAFAFA7AFAFA7A42
:10CE5000FAFA7A7AFAFA7A0A7AFAFA7AFAFA7AFA22
:10CE6000FA7A7A7AFAFAFA06FE060282E2F2F2FA1E
:10CE7000FAF2F2E2820206FEFE003F60DFD0DFDF60
:10CE8000DFD0DFDFD0DEDDDBD7DFDEDEDEDEDEDFE4
:10CE9000D0DDDEDFDFD8D5D5D4DFDFD8D7D7DFD000
:10CEA000DDDEDFDFD8D7D7D7D8DFDFE0FFE0C0C1D6
:10CEB000C7CFCFDFDFCFCFC7C1C0C0BF7F00FE026B
:10CEC00002F2828282F20202F292929262020202E2
:10CED00002020202020212121292720202221212C2
:10CEE000926202028202020282020202020202062E
:10CEF000FE0602826212120A0A121262820206FE02
:10CF000000007F40404F4040404F40404F4142442E
:10CF100048404041414141414040404E41404040F5
:10CF2000404C4A49484840404845424548404040B6
:10CF3000404040607F604041464848505048484625
:10CF40004140607F0000FE0202F2828282F2020211
:10CF5000F292929262020202020202020202121291
:10CF600012927202022212129262020282020202E1
:10CF70008202020202020206FE0602826212120A05
:10CF80000A121262820206FEFE003F40C0CFC0C0FD
:10CF9000C0CFC0C0CFC1C2C4C8C0C0C1C1C1C1C15F
:10CFA000C0C0C0CEC1C0C0C0C0CCCAC9C8C8C0C043
:10CFB000C8C5C2C5C8C0C0C0C0C0C0E0FFE0C0C1D5
:10CFC000C6C8C8D0D0C8C8C6C1C0C0BF7F00FE0692
:10CFD000FA0A7A7A7A0AFAFA0A6A6A6A9AFAFAFA11
:10CFE000FAFAFAFAFAFAEAEAEA6A8AFAFADAEAEA11
:10CFF0006A9AFAFA7AFAFAFA7AFAFAFAFAFAFA0675
:10D00000FE060282E2F2F2FAFAF2F2E2820206FE90
:10D0100000007F605F505F5F5F505F5F505E5D5BF1
:10D02000575F5F5E5E5E5E5E5F5F5F515E5F5F5F2C
:10D030005F53555657575F5F575A5D5A575F5F5F4B
:10D040005F5F5F607F604041474F4F5F5F4F4F477B
:10D050004140607F0000FE06FA0A7A7A7A0AFAFAFC
:10D060000A6A6A6A9AFAFAFAFAFAFAFAFAFAEAEA40
:10D07000EA6A8AFAFADAEAEA6A9AFAFA7AFAFAFAD0
:10D080007AFAFAFAFAFAFA06FE060282E2F2F2FAFC
:10D09000FAF2F2E2820206FEFE003F60DFD0DFDF3E
:10D0A000DFD0DFDFD0DEDDDBD7DFDFDEDEDEDEDEC2
:10D0B000DFDFDFD1DEDFDFDFDFD3D5D6D7D7DFDFBE
:10D0C000D7DADDDAD7DFDFDFDFDFDFE0FFE0C0C1A7
:10D0D000C7CFCFDFDFCFCFC7C1C0C0BF7F00FCFA53
:10D0E00006060606060606060606060606060606E0
:10D0F0000686E6763676E686060606F6F606060620
:10D10000F6F60606E6F6B6B6B6B63606060606061F
:10D110000606060606060606060606060606FAFCC5
:10D1200000003F5F606060606060606060606060E1
:10D13000606060606E6F63636363636F6E6060679F
:10D140006F6C6C6C6F6F60606C6D6D6D6D6F676038
:10D1500060606060606060606060606060606060CF
:10D1600060605F3F0000FCFA0606E6C6860606061B
:10D1700006060606060606060686E6763676E6867F
:10D18000060606F6F6060606F6F60606E6F6B6B64F
:10D19000B6B636060606060606060606060606069F
:10D1A0000686C6E60606FAFCFE003F5FE0E0EFE713
:10D1B000E3E1E0E0E0E0E0E0E0E0E0E0EEEFE3E348
:10D1C000E3E3E3EFEEE0E0E7EFECECECEFEFE0E0E1
:10D1D000ECEDEDEDEDEFE7E0E0E0E0E0E0E0E0E0F9
:10D1E000E0E0E0E0E1E3E7EFE0E0DFBF7FFF030541
:10D1F000F9F9F9F9F9F9F9F9F9F9F9F9F9F9F9F99F
:10D20000F9791989E9891979F9F9F90909F9F9F91E
:10D210000909F9F91909494949C9F9F9F9F9F9F96E
:10D22000F9F9F9F9F9F9F9F9F9F9F9F9F9F9050358
:10D23000FFFFC0A09F9F9F9F9F9F9F9F9F9F9F9F1C
:10D240009F9F9F9F91909C9C9C9C9C90919F9F983E
:10D250009093939390909F9F9392929290989F9F78
:10D260009F9F9F9F9F9F9F9F9F9F9F9F9F9F9F9FCE
:10D270009F9FA0C0FF00FCFA0606060606060606EB
:10D28000060606060606066696961626060686F61E
:10D290008606060686464686C60606C606864646AE
:10D2A000060686F68606060606060606060606062E
:10D2B000060606060606FAFC00003F5F6060606036
:10D2C000606060606060606060606064686969663A
:10D2D0006060606768686060676868646F60606FFE
:10D2E0006160606060606067686860606060606026
:10D2F000606060606060606060605F3F0000FCFADA
:10D300000606E6C68606060606060606060606663D
:10D3100096961626060686F68606060686464686ED
:10D32000C60606C606864646060686F6860606062D
:10D3300006060606060606060686C6E60606FAFC83
:10D34000FE003F5FE0E0EFE7E3E1E0E0E0E0E0E0A7
:10D35000E0E0E0E4E8E9E9E6E0E0E0E7E8E8E0E092
:10D36000E7E8E8E4EFE0E0EFE1E0E0E0E0E0E0E77C
:10D37000E8E8E0E0E0E0E0E0E0E0E0E0E1E3E7EF83
:10D38000E0E0DFBF7FFF0305F9F9F9F9F9F9F9F9F1
:10D39000F9F9F9F9F9F9F9996969E9D9F9F979091D
:10D3A00079F9F9F979B9B97939F9F939F979B9B96D
:10D3B000F9F9790979F9F9F9F9F9F9F9F9F9F9F9CD
:10D3C000F9F9F9F9F9F90503FFFFC0A09F9F9F9FA5
:10D3D0009F9F9F9F9F9F9F9F9F9F9F9B9796969981
:10D3E0009F9F9F9897979F9F9897979B909F9F909D
:10D3F0009E9F9F9F9F9F9F9897979F9F9F9F9F9F55
:10D400009F9F9F9F9F9F9F9F9F9FA0C0FF2A3E001F
:10D410003E00F8080808080808080808C83800008E
:10D42000000000FF0000000000000000F8070000FE
:10D4300000000000FF000000000000C03F000000EE
:10D440000000000000FF0000000000F807000000DE
:10D4500000001C221C000F080808080F0000000034
:10D4600000002A3E003E00F80808080808080808DE
:10D4700008C8380000000000FF00000000000000A5
:10D4800000F807000000000000FF0000000000009E
:10D49000C03F0000000000000000FF00000000008E
:10D4A000F80700000000001C221C000F0C0C0C0CE4
:10D4B0000F0000000000002A3E003E00F8080808A7
:10D4C000080808080808C8380000000000FF00002D
:10D4D000000000000000F807000000000000FF004E
:10D4E0000000000000C03F0000000000000000FF3E
:10D4F0000000000000F80700000000001C221C00D3
:10D500000F0E0E0E0E0F0000000000002A3E003E1F
:10D5100000F8080808080808080808C838000000CB
:10D520000000FF0000000000000000F807000000FD
:10D53000000000FF000000000000C03F00000000ED
:10D5400000000000FF0000000000F80700000000DD
:10D55000001C221C000F0F0F0F0F0F000000000017
:10D56000002A3E003E00F8080808080808080808D5
:10D57000C8380000000000FF0000000000000000AC
:10D58000F807000000000000FF000000000000C0DD
:10D590003F0000000000000000FF8080808080F8D5
:10D5A0000700000000001C221C000F0F0F0F0F0FC0
:10D5B0000000000000002A3E003E00F808080808AD
:10D5C0000808080808C8380000000000FF00000034
:10D5D0000000000000F807000000000000FF00004D
:10D5E00000000000C03F0000000000000000FFC07D
:10D5F000C0C0C0C0F80700000000001C221C000FC3
:10D600000F0F0F0F0F0000000000002A3E003E0029
:10D61000F8080808080808080808C83800000000CA
:10D6200000FF0000000000000000F80700000000FC
:10D630000000FF000000000000C03F0000000000EC
:10D64000000000FFE0E0E0E0E0F80700000000007C
:10D650001C221C000F0F0F0F0F0F00000000000016
:10D660002A3E003E00F8080808080808080808C80C
:10D67000380000000000FF0000000000000000F87B
:10D6800007000000000000FF000000000000C03F95
:10D690000000000000000000FFF0F0F0F0F0F807DC
:10D6A00000000000001C221C000F0F0F0F0F0F00C6
:10D6B00000000000002A3E003E00F80808080808A4
:10D6C00008080808C8380000000000FF000000003B
:10D6D00000000000F807000000000000FF0000004C
:10D6E000000000C03F0000000000000000FFF8F84C
:10D6F000F8F8F8F80700000000001C221C000F0FCB
:10D700000F0F0F0F0000000000002A3E003E00F83F
:10D71000080808080808080808C8380000000000C1
:10D72000FF0000000000000000F8070000000000FB
:10D7300000FF000000000000C03F000000000000EB
:10D740000000FFFCFCFCFCFCFC0700000000001CCF
:10D75000221C000F0F0F0F0F0F0000000000002A07
:10D760003E003E00F8080808080808080808C838FD
:10D770000000000000FF0000000000000000F807AB
:10D78000000000000000FF000000000000C03F009B
:10D7900000000000000000FFFEFEFEFEFEFE07008F
:10D7A000000000001C221C000F0F0F0F0F0F0000C5
:10D7B000000000002A3E003E00F80808080808089B
:10D7C000080808C8380000000000FF000000000042
:10D7D000000000F807000000000000FF000000004B
:10D7E0000000C03F0000000000000000FFFFFFFF3E
:10D7F000FFFFFF0700000000001C221C000F0F0F9E
:10D800000F0F0F0000000000002A3E003E00F80845
:10D810000808080808080808C8380000000000FFC9
:10D820000000000000000000F807000000000000F9
:10D83000FF808080808080C03F00000000000000EA
:10D8400000FFFFFFFFFFFFFF0700000000001C229A
:10D850001C000F0F0F0F0F0F0000000000002A3EEA
:10D86000003E00F8080808080808080808C838003A
:10D8700000000000FF0000000000000000F80700AA
:10D880000000000000FFC0C0C0C0C0C0C03F00001A
:10D89000000000000000FFFFFFFFFFFFFF07000088
:10D8A0000000001C221C000F0F0F0F0F0F000000C4
:10D8B0000000002A3E003E00F80808080808080892
:10D8C0000808C8380000000000FF00000000000049
:10D8D0000000F807000000000000FFE0E0E0E0E0EA
:10D8E000E0E03F0000000000000000FFFFFFFFFF3E
:10D8F000FFFF0700000000001C221C000F0F0F0F8D
:10D900000F0F0000000000002A3E003E00F808084B
:10D9100008080808080808C8380000000000FF00D0
:10D9200000000000000000F807000000000000FFF9
:10D93000F0F0F0F0F0F0F03F000000000000000018
:10D94000FFFFFFFFFFFFFF0700000000001C221C7D
:10D95000000F0F0F0F0F0F0000000000002A3E0005
:10D960003E00F8080808080808080808C838000039
:10D97000000000FF0000000000000000F8070000A9
:10D9800000000000FFF8F8F8F8F8F8F83F00000091
:10D990000000000000FFFFFFFFFFFFFF0700000087
:10D9A00000001C221C000F0F0F0F0F0F00000000C3
:10D9B00000002A3E003E00F8080808080808080889
:10D9C00008C8380000000000FF0000000000000050
:10D9D00000F807000000000000FFFCFCFCFCFCFC61
:10D9E000FC3F0000000000000000FFFFFFFFFFFF02
:10D9F000FF0700000000001C221C000F0F0F0F0F7C
:10DA00000F0000000000002A3E003E00F808080851
:10DA1000080808080808C8380000000000FF0000D7
:10DA2000000000000000F807000000000000FFFEFA
:10DA3000FEFEFEFEFEFE3F0000000000000000FFB4
:10DA4000FFFFFFFFFFFF0700000000001C221C007B
:10DA50000F0F0F0F0F0F0000000000002A3E003EC6
:10DA600000F8080808080808080808C83800000076
:10DA70000000FF0000000000000000F807000000A8
:10DA8000000000FFFFFFFFFFFFFFFF3F000000005F
:10DA900000000000FFFFFFFFFFFFFF070000000086
:10DAA000001C221C000F0F0F0F0F0F0000000000C2
:10DAB000002A3E003E00F808080808080808080880
:10DAC000C8380000000000FF808080808080808057
:10DAD000F807000000000000FFFFFFFFFFFFFFFF4F
:10DAE0003F0000000000000000FFFFFFFFFFFFFFFE
:10DAF0000700000000001C221C000F0F0F0F0F0F6B
:10DB00000000000000002A3E003E00F80808080857
:10DB10000808080808C8380000000000FFC0C0C09E
:10DB2000C0C0C0C0C0F807000000000000FFFFFF39
:10DB3000FFFFFFFFFF3F0000000000000000FFFFAD
:10DB4000FFFFFFFFFF0700000000001C221C000F6A
:10DB50000F0F0F0F0F0000000000002A3E003E00D4
:10DB6000F8080808080808080808C8380000000075
:10DB700000FFE0E0E0E0E0E0E0E0F80700000000A7
:10DB80000000FFFFFFFFFFFFFFFF3F00000000005E
:10DB9000000000FFFFFFFFFFFFFF07000000000085
:10DBA0001C221C000F0F0F0F0F0F000000000000C1
:10DBB0002A3E003E00F8080808080808080808C8B7
:10DBC000380000000000FFF0F0F0F0F0F0F0F0F8A6
:10DBD00007000000000000FFFFFFFFFFFFFFFF3F07
:10DBE0000000000000000000FFFFFFFFFFFFFF0735
:10DBF00000000000001C221C000F0F0F0F0F0F0071
:10DC000000000000002A3E003E00F808080808084E
:10DC100008080808C8380000000000FFF8F8F8F805
:10DC2000F8F8F8F8F807000000000000FFFFFFFF19
:10DC3000FFFFFFFF3F0000000000000000FFFFFFAC
:10DC4000FFFFFFFF0700000000001C221C000F0F59
:10DC50000F0F0F0F0000000000002A3E003E00F8EA
:10DC6000080808080808080808C83800000000006C
:10DC7000FFFCFCFCFCFCFCFCFCFC070000000000C2
:10DC800000FFFFFFFFFFFFFFFF3F0000000000005D
:10DC90000000FFFFFFFFFFFFFF0700000000001C68
:10DCA000221C000F0F0F0F0F0F0000000000002AB2
:10DCB0003E003E00F8080808080808080808C838A8
:10DCC0000000000000FFFEFEFEFEFEFEFEFEFE0760
:10DCD000000000000000FFFFFFFFFFFFFFFF3F000D
:10DCE00000000000000000FFFFFFFFFFFFFF070034
:10DCF000000000001C221C000F0F0F0F0F0F000070
:10DD0000000000002A3E003E00F808080808080845
:10DD1000080808C8380000000000FFFFFFFFFFFFF1
:10DD2000FFFFFFFF07000000000000FFFFFFFFFFF5
:10DD3000FFFFFF3F0000000000000000FFFFFFFFAB
:10DD4000FFFFFF0700000000001C221C000F0F0F48
:10DD50000F0F0F0000000000002A3E003E00F88870
:10DD60008888888888888888C8380000000000FF74
:10DD7000FFFFFFFFFFFFFFFFFF07000000000000A5
:10DD8000FFFFFFFFFFFFFFFF3F000000000000005C
:10DD900000FFFFFFFFFFFFFF0700000000001C2245
:10DDA0001C000F0F0F0F0F0F0000000000002A3E95
:10DDB000003E00F8C8C8C8C8C8C8C8C8C8C8380025
:10DDC00000000000FFFFFFFFFFFFFFFFFFFF070056
:10DDD0000000000000FFFFFFFFFFFFFFFF3F00000C
:10DDE000000000000000FFFFFFFFFFFFFF07000033
:10DDF0000000001C221C000F0F0F0F0F0F0000006F
:10DE00000000002A3E003E00F8E8E8E8E8E8E8E81C
:10DE1000E8E8E8380000000000FFFFFFFFFFFFFF19
:10DE2000FFFFFF07000000000000FFFFFFFFFFFFF4
:10DE3000FFFF3F0000000000000000FFFFFFFFFFAA
:10DE4000FFFF0700000000001C221C000F0F0F0F37
:10DE50000F0F0000000000002A3E003E00F8F8F816
:10DE6000F8F8F8F8F8F8F8F8380000000000FFFFBC
:10DE7000FFFFFFFFFFFFFFFF07000000000000FFA4
:10DE8000FFFFFFFFFFFFFF3F00000000000000005A
:10DE9000FFFFFFFFFFFFFF0700000000001C221C28
:10DEA000000F0F0F0F0F0F00000000000000000018
:10DEB0000000000000000000000000000000000062
:10DEC0000000000000000000000000000000000052
:10DED0000000000000000000000000000000000042
:10DEE0000000000000000000000000000000000032
:10DEF0000000000000000000000000000000000022
:10DF00000000000000000000000000000000000011
:10DF10000000000000000000000000000000000001
:10DF200000000000000000000000000000000000F1
:10DF300000000000000000000000000000000000E1
:10DF400000000000000000000000000000000000D1
:10DF500000000000000000000000000000000000C1
:10DF600000000000000000000000000000000000B1
:10DF700000000000000000000000000000000000A1
:10DF80000000000000000000000000000000000091
:10DF90000000000000000000000000000000000081
:10DFA0000000000000000000000000000000000071
:10DFB0000000000000000000000000000000000061
:10DFC0000000000000000000000000000000000051
:10DFD0000000000000000000000000000000000041
:10DFE0000000000000000000000000000000000031
:10DFF0000000000000000000000000000000000021
:10E000000000000000000000000000000000000010
:10E010000000000000000000000000000000000000
:10E0200000000000000000000000000000000000F0
:10E0300000000000000000000000000000000000E0
:10E0400000000000000000000000000000000000D0
:10E0500000000000000000000000000000000000C0
:10E0600000000000000000000000000000000000B0
:10E0700000000000000000000000000000000000A0
:10E080000000000000000000000000000000000090
:10E090000000000000000000000000000000000080
:10E0A000000080B0B4B6B63636363636363636363A
:10E0B00036363636360600000000F0F0F0F0F0F0AC
:10E0C000F0F0F0F0E0C00000F0F0F00000C0E0F090
:10E0D000F0F0F0F0F0F0E0C00000F0F0F00000F040
:10E0E000F0F00000000000000000F0F0F0F0F0F0B0
:10E0F000F0F0F0E0C00000F0F0F0000000000000E0
:10E10000000000000000606C6D6D6D0D01000000EE
:10E1100000000000000000C0C0C0C0C0C0C0C000FF
:10E12000FFFFFF000000000000FFFFFF0000F8F805
:10E13000F80000FFFFFFC0C0C0C0C0FFFFFF00002D
:10E14000F8F8F80000FFFFFF1E1E1E1E1E1E000036
:10E15000F0F8FC3C3C3C3C3CFCFFFF0000FFFFFFB8
:10E16000000000000000000000C0D8DBDBDBDBC3E8
:10E17000C0C0C0C0C0C0C0C0C0C0C000000101015C
:10E18000010101010100FFFFFFF0F0F0F0F0F0FFEE
:10E190007F3F0000FFFFFF0000F0F1F3F3F3F3F324
:10E1A000F3FF7F3F0000FFFFFF00003F7FFFF0F025
:10E1B000F0F0F0F000003F7FFFF0F0F0F0F0FF7FB4
:10E1C0003F00003F7FFFF0F0F0F0F0F000000206AB
:10E1D00006060606060606060606060606060606DF
:10E1E000000000000000000000000000000000002F
:10E1F000000000000000000000000000000000001F
:10E20000000000000000000000000000000000000E
:10E2100000000000000000000000000000000000FE
:10E2200000000000000000000000000000000000EE
:10E230000000000000000000000080F8FE7E0600E4
:10E24000000000000080F8FE7E060080F8FE7E0ED2
:10E250000E0E0E0E0E0E0ECEFEFC380000000E7ED0
:10E26000FEF080000000000080E0F07C1E0F030143
:10E27000000000000000000000000000000000009E
:10E28000000000000000000000000000000000008E
:10E290000000000000000000000000000000C0F8C6
:10E2A000FFFFC7C0C0C0C0C0C0C0F8FF3F0700C06C
:10E2B000F8FFFFC7C0C0C0C0C0C0C0F0FE7F0F01E4
:10E2C000000000000000037FFFFCF0783E0F070114
:10E2D000000000000000000000000000000000003E
:10E2E000000000000000000000000000000000002E
:10E2F000000000000000000000000000000000001E
:10E300000000E0FCFF1F03030303030303E3FFFF1D
:10E310001F0300E0FCFF1F070F3FFDF1C1010101DA
:10E3200001010000000000000080E0F07C1E0F0FE3
:10E330003FFFF0C0000000000000000000000000EF
:10E3400000000000000000000000000000000000CD
:10E3500000000000000000000000000000000000BD
:10E36000000000000000607E7F1F01000000000030
:10E3700000607E7F1F0100607E7F1F0100000000A3
:10E3800000030F3F7C7040000080C0F0783E0F0714
:10E3900001000000000000010F7F7E7000000000FF
:10E3A000000000000000000000000000000000006D
:10E3B000000000000000000000000000000000005D
:10E3C000000000000000000000000000000000004D
:10E3D000000000000000000000000000000000003D
:10E3E000000000000000000000000000000000002D
:10E3F000000000000000000000000000000000001D
:10E40000000000000000000000000000000000000C
:10E4100000000000000000000000000000000000FC
:10E4200000000000000000000000000000000000EC
:10E4300000000000000000000000000000000000DC
:10E4400000000000000000000000000000000000CC
:10E4500000000000000000000000000000000000BC
:10E4600000000000000000000000000000000000AC
:10E47000000000000000000000000000000000009C
:10E48000000000000000000000000000000000008C
:10E4900000000000000000000000008080808080FC
:10E4A000808080808080808080808080808080806C
:10E4B000808080808080808080808080808080805C
:10E4C000808080808080808080808080808080804C
:10E4D000808080808080808080808080808080803C
:10E4E000808080808080808080808080808080802C
:10E4F000808080808080808080808080000030F0FC
:10E50000F0F1793D3F3733F1F1F1793D3F3733F1A8
:10E51000F1F1793D3F3733F1F1F1793D3F3733F197
:10E52000F1F1793D3F3733F1F1F1793D3F3733F187
:10E53000F1F1793D3F3733F1F1F1793D3F3733F177
:10E54000F1F1793D3F3733F1F1F1793D3F3733F167
:10E55000F1F1793D3F3733F1F1F1793D3F37330147
:10E5600001010000000000000000000000000000A9
:10E57000000000FCFC00000000000D0D0000000089
:10E580001C3C00001C3C000000000000002020F0AB
:10E590002C20F02C120F02120F0202F0F898FE98B5
:10E5A00098100819197F191F0F18242498E0380CA7
:10E5B000301C07192424181834C4840404000609E4
:10E5C000101009061B00003C1C00000000000000A9
:10E5D00000000000E0F81C0C000000071F383000AD
:10E5E0000000000C1CF8E000000030381F0700009D
:10E5F000008080000000000001010000008080E039
:10E60000E080800001010707010100000000000018
:10E61000000000301E0E000000808080808080801E
:10E6200001010101010101000000000000000000E3
:10E63000181800000000000000C0300C00300C036F
:10E64000000000F0F87C840CF8F00F1F30213E1F12
:10E650000F30381CFCFC00000030303F3F303030C1
:10E66000381C0C9CF8F0383C3E37333130181C0C09
:10E670008C8CFCF818383031313F1FFCFC808080D6
:10E68000FCFC00010101013F3FFCFCCCCCCC8C0C1C
:10E6900018383030391F0FC0E0F0B89C8C041F3F91
:10E6A0003131313F1F0C0C0C8CCCFC78003E3F0309
:10E6B000010000F8FC8C8C8CFCF81F3F3131313F9D
:10E6C0001FF8FC8C8C8CFCF818393131313F1F005D
:10E6D000006060000000000006060000000000006E
:10E6E000606000000020301E0E000080C060301806
:10E6F0000C040103060C18302060606060606060EC
:10E7000006060606060606040C183060C080203097
:10E71000180C060301181C0C8CCCFC780000373751
:10E72000010000E0108848C810E007081112131219
:10E7300009F0F89C8C9CF8F01F1F0101011F1FFCC1
:10E74000FCCCCCCCFC381F1F1818181F0FF8FC0C81
:10E750000C0C3C380F1F1818181E0EFCFC0C0C1C5F
:10E76000F8F01F1F18181C0F07FCFCCCCCCC0C0CAD
:10E770001F1F1818181818FCFC8C8C8C0C0C1F1FF1
:10E780000101010000F8FC0C8C8C9C980F1F1819DB
:10E79000191F0FFCFCC0C0C0FCFC1F1F0000001FA5
:10E7A0001F00FCFC00000000001F1F000000000C08
:10E7B0000C0C0C0CFCFC0E1E3830381F0FFCFCC07F
:10E7C000E070381C1F1F0103070E1CFCFC0000003A
:10E7D00000001F1F1818181818FCFC70E070FCFCD3
:10E7E0001F1F0000001F1FFCFC3CF000FCFC1F1F53
:10E7F00000031E1F1FF0F81C0C1CF8F0070F1C185C
:10E800001C0F07FCFC8C8C8CFCF81F1F0101010104
:10E8100000F0F80C0C0CF8F0070F181A1C0F13FC82
:10E82000FCCCCCCCFC781F1F0103071E1C70F8DC4D
:10E83000CC9C9830060C1C191D0F070C0C0CFC0C02
:10E840000C0C0000001F000000FCFC000000FCFCA1
:10E850000F1F18180C1F1FFCFC800080FCFC00031D
:10E860000F1E0F0300FCFC00F800FCFC0F1F1C0F28
:10E870001C1F0F0C3CF0C0F03C0C181E0701071EBB
:10E88000187CFCC0C0FC7C0000001F1F0000000CB6
:10E890000C8CCCEC7C3C1E1F1B19181818FCFC0CB3
:10E8A0000C0C0C003F3F30303030000C30C000000A
:10E8B0000000000000030C3000000C0C0C0CFCFCF1
:10E8C00000303030303F3F6030180C1830600000AE
:10E8D0000000000000000000000000003030303078
:10E8E00030303000000C3C00000000000000000050
:10E8F000000060606060E0C00E1F1B1B0F1F1FFC4C
:10E90000FC80C0C0C0801F1F0D18181F0F80C0E002
:10E910006060E0C0070F1C18181C0C80C0C0C080CD
:10E92000FCFC0F1F18180D1F1FC0E0606060E0C0E6
:10E930000F1F1B1B1B1B0BC0C0F8FCCCCC0C00001A
:10E940003F3F000000C0E0606060E0C00133363649
:10E95000363F1FFCFCC0C0C0C0801F1F0000001F4E
:10E960001F00CCCC00000000001F1F0000000000B2
:10E97000000000ECEC001C3C30303F3F00FCFC0091
:10E9800080C0E0601F1F03070F1C18FCFC00000084
:10E990000000070F1C181C0C00E0E060C060E0C025
:10E9A0001F1F001F001F1FE0E0C0E0E0E0C01F1FAE
:10E9B0000100001F1F80C0E060E0C080070F1C182E
:10E9C0001C0F07E0E0606060E0C03F3F06060607FE
:10E9D00003C0E0606060E0E003070606063F3FE03A
:10E9E000E080C0C060601F1F0101000000C0E06047
:10E9F0006060604008191B1B1B1E0CC0C0FCFCC0E3
:10EA0000C0C000000F1F181818E0E0000000E0E090
:10EA1000070F18180C1F1FE0E0000000E0E00003E3
:10EA20000F1C0F0300E0E0000000E0E0070F1C0FE8
:10EA30001C0F0760E0800080E060181C0703071CC3
:10EA400018E0E0000000E0E001333333333F1F60A3
:10EA50006060E0E0E0601C1E1F1B19181880C07089
:10EA6000080C0C0001030E103030000000FCFC000C
:10EA7000000000003F3F000000000C0C0870C08048
:10EA8000003030100E0301C0E0E0C00080C0030180
:10EA90000003070703FCF8F0E0C080007F3F1F0F72
:10EAA000070301FCFE1F6183FEFC43474C484F47B0
:10EAB000430C0E07FFFF0000404C4C4F4F4C4C0CDA
:10EAC0000E87C3E77E3C4E4F4F4D4C4C4C06070320
:10EAD0006363FFFE464E4C4C4C4F473F7F60606087
:10EAE000FFFF40404040404F4F3F3F333373E3C34D
:10EAF000464E4C4C4E4743F0F87C6E67E3C1474F9F
:10EB00004C4C4C4F470383C3E3733F1E404F4F4071
:10EB1000404040FEFF636363FFFE474F4C4C4C4F49
:10EB2000473E7F636363FFFE464E4C4C4C4F47604D
:10EB3000F0B0B0B03020444C4D4D4D4F460080C039
:10EB4000E0F0F8FC0103070F1F3F7F00000000000A
:10EB500000004040404040404000000000000000F5
:10EB600000000000000000000000000000000000A5
:10EB70000000000000000000000000000000000095
:10EB80000000000000000000000000000000000085
:10EB90000000000000000000000000000000000075
:10EBA0000000000000000000000000000000000065
:10EBB0000000000000000000000000000000000055
:10EBC0000000000000000000000000000000000045
:10EBD0000000000000000000000000000000000035
:10EBE000000000000000000000000010284444C4A1
:10EBF000040404C444442810000000000000000085
:10EC000000000000F008040404F4F404040484C4C4
:10EC1000E4670000000784848484848484040404FA
:10EC2000040408F00000FF00000000FFFF1C3E7716
:10EC3000E3C1800000003E7FE3C1C1C1C1C163FFE9
:10EC4000FE00000000FF00003F20202020232320A2
:10EC5000202020212323202020282C2C2C2C2C2C5D
:10EC60002C2F27202020203F000000000000000063
:10EC700000000010284444C4040404C44444281080
:10EC8000000000000000000000000000F008040484
:10EC900004F4F404040484C4E467000000078484DA
:10ECA0008484848484040404040408F00000FF00C5
:10ECB000000000FFFF1C3E77E3C1800000003E7FA4
:10ECC000E3C1C1C1C1C163FFFE00000000FF00003D
:10ECD0003F3F3F3F3F3C3C3F3F3F3F3E3C3C3F3F51
:10ECE0003F373333333333333330383F3F3F3F3FA6
:10ECF000000000000000000000000010284444C490
:10ED0000040404C444442810000000000000000073
:10ED100000000000F008040404F4F404040484C4B3
:10ED2000E4670000000784848484848484040404E9
:10ED3000040408F00000FFF8F8F8F80707E4C68FAD
:10ED40001B3978F8F8F8C6873B39393939399B07C8
:10ED500006F8F8F8F8FF00003F3F3F3F3F3C3C3FDC
:10ED60003F3F3F3E3C3C3F3F3F373333333333330A
:10ED70003330383F3F3F3F3F0000000000000000BD
:10ED800000000010284444C4040404C4444428106F
:10ED9000000000000000000000000000F0C8C4C433
:10EDA000C43434C4C4C4440424A7C0C0C0C7444449
:10EDB0004444444444C4C4C4C4C4C8F00000FFFF75
:10EDC000FFFFFF0000E3C1881C3E7FFFFFFFC18003
:10EDD0003C3E3E3E3E3E9C0001FFFFFFFFFF000029
:10EDE0003F3F3F3F3F3C3C3F3F3F3F3E3C3C3F3F40
:10EDF0003F373333333333333330383F3F3F3F3F95
:10EE0000000000000000000000000010387C7CFCC6
:10EE1000FCFCFCFC7C7C38100000000000000000C2
:10EE200000000000F0F8FCFCFC0C0CFCFCFC7C3C42
:10EE30001C9FFFFFFFFF7C7C7C7C7C7C7CFCFCFCC3
:10EE4000FCFCF8F00000FFFFFFFFFF0000E3C188BB
:10EE50001C3E7FFFFFFFC1803C3E3E3E3E3E9C008D
:10EE600001FFFFFFFFFF00003F3F3F3F3F3C3C3FB4
:10EE70003F3F3F3E3C3C3F3F3F37333333333333F9
:10EE80003330383F3F3F3F3F0000000000000000AC
:10EE90000000000000000000000000000000000072
:10EEA0000000000000000000000000000000000062
:10EEB0000000000000000000000000000000000052
:10EEC0000000000000000000000000000000000042
:10EED0000000000000000000000000000000000032
:10EEE00000000000000000000000000000FCFA0626
:10EEF0000606060606066696961626060686F68612
:10EF000006060686464686C60606C60686464606A1
:10EF10000686F6860606060606060606FAFC003F84
:10EF20005F606060606060606468696966606060BE
:10EF30006768686060676868646F60606F61606080
:10EF400060606060676868606060606060605F3FCC
:10EF500000FCFA06E6C6860606066696961626069D
:10EF60000686F68606060686464686C60606C60651
:10EF7000864646060686F6860606060686C6E60621
:10EF8000FAFCFE3F5FE0EFE7E3E1E0E0E4E8E9E917
:10EF9000E6E0E0E0E7E8E8E0E0E7E8E8E4EFE0E02A
:10EFA000EFE1E0E0E0E0E0E0E7E8E8E0E0E1E3E72F
:10EFB000EFE0DFBF7FFF0305F9F9F9F9F9F9996986
:10EFC00069E9D9F9F9790979F9F9F979B9B97939A1
:10EFD000F9F939F979B9B9F9F9790979F9F9F9F951
:10EFE000F9F9F9F90503FFFFC0A09F9F9F9F9F9F1D
:10EFF0009B979696999F9F9F9897979F9F98979773
:10F000009B909F9F909E9F9F9F9F9F9F9897979F4A
:10F010009F9F9F9F9F9FA0C0FFFCFA0606060606C3
:10F0200006060606066696961626060686F68606E0
:10F030000606068686860606068606868606060670
:10F040000606060606060606FAFC003F5F606060DC
:10F050006060606060606064686969666060606785
:10F0600068686060676868686760607F656464633B
:10F07000606060606060606060605F3F00FCFA0636
:10F08000E6C6860606060606066696961626060650
:10F0900086F68606060606868686060606860686A0
:10F0A000860606060606060686C6E606FAFCFE3F45
:10F0B0005FE0EFE7E3E1E0E0E0E0E0E4E8E9E9E693
:10F0C000E0E0E0E7E8E8E0E0E7E8E8E8E7E0E0FFE4
:10F0D000E5E4E4E3E0E0E0E0E0E1E3E7EFE0DFBF28
:10F0E0007FFF0305F9F9F9F9F9F9F9F9F99969696E
:10F0F000E9D9F9F9790979F9F9F9F9797979F9F920
:10F10000F979F97979F9F9F9F9F9F9F9F9F9F9F9EF
:10F110000503FFFFC0A09F9F9F9F9F9F9F9F9F9B57
:10F12000979696999F9F9F9897979F9F9897979745
:10F13000989F9F809A9B9B9C9F9F9F9F9F9F9F9F15
:10F140009F9FA0C0FFF0F8FC1E0E0E1EFCF8F0FF03
:10F15000FFFF00000000FFFFFF070F1F3C38383C97
:10F160001F0F0780C0E0F0783C1EFEFEFE03030187
:10F1700000000000FFFFFF000000000000003F3F14
:10F180003FF8FCFE1E0E0E9EFEFCF8000080E0F82C
:10F19000FE3F0F03003C3E3F3F3B38383838381CB9
:10F1A0001E1E0E0E0E1EFEFCF80000001C1C1C3E57
:10F1B000FFF7E31C3C3C3838383C3F1F0FFEFEFE97
:10F1C00000000000FEFEFE070F1F1C1C1C1CFFFFA2
:10F1D000FF000000000000003F3F3FFEFEFE0E0E5D
:10F1E0000E0E0E0E0E0F0F0F0E0E0E1EFEFCF8383A
:10F1F00038383838383C3F1F0FFCFEFE0E0E0E0E1E
:10F200001E1E1CFFFFFF1C1C1C1CFCFCF81F3F3FAC
:10F21000383838383F3F1F0E0E0E0E0E0E0EFEFE13
:10F22000FC000000C0F0FC3F0F030100003F3F3F27
:10F230000000000000F8FCFE1E0E0E1EFEFCF8E3AF
:10F24000F7FF3E1C1C3EFFF7E30F1F3F3C38383CE6
:10F250003F1F0FFCFEFE0E0E0E0EFEFEFC0F1F1FCC
:10F260001C1C1C1CFFFFFF183838383838383F3F4B
:10F270001FF8FCFE1E0E0E1EFEFCF8FFFFFF8000B6
:10F280000080FFFFFF01030707070707070301804F
:10F29000C0E0F0783C1EFEFEFE030301000000000B
:10F2A000FFFFFF00000000000000070707F8FCFE5A
:10F2B0001E0E0E1EFEFCF8C0E0F0783C1E0F070389
:10F2C00001070707070707070707071C1E1E0E0E83
:10F2D0000E1EFEFEFC8080800006068FFFFFF903F5
:10F2E000070707070707070703FEFEFE00000000E9
:10F2F000FEFEFE03070F0E0E0E0EFFFFFF000000C6
:10F3000000000000070707FEFEFE0E0E0E0E0E0E9A
:10F310000E07070707070707FFFFFE07070707078F
:10F320000707070703FCFEFE0E0E0E0E1E1E1CFF37
:10F33000FFFF07070707FFFFFE030707070707078A
:10F340000707030E0E0E0E0E0ECEFEFE3C0000C092
:10F35000F0FC3F0F0300000000070707000000005B
:10F3600000F8FCFE1E0E0E1EFEFCF8F9FFFF8F06D5
:10F37000068FFFFFF901030707070707070301FCD3
:10F38000FEFE0E0E0E0EFEFEFC0307070707070724
:10F39000FFFFFF0307070707070707070300000032
:10F3A000000000000000000000000000000000005D
:10F3B000000000000000000000000000808080804D
:10F3C000808080808080808080808080808080803D
:10F3D000808080808080808080808080808080802D
:10F3E0008080808080808080808080808080FF809E
:10F3F0008080808482BE80808080FF80808080B218
:10F40000AAAAA4808080FF80808080A2A2AA948083
:10F410008080FF80808080868888BE808080FF809A
:10F42000FF808080AEAAAA9280808080FF8080804A
:10F43000BCAAAABA80808080FF80808082B28A863F
:10F4400080808080FF808080BEAAAABE808080806D
:10F45000FF80FF808080AEAAAA9E80808080FF808F
:10F460008084BE809CA2A29C8080FF80808084BE1D
:10F470008084BE808080FF808084BE80A4B2AAA4E5
:10F480008080FF80FF808084BE80A2A2AA948080BA
:10F49000FF808084BE80868888BE8080FF808084D4
:10F4A000BE80AEAAAA928080FF808084BE80BCAA63
:10F4B000AABA8080FF80FF808084BE8082B28A8664
:10F4C0008080FF808084BE80BEAAAABE8080FF802C
:10F4D0008084BE80AEAAAA9E8080FF80A2B2AAA429
:10F4E000809CA2A29C80FF80FF80B2AAAAA48080F8
:10F4F0008482BE80FF80B2AAAAA480B2AAAAA480F5
:10F50000FF80B2AAAAA480A2A2AA9480FF80B2AA75
:10F51000AAA480868888BE80FF80FF80B2AAAAA4A1
:10F5200080AEAAAA9280FF80B2AAAAA480BCAAAA8E
:10F53000BA80FF80B2AAAAA48082B28A8680FF80A5
:10F54000B2AAAAA480BEAAAABE80FF80FF80B2AAE7
:10F55000AAA480AEAAAA9E80FF80A2A2AA94809CA0
:10F56000A2A29C80FF80A2A2AA94808084BE8080F8
:10F57000FF80A2A2AA9480B2AAAAA480FF80FF80E2
:10F58000A2A2AA9480A2A2AA9480FF80A2A2AA9476
:10F5900080868888BE80FF80A2A2AA9480AEAAAA94
:10F5A0009280FF80A2A2AA9480BCAAAABA80FF80FF
:10F5B000000000000000002F0000000300030054C2
:10F5C0003F147E152E2A7F2A3A22152A5422122D04
:10F5D0002911280003000000001C224100004122E4
:10F5E0001C00000C0C000008083E08080040300019
:10F5F0000008080808080040000000403008060124
:10F600003E4749713E0402017F0062514946002293
:10F6100041493E000708087F004F494931003C4AF4
:10F620004930000161190700364949360026494929
:10F630007E00000012000000403400000814224147
:10F6400000141414141400412214080229050200A5
:10F650000E152B2D123E0909093E3F2525251A1EA0
:10F66000212121123F2121211E3F252525213F094E
:10F670000909011E2121293A3F0404043F3F0000EB
:10F680000000214141413F3F0C1221003F2020203A
:10F69000003F060C063F3F030E183F1E2121211E8E
:10F6A0003F090909061E2129112E3F0909192612B1
:10F6B0002529120001013F01011F2020203F030CDA
:10F6C000300C031F301C301F22140814220304388E
:10F6D00004033129252321007F4141000106083020
:10F6E000400041417F00040201020440404040408C
:10F6F0000001020000102A2A2A3C3F242424181C5E
:10F7000022222222182424243F1C2A2A2A2C087E62
:10F710000901004C5252523C3F040404383D0000A1
:10F7200000002040403D003F081422001F20202000
:10F73000003C023C023C3E0402023C1C2222221CF1
:10F740007E1212120C0C1212127E3E0404020214DB
:10F75000262A3214041F2424001E2020203E0618CE
:10F760002018061E201C201E24181824004E50505D
:10F77000503E22322A2622083641410000007F00F6
:10F780000041413E0800180408100C000000000071
:10F790000000000000000000000000000000000069
:10F7A00000000000000000000000C02010D0121572
:10F7B0001D111D1512101020C0FF80809F848A919A
:10F7C0008086A9A9BE8080FFC02010D012151D110F
:10F7D0001D1512101020C0FFF0F0EFF4FAE1F0F662
:10F7E000D9D9CEF0F0FFC02010D012151D111D1573
:10F7F00012101020C0FFFEFEE1FAF4EFFEF8D7D79A
:10F80000C0FEFEFFC0E0D010D2D5DDD1DDD5D2D014
:10F81000D0E0C0FFFFFFE0FBF5EEFFF9D6D6C1FF59
:10F82000FFFFC0E0F030F2F7FFFFFFF7F2F0F0E08B
:10F83000C0FFFFFFE0FBF5EEFFF9D6D6C1FFFFFFEB
:10F840000F3FFFFCF0C00000C0F0FCFF3F0F0000C6
:10F850000000030F3F7E7E3F0F03000000005500B5
:10F86000810081008100412214000000006A000034
:10F870000000000001020468000000000316504070
:10F8800000000000000040501603000000000105C9
:10F8900014404014050100000000FFFFFFC7C7C768
:10F8A000C7C7EFFFFE7C0000007F7F7F01010103DF
:10F8B000071F7F7C7800000000804040202020400F
:10F8C000408000000000000E31404E919191404078
:10F8D000310E000000008060100808E42424C408F1
:10F8E000081060800007182040409F8385984040A2
:10F8F00020180700000000000000000000000000C9
:10F9000000000000000000000000000000000000F7
:10F9100000000000000000000000000000000000E7
:10F9200000000000000000000000000000000000D7
:10F9300000000000000000000000000000000000C7
:10F9400000000000000000000000000000000000B7
:10F9500000000000000000000000000000000000A7
:10F960000000000000000000000000000000000097
:10F970000000000000000000000000000000000087
:10F980000000000000000000000000000000000077
:10F990000000000000000000000000000000000067
:10F9A0000000FE02FA0A0A0A0A0A0A0A0A0A0A0AEF
:10F9B0000A0A0A0A0A0A0A0A0A0A0A0A0A0A0A0AA7
:10F9C0000A0A0A0A0A0A0A0A0A0A0A0A0A8A8A8A17
:10F9D0008A8A8A8A8A8A8A8A8ACACACACACACACAC7
:10F9E000CACACACAEAEAEAEAEAEAEAEAEAEAEAEAF7
:10F9F000FAFAFAFAFAFAFA02FE7F405F58585858B3
:10FA000058585C5C5C5C5C5C5C5C5C5C5C5C5E5E3A
:10FA10005E5E5E5E5E5E5E5E5E5F5F5F5F5F5F5FFF
:10FA20005F5F5F5F5F5F5F5F5F5F5F5F5F5F5F5FE6
:10FA30005F5F5F5F5F5F5F5F5F5F5F5F5F5F5F5FD6
:10FA40005F5F5F5F5F5F5F5F5F5F5F5F5F5F407FC5
:10FA500080808080808080808080808C8C8C9EBF25
:10FA6000BFBFBF9292928482898595B59585898220
:10FA7000848080888494B49484888080808080800E
:10FA800090B090808080808080808080A080808006
:10FA900080809F909F80969589809F958A8080BF67
:10FAA000A1A1A1A1A18780808080BFA1A1A1818106
:10FAB0009F80808080BFA1818181A1BF8080808064
:10FAC0009F8181A1A1A1BF8080808087A1A1A1A1E8
:10FAD000A1BF80808080B1A1A1A1A1A1BF808080B1
:10FAE00080BCA0A1A1A1A1BF80808080BFA0A0A058
:10FAF000A1A1BF80808080BFA1A1A0A0A0BF808065
:10FB00008080BFA1A1A1A1A0BC80808080BFA1A155
:10FB1000A1A1A1B18080808C92A1A1A181828C80C1
:10FB200080808C92A18181A1928C8080808C828146
:10FB3000A1A1A1928C8080808092A1A1A1A1928C90
:10FB40008080808C90A0A1A1A1928C8080808C92DA
:10FB5000A1A0A0A1928C8080808C92A1A1A1A09054
:10FB60008C8080808C92A1A1A1A192808080BE898E
:10FB700089BE80B8A8BF80B888406070787C7E7CE1
:10FB80007870604002060E1E3E7E3E1E0E0602008B
:10FB90000000000000000000000080808080808065
:10FBA0008080808080808080808080808080809E37
:10FBB0009EBFBFAFB7BBBDAFB7BBBDAFB7BBBDAFE0
:10FBC000B7BBBDBF9E92A1A1A1B1B9BDAFB7BBBD2F
:10FBD000AFB7BBBDAFB7BBBDBF9E92A1A1A1A1A155
:10FBE000A1A1B1B9BDAFB7BBBDAFB7BBBDBF9E9201
:10FBF000A1A1A1A1A1A1A1A1A1A1A1B1B9BDAFB78D
:10FC0000BBBDBF9E92A1A1A1A1A1A1A1A1A1A1A1A2
:10FC1000A1A1A1A1B1B9BDBF9E92A1A1A1A1A1A184
:10FC2000A1A1A1A1A1A1A1A1A1A1A1A1BF9E92A1B8
:10FC3000A1B1A9A5A3B1A9A5A3B1A9A5A3B1A9A53E
:10FC4000A3BFFCFE9393FEFC8098BCE6E6BCFFFFDE
:10FC50008080FEFE988C8698BEB7B3B3B383B0BCE9
:10FC6000BFB7B3BB9F86B0BBBBBFB7870000000068
:10FC70000000000000000000000000000000000084
:10FC80000000000000000000000000000000000074
:10FC90000000000000000000000000000000000064
:10FCA0000000000000000000000000000000000054
:10FCB0000000000000000000000000000000000044
:10FCC0000000000000000000000000000000000034
:10FCD000000000000000000000007EFFC3FF7E0067
:10FCE0000607FFFFE7F3FBDFCEC3DBDBFF7E0F1F63
:10FCF00018FFFFDFDFDBFB737EFFDBFB7103F3FB32
:10FD00001F0F66FFDBFF660EDFDBFFFE000000005B
:10FD100000000000000000000000000000000406D9
:10FD2000FF060400E3F3FBDFCFC70406FF06040071
:10FD3000FFFF1818FFFF0406FF0604000303FFFF80
:10FD4000030300000000000000111B1511110A043C
:10FD5000111B1F1F1F0E0446756E6B2D5369676EB6
:10FD6000616C3A0050726F66692F45636F2F4E5A6F
:10FD7000004465636F64657235362F35370048651A
:10FD80006C6C69676B6569743A00416B6B756C618B
:10FD900064756E673A00525353492D4261636B3A62
:10FDA0000048616E647265676C6572005A776569B8
:10FDB0007465204C6F6B004C6F6B6164726573737C
:10FDC000650046756E6B74696F6E656E00FEFF01AF
:10FDD000FFFE7FFF80FF7F536F6674776172653A25
:10FDE000004164722D46756E6B3A00566572626909
:10FDF0006E64656E004C6F6B2D5375636865002DE6
:10FE00002D2D2D2D2D2D2D004B6F6E747261737461
:10FE10000056657273696F6E0050726F6772616D24
:10FE2000004C6F6B7761686C00537461747573007C
:10FE3000526573657400536574757000200020006E
:10FE400020002000200056657262696E64756E673E
:10FE5000206D69742043445A002020206E6575206F
:10FE6000617566626175656E2E00204C6173742049
:10FE700065696E7374656C6C656E00447265686B61
:10FE80006E6F706620647275652D006475726368AC
:10FE90007A756675656872656E2E004C6F6B61646D
:10FEA00072657373652050726F67004465636F6499
:10FEB00065722050726F6772616D00636B656E2CA6
:10FEC00020756D2065696E656E0048616E647265AF
:10FED000676C65722D5479700049324320616B74F0
:10FEE00075656C6C3A200050726F6772616D6D6958
:10FEF0006572656E002020202020202020202020F8
:10FF000020004932432D416472657373653A0041A4
:10FF1000647265737365206E65753A004C6F6B6132
:10FF20006472657373653A0048617570746D656ECF
:10FF30007565005A7765697465204C6F6B004C6F6E
:10FF40006B7765636873656C004C6F6B20737563CA
:10FF500068656E0046756E6B74696F6E656E0049FC
:10FF600032432D5374617475730056657262696E05
:10FF700064656E0052616E67696572656E004175F9
:10FF8000746F66616872740043445A2D49443A2084
:10FF9000005A656E7472616C65004B6F6E747261AD
:10FFA000737400426567696E6E3A004C6F6B7761DF
:10FFB000686C004272656D736500204F4B20200015
:10FFC0004164723A2000585858582000456E6465C4
:10FFD0003A00436F64653A00576572743A005245BF
:10FFE000534554005365747570004572726F72000A
:10FFF0005265736574004164723A003F3F3F0000F0
:020000040001F9
:100000000301116F0A0E111901E0A3D100019F0530
:1000100001E085D09F6B070ED66F6000D8F3D7F054
:10002000010E8DECFFF0C00ED66FFF0ED76F060EDF
:10003000D86FD96B010EDA6FDB6BDC6BDD6BDE6BBF
:10004000DF6B68ECF1F0010E0101656F00019A05AC
:1000500004E1010E0101636F5BD0630EBC6FE50E1E
:10006000BD6F070EBE6F020EBF6FC06BC16B050E7A
:10007000C26FC36BC46BC56BC66BC76B6000D8F334
:10008000C8F0B3ECEAF0630EBC6FE50EBD6F070E6F
:10009000BE6F020EBF6FC06B090EC16F050EC26F3F
:1000A000C36BC46BC56BC66BC76B6000D8F3C8F07D
:1000B000B3ECEAF0630EBC6FE50EBD6F070EBE6FCA
:1000C000020EBF6FC06B120EC16F050EC26FC36B05
:1000D000C46BC56BC66BC76B6000D8F3C8F0B3ECDC
:1000E000EAF0630EBC6FE50EBD6F070EBE6F020E29
:1000F000BF6FC06B1A0EC16F050EC26FC36BC46BAE
:10010000C56BC66BC76B6000D8F3C8F0B3ECEAF000
:10011000010E01016B6F686F676FB0ECFAF00101BF
:10012000850526E1010EC86F2B5103E1320E2A5DD1
:100130000EE345040CE1456A2A6B2B6B010E656FDB
:1001400000019A0519E1010E0101636F15D02B51D1
:1001500003E11E0E2A5D10E345500EE1010E456ECF
:100160002A6B2B6B010E656F00019A05ECE004D041
:100170002A6B2B6BC86BF6D7010184051AE1010EBF
:10018000C76F295103E1460E285D07E3830505E1AA
:10019000836B0CD0010E6B6F10D0295103E1140E4C
:1001A000285D0BE3835109E1010E836F286B296BF6
:1001B000F1D7286B296BC76BEDD70001875103E09E
:1001C000010158055DE10001865103E0010153057D
:1001D00057E10001855103E00101510551E10101A1
:1001E000650522E100019A0509E16000D8F1D6F029
:1001F0006000DCF1D7F026ECC6F008D06000D8F142
:10020000D6F06000DCF1D7F023ECCDF076C078F0CA
:1002100077C079F06000E0F1BBF06000E4F1BCF081
:10022000E3ECF1F00101656B63050EE16000C0F1E4
:10023000D6F06000C4F1D7F026ECC6F070C072F0C2
:1002400071C073F00101636B6B0509E100018F510F
:10025000A6ECE8F060003CF23FF001016B6B680532
:1002600005E169510AECFAF00101686B670508E1E4
:1002700000018D51E7ECFAF08DC08EF00101676B43
:10028000590521E15A51000187191BE001015A0566
:100290000EE10001D76BD66B100ED86F020ED96F2E
:1002A000080E42ECD1F0010E0101C96F06D0010E1B
:1002B00000019F6F0101C96B586B2C6B2D6B5AC1EC
:1002C00087F00101596B52051FE13D50000185196E
:1002D00019E03D040DE1D76BD66B100ED86F020EFE
:1002E000D96F070E42ECD1F0010E0101C96F05D0A4
:1002F000010E9F6F0101C96B516B2C6B2D6B600060
:10030000F4F085F00101526B5405D8A41200555148
:10031000000186191BE0010155050EE10001D76BB4
:10032000D66B100ED86F020ED96F090E42ECD1F0C9
:10033000010E0101C96F06D0010E00019F6F01017E
:10034000C96B536B2C6B2D6B55C186F00101546B3F
:1003500012000B0E111927E100019F0513E1070E92
:10036000D66F6000D8F3D7F0010E8DECFFF06A0E67
:10037000EA6FFE0EEB6F110EEC6FF7ECFBF09F6B6C
:10038000010E9E6F0101670504E000019E05D8A4DF
:10039000120000018D511EECFBF08DC08EF09E6BA3
:1003A0000101676B12000C0E111901E0D3D1100E80
:1003B0000F6F030E106F6C0E006F016F026F036FF3
:1003C00000019F0501E0BDD0210EBC6FAF0EBD6FD7
:1003D000440EBE6F050EBF6FC06B60003CFCC1F0E9
:1003E000600040FCC2F0C36BC46B010EC56FC66BEE
:1003F000C76B6000D8F3C8F0B3ECEAF0210EBC6F15
:10040000AF0EBD6F440EBE6F050EBF6F0E0EC06FF8
:1004100060003CFCC1F0600040FCC2F0C36BC46BE8
:10042000010EC56FC66BC76B6000D8F3C8F0B3ECA4
:10043000EAF0630EBC6FE50EBD6F070EBE6F020ED5
:10044000BF6F6C0EC06F03010F510C0F0001C16F25
:1004500003011051030F0001C26FC36BC46B010E87
:10046000C56FC66BC76B6000D8F3C8F0B3ECEAF099
:10047000630EBC6FE50EBD6F070EBE6F020EBF6F41
:100480006C0EC06F03010F51150F0001C16F030106
:100490001051030F0001C26FC36BC46B010EC56F17
:1004A000C66BC76B6000D8F3C8F0B3ECEAF0630E1C
:1004B000BC6FE50EBD6F070EBE6F020EBF6F6C0EF8
:1004C000C06F03010F511E0F0001C16F03011051D6
:1004D000030F0001C26FC36BC46B010EC56FC66B07
:1004E000C76B6000D8F3C8F0B3ECEAF0630EBC6FE2
:1004F000E50EBD6F070EBE6F020EBF6F6C0EC06FB4
:1005000003010F51270F0001C16F03011051030FA9
:100510000001C26FC36BC46B010EC56FC66BC76BA6
:100520006000D8F3C8F0B3ECEAF03E0EEA6FFF0EBD
:10053000EB6F0B0EEC6FF7ECFBF09F6B010E9E6FF9
:10054000986F0101650504E000019E0501E0F7D008
:10055000E80E0001765D030E77591CE3270EBE6F8F
:10056000100EBD6F6000D8F1BBF06000DCF1BCF094
:10057000D0ECFFF06000ECF2C0F06000F0F2C1F0EF
:10058000030EC36FE80EC26F1DECFFF0C051600F89
:100590000301006F0001775103E1640E765D1BE3F8
:1005A000030EBE6FE80EBD6F6000D8F1BBF06000B7
:1005B000DCF1BCF0D0ECFFF06000ECF2C0F06000C9
:1005C000F0F2C1F0C36B640EC26F1DECFFF0C051BE
:1005D000600F0301016F0001775103E10A0E765DA0
:1005E0001AE3BE6B640EBD6F6000D8F1BBF0600013
:1005F000DCF1BCF0D0ECFFF06000ECF2C0F0600089
:10060000F0F2C1F0C36B0A0EC26F1DECFFF0C051D7
:10061000600F0301026F6000D8F1BBF06000DCF1F5
:10062000BCF00001BE6B0A0EBD6FD0ECFFF0BB51F9
:10063000600F0301036F630E0001BC6FE50EBD6F19
:10064000070EBE6F020EBF6F600000FCC0F003011A
:100650000F510C0F0001C16F03011051030F000176
:10066000C26FC36BC46B010EC56FC66BC76B6000F6
:10067000D8F3C8F0B3ECEAF0630EBC6FE50EBD6FC3
:10068000070EBE6F020EBF6F600004FCC0F00301D6
:100690000F51150F0001C16F03011051030F00012D
:1006A000C26FC36BC46B010EC56FC66BC76B6000B6
:1006B000D8F3C8F0B3ECEAF0630EBC6FE50EBD6F83
:1006C000070EBE6F020EBF6F600008FCC0F0030192
:1006D0000F511E0F0001C16F03011051030F0001E4
:1006E000C26FC36BC46B010EC56FC66BC76B600076
:1006F000D8F3C8F0B3ECEAF0630EBC6FE50EBD6F43
:10070000070EBE6F020EBF6F60000CFCC0F003014D
:100710000F51270F0001C16F03011051030F00019A
:10072000C26FC36BC46B010EC56FC66BC76B600035
:10073000D8F3C8F0B3ECEAF09E6B0101656B410E93
:100740000001BB6F140EBC6F985198ECF9F00101D9
:10075000656F1200640E111901E0F5D200019F05CA
:1007600014E1070ED66F6000D8F3D7F0010E8DECC0
:10077000FFF0280EEA6FFF0EEB6F0B0EEC6FF7EC3D
:10078000FBF09F6B010E9E6F946F960501E1C6D240
:100790009E0501E1C3D21200210EE96FFE0EEA6F41
:1007A000080EEB6F600094F2ECF0020EAEECE0F09D
:1007B0006C0EBC6FFC0EBD6F5A0EBE6F010EBF6F8C
:1007C000C06BC16B040EC26FC36BC46BC56BC66BD1
:1007D000C76B6000D8F3C8F0B3ECEAF0190ED66F1F
:1007E000FE0ED76F080ED86F030ED96F040EDA6FA6
:1007F000DB6BDC6BDD6BDE6B010EDF6FF1ECD4F0DD
:100800006C0EBC6FFC0EBD6F660EBE6F010EBF6F2F
:10081000C06BC16B050EC26FC36BC46BC56BC66B7F
:10082000C76B6000D8F3C8F0B3ECEAF0C20ED66F25
:10083000FD0ED76F0B0ED86F030ED96F050EDA6F52
:10084000DB6BDC6BDD6BDE6B010EDF6FF1ECD4F08C
:100850006C0EBC6FFC0EBD6F660EBE6F010EBF6FDF
:10086000C06BC16B060EC26FC36BC46BC56BC66B2E
:10087000C76B6000D8F3C8F0B3ECEAF0360ED66F61
:10088000FE0ED76F060ED86F030ED96F060EDA6F05
:10089000DB6BDC6BDD6BDE6B010EDF6FF1ECD4F03C
:1008A0006C0EBC6FFC0EBD6F660EBE6F010EBF6F8F
:1008B000C06BC16B070EC26FC36BC46BC56BC66BDD
:1008C000C76B6000D8F3C8F0B3ECEAF0290ED66F1E
:1008D000FE0ED76F070ED86F030ED96F070EDA6FB3
:1008E000DB6BDC6BDD6BDE6B010EDF6FF1ECD4F0EC
:1008F00025D2190EE96FFE0EEA6F080EEB6F60004D
:1009000094F2ECF0030EAEECE0F06C0EBC6FFC0E5B
:10091000BD6F5A0EBE6F010EBF6FC06BC16B020E72
:10092000C26FC36BC46BC56BC66BC76B6000D8F37B
:10093000C8F0B3ECEAF0210ED66FFE0ED76F080EAA
:10094000D86F030ED96F020EDA6FDB6BDC6BDD6BD9
:10095000DE6B010EDF6FF1ECD4F06C0EBC6FFC0EA1
:10096000BD6F5A0EBE6F010EBF6FC06BC16B050E1F
:10097000C26FC36BC46BC56BC66BC76B6000D8F32B
:10098000C8F0B3ECEAF0C20ED66FFD0ED76F0B0EB7
:10099000D86F030ED96F050EDA6FDB6BDC6BDD6B86
:1009A000DE6B010EDF6FF1ECD4F052D7C20EE96FAF
:1009B000FD0EEA6F0B0EEB6F600094F2ECF0040E8C
:1009C000AEECE0F06C0EBC6FFC0EBD6F5A0EBE6F4D
:1009D000010EBF6FC06BC16B020EC26FC36BC46BE5
:1009E000C56BC66BC76B6000D8F3C8F0B3ECEAF018
:1009F000210ED66FFE0ED76F080ED86F030ED96F7B
:100A0000020EDA6FDB6BDC6BDD6BDE6B010EDF6F12
:100A1000F1ECD4F06C0EBC6FFC0EBD6F5A0EBE6FC5
:100A2000010EBF6FC06BC16B030EC26FC36BC46B93
:100A3000C56BC66BC76B6000D8F3C8F0B3ECEAF0C7
:100A4000190ED66FFE0ED76F080ED86F030ED96F32
:100A5000DA6FDB6BDC6BDD6BDE6B010EDF6FF1ECF5
:100A6000D4F06C0EBC6FFC0EBD6F5A0EBE6F010E43
:100A7000BF6FC06BC16B060EC26FC36BC46BC56B1F
:100A8000C66BC76B6000D8F3C8F0B3ECEAF0F6D6DB
:100A9000360EE96FFE0EEA6F060EEB6F600094F201
:100AA000ECF0050EAEECE0F06C0EBC6FFC0EBD6F12
:100AB0005A0EBE6F010EBF6FC06BC16B020EC26FCC
:100AC000C36BC46BC56BC66BC76B6000D8F3C8F053
:100AD000B3ECEAF0210ED66FFE0ED76F080ED86F7A
:100AE000030ED96F020EDA6FDB6BDC6BDD6BDE6B36
:100AF000010EDF6FF1ECD4F06C0EBC6FFC0EBD6F1D
:100B00005A0EBE6F010EBF6FC06BC16B030EC26F7A
:100B1000C36BC46BC56BC66BC76B6000D8F3C8F002
:100B2000B3ECEAF0190ED66FFE0ED76F080ED86F31
:100B3000030ED96FDA6FDB6BDC6BDD6BDE6B010EE6
:100B4000DF6FF1ECD4F06C0EBC6FFC0EBD6F5A0E73
:100B5000BE6F010EBF6FC06BC16B040EC26FC36B63
:100B6000C46BC56BC66BC76B6000D8F3C8F0B3EC41
:100B7000EAF0C20ED66FFD0ED76F0B0ED86F030EC4
:100B8000D96F040EDA6FDB6BDC6BDD6BDE6B010E95
:100B9000DF6FF1ECD4F06C0EBC6FFC0EBD6F5A0E23
:100BA000BE6F010EBF6FC06BC16B070EC26FC36B10
:100BB000C46BC56BC66BC76B6000D8F3C8F0B3ECF1
:100BC000EAF084D6290EE96FFE0EEA6F070EEB6F8E
:100BD000600094F2ECF0060EAEECE0F06C0EBC6F30
:100BE000FC0EBD6F5A0EBE6F010EBF6FC06BC16BA6
:100BF000020EC26FC36BC46BC56BC66BC76B600064
:100C0000D8F3C8F0B3ECEAF0210ED66FFE0ED76F22
:100C1000080ED86F030ED96F020EDA6FDB6BDC6B38
:100C2000DD6BDE6B010EDF6FF1ECD4F06C0EBC6F90
:100C3000FC0EBD6F5A0EBE6F010EBF6FC06BC16B55
:100C4000030EC26FC36BC46BC56BC66BC76B600012
:100C5000D8F3C8F0B3ECEAF0190ED66FFE0ED76FDA
:100C6000080ED86F030ED96FDA6FDB6BDC6BDD6BB0
:100C7000DE6B010EDF6FF1ECD4F06C0EBC6FFC0E7E
:100C8000BD6F5A0EBE6F010EBF6FC06BC16B040EFD
:100C9000C26FC36BC46BC56BC66BC76B6000D8F308
:100CA000C8F0B3ECEAF0C20ED66FFD0ED76F0B0E94
:100CB000D86F030ED96F040EDA6FDB6BDC6BDD6B64
:100CC000DE6B010EDF6FF1ECD4F06C0EBC6FFC0E2E
:100CD000BD6F5A0EBE6F010EBF6FC06BC16B050EAC
:100CE000C26FC36BC46BC56BC66BC76B6000D8F3B8
:100CF000C8F0B3ECEAF0360ED66FFE0ED76F060ED4
:100D0000D86F030ED96F050EDA6FDB6BDC6BDD6B12
:100D1000DE6B010EDF6FF1ECD4F010D09451010ABC
:100D200001E13AD5030A01E1E4D5010A01E13ED629
:100D3000070A01E1ADD6010A01E144D794C095F05C
:100D4000966B9E6B1200650E111964E100019F0500
:100D50003DE1070ED66F6000D8F3D7F0010E8DECA1
:100D6000FFF0AB0EEA6FFF0EEB6F080EEC6FF7ECC7
:100D7000FBF01C0ED66FFF0ED76F0C0ED86FD96B21
:100D8000020EDA6FDB6BDC6BDD6BDE6BDF6B68EC4E
:100D9000F1F0B00506E15A0ED66F480EDAECEEF02F
:100DA00011D0020EB01906E15A0ED66F200EDAEC01
:100DB000EEF008D0030EB01905E15A0ED66F200EE2
:100DC000DAECEEF09F6B010E9E6F986F01016505E6
:100DD00003E000019E0513E16000D8F1D6F0600049
:100DE000DCF1D7F00A0E0001D86F040ED96F600055
:100DF00094F2DAF06EECC3F09E6B0101656B410E6C
:100E00000001BB6F140EBC6F985198ECF9F0010112
:100E1000656F12006D0E111901E092D200019F055D
:100E200001E030D1070ED66F6000D8F3D7F0010E85
:100E30008DECFFF0630EEA6FFF0EEB6F070EEC6FA9
:100E4000F7ECFBF0905145E08A0ED66FFD0ED76FA0
:100E50000C0ED86FD96B020EDA6FDB6BDC6BDD6BBF
:100E6000DE6B010EDF6FF1ECD4F0570ED66FFD0E86
:100E7000D76F0D0ED86FD96B030EDA6FDB6BDC6B9F
:100E8000DD6BDE6B010EDF6FF1ECD4F0E10ED66F9F
:100E9000FD0ED76F0A0ED86FD96B040EDA6FDB6BBD
:100EA000DC6BDD6BDE6B010EDF6FF1ECD4F0960EC8
:100EB000D66FFD0ED76F0B0ED86FD96B050EDA6F9C
:100EC000DB6BDC6BDD6BDE6B010EDF6FF1ECD4F006
:100ED00044D0880ED66FFF0ED76F090ED86FD96B2E
:100EE000020EDA6FDB6BDC6BDD6BDE6B010EDF6F2E
:100EF000F1ECD4F0D90ED66FFE0ED76F0E0ED86F70
:100F0000D96B030EDA6FDB6BDC6BDD6BDE6B010E16
:100F1000DF6FF1ECD4F0020ED66FFF0ED76F0D0E1F
:100F2000D86FD96B040EDA6FDB6BDC6BDD6BDE6BBD
:100F3000010EDF6FF1ECD4F05F0ED66FFF0ED76FAE
:100F40000B0ED86FD96B050EDA6FDB6BDC6BDD6BCC
:100F5000DE6B010EDF6FF1ECD4F07E0ED66FFD0E6E
:100F6000D76F0C0ED86FD96B060EDA6FDB6BDC6BAC
:100F7000DD6BDE6B010EDF6FF1ECD4F0D70ED66FB8
:100F8000FD0ED76F0A0ED86FD96B070EDA6FDB6BC9
:100F9000DC6BDD6BDE6B010EDF6FF1ECD4F0C70EA6
:100FA000D66FFF0ED76F050ED86F4F0ED96F020E9A
:100FB000DA6FDB6BDC6BDD6BDE6B010EDF6FF1EC90
:100FC000D4F0C70ED66FFF0ED76F050ED86F4F0E39
:100FD000D96F030EDA6FDB6BDC6BDD6BDE6B010E42
:100FE000DF6FF1ECD4F0C70ED66FFF0ED76F050E92
:100FF000D86F4F0ED96F040EDA6FDB6BDC6BDD6BD5
:10100000DE6B010EDF6FF1ECD4F0C70ED66FFF0E72
:10101000D76F050ED86F4F0ED96F050EDA6FDB6BE9
:10102000DC6BDD6BDE6B010EDF6FF1ECD4F0C70E15
:10103000D66FFF0ED76F050ED86F4F0ED96F060E05
:10104000DA6FDB6BDC6BDD6BDE6B010EDF6FF1ECFF
:10105000D4F0EE0ED66F020ED76F050ED86F4F0E7E
:10106000D96F070EDA6FDB6BDC6BDD6BDE6B010EAD
:10107000DF6FF1ECD4F09F6B010E0101766FB96F59
:10108000B86FB46F0001905101E191D001016E057C
:1010900023E1FC0E0001D66FFE0ED76F060ED86F4F
:1010A000430ED96F020EDA6FDB6BDC6BDD6BDE6B30
:1010B000DF6BF1ECD4F0600030F4D6F0600034F473
:1010C000D7F04F0ED86F020ED96FDA6BDB6BDC6B8B
:1010D000AFECC0F001016E6B730521E1FC0E000165
:1010E000D66FFE0ED76F060ED86F430ED96F030E64
:1010F000DA6FDB6BDC6BDD6BDE6BDF6BF1ECD4F09E
:101100006000D0F5D6F0D76B4F0ED86F030ED96FB5
:10111000DA6BDB6BDC6BAFECC0F00101736BB90514
:1011200021E1FC0E0001D66FFE0ED76F060ED86FC0
:10113000430ED96F040EDA6FDB6BDC6BDD6BDE6B9D
:10114000DF6BF1ECD4F060006CF1D6F0D76B4F0E92
:10115000D86F040ED96FDA6BDB6BDC6BAFECC0F0D1
:101160000101B96BAC0501E0C4D0FC0E0001D66FE3
:10117000FE0ED76F060ED86F430ED96F050EDA6FCD
:10118000DB6BDC6BDD6BDE6BDF6BF1ECD4F06000F6
:10119000B4F6D6F0D76B4F0ED86F050ED96FDA6B59
:1011A000DB6BDC6BAFECC0F00101AC6BA2D00101DA
:1011B000760521E1FC0E0001D66FFE0ED76F060EFC
:1011C000D86F430ED96F020EDA6FDB6BDC6BDD6B11
:1011D000DE6BDF6BF1ECD4F0600004F1D6F0D76B7E
:1011E0004F0ED86F020ED96FDA6BDB6BDC6BAFEC96
:1011F000C0F00101766BB8053FE1FC0E0001D66F2F
:10120000FE0ED76F060ED86F430ED96F030EDA6F3E
:10121000DB6BDC6BDD6BDE6BDF6BF1ECD4F0600065
:10122000D0F2D6F0D76B4F0ED86F030ED96FDA6BB2
:10123000DB6BDC6BAFECC0F0FC0ED66FFE0ED76F35
:10124000060ED86F430ED96F040EDA6FDB6BDC6BC2
:10125000DD6BDE6BDF6BF1ECD4F06000C4F2D6F036
:10126000D76B4F0ED86F040ED96FDA6BDB6BDC6B6C
:10127000AFECC0F00101B86BB4053BE1FC0E00011E
:10128000D66FFE0ED76F060ED86F430ED96F050EC0
:10129000DA6FDB6BDC6BDD6BDE6BDF6BF1ECD4F0FC
:1012A000AE0513E1BA0ED66FFF0ED76F060ED86FDC
:1012B0004A0ED96F050EDA6FDB6BDC6BDD6BDE6B14
:1012C000010EDF6FF1ECD4F012D0EA0ED66FFF0EF4
:1012D000D76F060ED86F490ED96F050EDA6FDB6B2C
:1012E000DC6BDD6BDE6B010EDF6FF1ECD4F0010126
:1012F000B46B8E05D8A41200FC0E0001D66FFE0E52
:10130000D76F060ED86F430ED96F060EDA6FDB6B00
:10131000DC6BDD6BDE6BDF6BF1ECD4F06000A0FA10
:10132000D6F06000A4FAD7F04F0ED86F060ED96F32
:10133000DA6BDB6BDC6BAFECC0F001018E6B120083
:101340006E0E111901E0F3D200019F0514E1070EA2
:10135000D66F6000D8F3D7F0010E8DECFFF0E70EEA
:10136000EA6FFE0EEB6F0E0EEC6FF7ECFBF09F6B6F
:10137000010E9E6F946F960501E1C7D29E0501E1B3
:10138000C4D21200710EE96FFD0EEA6F0D0EEB6F05
:10139000600094F2ECF0020EAEECE0F06C0EBC6F6C
:1013A000FC0EBD6F5A0EBE6F010EBF6FC06BC16BDE
:1013B000040EC26FC36BC46BC56BC66BC76B60009A
:1013C000D8F3C8F0B3ECEAF0640ED66FFD0ED76F19
:1013D0000D0ED86F030ED96F040EDA6FDB6BDC6B6A
:1013E000DD6BDE6B010EDF6FF1ECD4F06C0EBC6FC9
:1013F000FC0EBD6F660EBE6F010EBF6FC06BC16B82
:10140000050EC26FC36BC46BC56BC66BC76B600048
:10141000D8F3C8F0B3ECEAF0B70ED66FFD0ED76F75
:101420000B0ED86F030ED96F050EDA6FDB6BDC6B1A
:10143000DD6BDE6B010EDF6FF1ECD4F06C0EBC6F78
:10144000FC0EBD6F660EBE6F010EBF6FC06BC16B31
:10145000060EC26FC36BC46BC56BC66BC76B6000F7
:10146000D8F3C8F0B3ECEAF0440ED66FFE0ED76F97
:10147000020ED86F030ED96F060EDA6FDB6BDC6BD2
:10148000DD6BDE6B010EDF6FF1ECD4F06C0EBC6F28
:10149000FC0EBD6F660EBE6F010EBF6FC06BC16BE1
:1014A000070EC26FC36BC46BC56BC66BC76B6000A6
:1014B000D8F3C8F0B3ECEAF0420ED66FFE0ED76F49
:1014C000020ED86F030ED96F070EDA6FDB6BDC6B81
:1014D000DD6BDE6B010EDF6FF1ECD4F02FD4640E08
:1014E000E96FFD0EEA6F0D0EEB6F600094F2ECF009
:1014F000030EAEECE0F06C0EBC6FFC0EBD6F5A0E2E
:10150000BE6F010EBF6FC06BC16B020EC26FC36BAB
:10151000C46BC56BC66BC76B6000D8F3C8F0B3EC87
:10152000EAF0710ED66FFD0ED76F0D0ED86F030E59
:10153000D96F020EDA6FDB6BDC6BDD6BDE6B010EDD
:10154000DF6FF1ECD4F06C0EBC6FFC0EBD6F5A0E69
:10155000BE6F010EBF6FC06BC16B050EC26FC36B58
:10156000C46BC56BC66BC76B6000D8F3C8F0B3EC37
:10157000EAF0B70ED66FFD0ED76F0B0ED86F030EC5
:10158000D96F050EDA6FDB6BDC6BDD6BDE6B010E8A
:10159000DF6FF1ECD4F052D7B70EE96FFD0EEA6FB2
:1015A0000B0EEB6F600094F2ECF0040EAEECE0F08A
:1015B0006C0EBC6FFC0EBD6F5A0EBE6F010EBF6F7E
:1015C000C06BC16B020EC26FC36BC46BC56BC66BC5
:1015D000C76B6000D8F3C8F0B3ECEAF0710ED66FB9
:1015E000FD0ED76F0D0ED86F030ED96F020EDA6F96
:1015F000DB6BDC6BDD6BDE6B010EDF6FF1ECD4F0CF
:101600006C0EBC6FFC0EBD6F5A0EBE6F010EBF6F2D
:10161000C06BC16B030EC26FC36BC46BC56BC66B73
:10162000C76B6000D8F3C8F0B3ECEAF0640ED66F75
:10163000FD0ED76F0D0ED86F030ED96FDA6FDB6B0F
:10164000DC6BDD6BDE6B010EDF6FF1ECD4F06C0E4A
:10165000BC6FFC0EBD6F5A0EBE6F010EBF6FC06B2C
:10166000C16B060EC26FC36BC46BC56BC66BC76B19
:101670006000D8F3C8F0B3ECEAF0F6D6440EE96F98
:10168000FE0EEA6F020EEB6F600094F2ECF0050EB6
:10169000AEECE0F06C0EBC6FFC0EBD6F5A0EBE6F70
:1016A000010EBF6FC06BC16B020EC26FC36BC46B08
:1016B000C56BC66BC76B6000D8F3C8F0B3ECEAF03B
:1016C000710ED66FFD0ED76F0D0ED86F030ED96F4A
:1016D000020EDA6FDB6BDC6BDD6BDE6B010EDF6F36
:1016E000F1ECD4F06C0EBC6FFC0EBD6F5A0EBE6FE9
:1016F000010EBF6FC06BC16B030EC26FC36BC46BB7
:10170000C56BC66BC76B6000D8F3C8F0B3ECEAF0EA
:10171000640ED66FFD0ED76F0D0ED86F030ED96F06
:10172000DA6FDB6BDC6BDD6BDE6B010EDF6FF1EC18
:10173000D4F06C0EBC6FFC0EBD6F5A0EBE6F010E66
:10174000BF6FC06BC16B040EC26FC36BC46BC56B44
:10175000C66BC76B6000D8F3C8F0B3ECEAF0B70E05
:10176000D66FFD0ED76F0B0ED86F030ED96F040E18
:10177000DA6FDB6BDC6BDD6BDE6B010EDF6FF1ECC8
:10178000D4F06C0EBC6FFC0EBD6F5A0EBE6F010E16
:10179000BF6FC06BC16B070EC26FC36BC46BC56BF1
:1017A000C66BC76B6000D8F3C8F0B3ECEAF084D620
:1017B000420EE96FFE0EEA6F020EEB6F600094F2CC
:1017C000ECF0060EAEECE0F06C0EBC6FFC0EBD6FE4
:1017D0005A0EBE6F010EBF6FC06BC16B020EC26F9F
:1017E000C36BC46BC56BC66BC76B6000D8F3C8F026
:1017F000B3ECEAF0710ED66FFD0ED76F0D0ED86FF9
:10180000030ED96F020EDA6FDB6BDC6BDD6BDE6B08
:10181000010EDF6FF1ECD4F06C0EBC6FFC0EBD6FEF
:101820005A0EBE6F010EBF6FC06BC16B030EC26F4D
:10183000C36BC46BC56BC66BC76B6000D8F3C8F0D5
:10184000B3ECEAF0640ED66FFD0ED76F0D0ED86FB5
:10185000030ED96FDA6FDB6BDC6BDD6BDE6B010EB9
:10186000DF6FF1ECD4F06C0EBC6FFC0EBD6F5A0E46
:10187000BE6F010EBF6FC06BC16B040EC26FC36B36
:10188000C46BC56BC66BC76B6000D8F3C8F0B3EC14
:10189000EAF0B70ED66FFD0ED76F0B0ED86F030EA2
:1018A000D96F040EDA6FDB6BDC6BDD6BDE6B010E68
:1018B000DF6FF1ECD4F06C0EBC6FFC0EBD6F5A0EF6
:1018C000BE6F010EBF6FC06BC16B050EC26FC36BE5
:1018D000C46BC56BC66BC76B6000D8F3C8F0B3ECC4
:1018E000EAF0440ED66FFE0ED76F020ED86F030ECD
:1018F000D96F050EDA6FDB6BDC6BDD6BDE6B010E17
:10190000DF6FF1ECD4F09EEF86F09451010A01E113
:1019100039D5030A01E1E3D5010A01E13DD6070A01
:1019200001E1ACD6010A01E143D79EEF86F06F0ECC
:10193000111901E051D200019F0501E0C2D0070E4C
:10194000D66F6000D8F3D7F0010E8DECFFF0AB0E30
:10195000EA6FFE0EEB6F100EEC6FF7ECFBF08ED023
:10196000D20ED66FFF0ED76F060ED86FD96B020E50
:10197000DA6FDB6BDC6BDD6BDE6BDF6B68ECF1F081
:10198000D80ED66FFF0ED76F060ED86FD96B040E28
:10199000DA6FDB6BDC6BDD6BDE6BDF6B68ECF1F061
:1019A000460409E1010ED66F020ED76FD86B6E5157
:1019B00038ECD3F011D0C70ED66FFF0ED76F050EDF
:1019C000D86F460ED96F020EDA6FDB6BDC6BDD6B06
:1019D000DE6BDF6B68ECF1F0010186050FE1600062
:1019E000A8F1D6F06000ACF1D7F0010E0001D86F7D
:1019F000040ED96FDA6BDDECCAF046D0C60E0001DA
:101A0000D66FFF0ED76F060ED86F3E0ED96F040E3D
:101A1000DA6FDB6BDC6BDD6BDE6BDF6B68ECF1F0E0
:101A200033D0D20ED66FFF0ED76F060ED86FD96B9C
:101A3000020EDA6FDB6BDC6BDD6BDE6BDF6B68EC91
:101A4000F1F0460409E1010ED66F020ED76FD86B94
:101A50006E5138ECD3F018D0C70ED66FFF0ED76F8B
:101A6000050ED86F460ED96F020EDA6FDB6BDC6B9A
:101A7000DD6BDE6BDF6B68ECF1F006D09D51010A87
:101A8000D0E0020A01E16CD70D0EBC6FC30EBD6F32
:101A9000440EBE6F020EBF6F010EC06F100EC16FFD
:101AA000060EC26FC36BC46BC56BC66BC76B6000A1
:101AB000D8F3C8F0B3ECEAF09F6B010E9E6F946F01
:101AC000966F960501E1F1D0FED0630EBC6FE50E76
:101AD000BD6F070EBE6F020EBF6FC06B250EC16FCC
:101AE000040EC26FC36BC46BC56BC66BC76B600063
:101AF000D8F3C8F0B3ECEAF00D0EBC6FC30EBD6FA7
:101B0000440EBE6F020EBF6F010EC06F100EC16F8C
:101B1000060EC26FC36BC46BC56BC66BC76B600030
:101B2000D8F3C8F0B3ECEAF0630EBC6FE50EBD6FFE
:101B3000070EBE6F020EBF6F5F0EC06F250EC16F26
:101B4000020EC26FC36BC46BC56BC66BC76B600004
:101B5000D8F3C8F0B3ECEAF0B1D0630EBC6FE50E79
:101B6000BD6F070EBE6F020EBF6FC06B250EC16F3B
:101B7000020EC26FC36BC46BC56BC66BC76B6000D4
:101B8000D8F3C8F0B3ECEAF09D0531E00D0EBC6F60
:101B9000C30EBD6F440EBE6F020EBF6F010EC06F4D
:101BA000100EC16F060EC26FC36BC46BC56BC66BE4
:101BB000C76B6000D8F3C8F0B3ECEAF0630EBC6FFB
:101BC000E50EBD6F070EBE6F020EBF6F5F0EC06FDA
:101BD000250EC16F040EC26FC36BC46BC56BC66BA1
:101BE000C76B6000D8F3C8F0B3ECEAF067D00D0E15
:101BF000BC6FC30EBD6F440EBE6F020EBF6FC06FD1
:101C0000100EC16F060EC26FC36BC46BC56BC66B83
:101C1000C76B6000D8F3C8F0B3ECEAF04FD0630EA6
:101C2000BC6FE50EBD6F070EBE6F020EBF6FC06BBF
:101C3000250EC16F020EC26FC36BC46BC56BC66B42
:101C4000C76B6000D8F3C8F0B3ECEAF0630EBC6F6A
:101C5000E50EBD6F070EBE6F020EBF6FC06B250E87
:101C6000C16F040EC26FC36BC46BC56BC66BC76B11
:101C70006000D8F3C8F0B3ECEAF00D0EBC6FC30EF1
:101C8000BD6F440EBE6F020EBF6FC06F100EC16FEE
:101C9000060EC26FC36BC46BC56BC66BC76B6000AF
:101CA000D8F3C8F0B3ECEAF009D09451010A01E18D
:101CB0000CD7030A01E151D7010AB1E094C095F0B5
:101CC000966B9E6B25D001014E050EE1010E0001C1
:101CD000D66F020ED76F600094F2D8F06C5138ECDA
:101CE000D3F001014E6B14D04D0512E16000A0F15C
:101CF000D6F06000A4F1D7F0010E0001D86F040EF9
:101D0000D96F600094F2DAF0DDECCAF001014D6B9E
:101D100000019E0548E19C050AE1010ED66F020E06
:101D2000D76F010ED86F6C5138ECD3F03AD09B05C9
:101D30000FE16000A0F1D6F06000A4F1D7F0010E31
:101D4000D86F040ED96F010EDA6FDDECCAF029D01E
:101D5000460427E19D0503E1020E95190AE0010101
:101D600086051FE1030E000195191BE1030E9D1965
:101D700018E10D0EBC6FC30EBD6F440EBE6F020E98
:101D8000BF6F030EC06F100EC16F060EC26FC36B24
:101D9000C46BC56BC66BC76B6000D8F3C8F0B3ECFF
:101DA000EAF000019E6B9C050AE1410EBB6F140E28
:101DB000BC6F985198ECF9F001014E6F12009B0531
:101DC000D8A41200410EBB6F140EBC6F985198EC52
:101DD000F9F001014D6F1200700E111963E100015D
:101DE0009F053CE1070ED66F6000D8F3D7F0010ED7
:101DF0008DECFFF09B0EEA6FFE0EEB6F100EEC6F9A
:101E0000F7ECFBF00F0ED66FFF0ED76F0D0ED86FED
:101E1000D96B020EDA6FDB6BDC6BDD6BDE6BDF6BBD
:101E200068ECF1F0B00506E15A0ED66F480EDAEC18
:101E3000EEF011D0020EB01906E15A0ED66F200E48
:101E4000DAECEEF008D0030EB01905E15A0ED66FA9
:101E5000200EDAECEEF09F6B010E9E6F01014C0537
:101E600003E000019E0513E1600098F1D6F06000E8
:101E70009CF1D7F00A0E0001D86F040ED96F6000F4
:101E800094F2DAF06EECC3F09E6B01014C6B410EE4
:101E90000001BB6F140EBC6F985198ECF9F0010172
:101EA0004C6F1200780E111901E0F3D200019F056A
:101EB00014E1070ED66F6000D8F3D7F0010E8DEC59
:101EC000FFF0E40EEA6FFF0EEB6F060EEC6FF7EC1F
:101ED000FBF09F6B010E9E6F946F960501E1C7D2D8
:101EE0009E0501E1C4D21200080EE96FFE0EEA6FF2
:101EF000090EEB6F600094F2ECF0020EAEECE0F035
:101F00006C0EBC6FFC0EBD6F5A0EBE6F010EBF6F24
:101F1000C06BC16B040EC26FC36BC46BC56BC66B69
:101F2000C76B6000D8F3C8F0B3ECEAF0A10ED66F2F
:101F3000FD0ED76F0B0ED86F030ED96F040EDA6F3C
:101F4000DB6BDC6BDD6BDE6B010EDF6FF1ECD4F075
:101F50006C0EBC6FFC0EBD6F660EBE6F010EBF6FC8
:101F6000C06BC16B050EC26FC36BC46BC56BC66B18
:101F7000C76B6000D8F3C8F0B3ECEAF0FF0ED66F81
:101F8000FD0ED76F090ED86F030ED96F050EDA6FED
:101F9000DB6BDC6BDD6BDE6B010EDF6FF1ECD4F025
:101FA0006C0EBC6FFC0EBD6F660EBE6F010EBF6F78
:101FB000C06BC16B060EC26FC36BC46BC56BC66BC7
:101FC000C76B6000D8F3C8F0B3ECEAF0EB0ED66F45
:101FD000FD0ED76F0A0ED86F030ED96F060EDA6F9B
:101FE000DB6BDC6BDD6BDE6B010EDF6FF1ECD4F0D5
:101FF0006C0EBC6FFC0EBD6F660EBE6F010EBF6F28
:10200000C06BC16B070EC26FC36BC46BC56BC66B75
:10201000C76B6000D8F3C8F0B3ECEAF0300ED66FAF
:10202000FE0ED76F060ED86F030ED96F070EDA6F4C
:10203000DB6BDC6BDD6BDE6B010EDF6FF1ECD4F084
:102040009EEF86F0A10EE96FFD0EEA6F0B0EEB6FAF
:10205000600094F2ECF0030EAEECE0F06C0EBC6F9E
:10206000FC0EBD6F5A0EBE6F010EBF6FC06BC16B11
:10207000020EC26FC36BC46BC56BC66BC76B6000CF
:10208000D8F3C8F0B3ECEAF0080ED66FFE0ED76FA7
:10209000090ED86F030ED96F020EDA6FDB6BDC6BA3
:1020A000DD6BDE6B010EDF6FF1ECD4F06C0EBC6FFC
:1020B000FC0EBD6F5A0EBE6F010EBF6FC06BC16BC1
:1020C000050EC26FC36BC46BC56BC66BC76B60007C
:1020D000D8F3C8F0B3ECEAF0FF0ED66FFD0ED76F61
:1020E000090ED86F030ED96F050EDA6FDB6BDC6B50
:1020F000DD6BDE6B010EDF6FF1ECD4F051D7FF0E1C
:10210000E96FFD0EEA6F090EEB6F600094F2ECF0E0
:10211000040EAEECE0F06C0EBC6FFC0EBD6F5A0E00
:10212000BE6F010EBF6FC06BC16B020EC26FC36B7F
:10213000C46BC56BC66BC76B6000D8F3C8F0B3EC5B
:10214000EAF0080ED66FFE0ED76F090ED86F030E99
:10215000D96F020EDA6FDB6BDC6BDD6BDE6B010EB1
:10216000DF6FF1ECD4F06C0EBC6FFC0EBD6F5A0E3D
:10217000BE6F010EBF6FC06BC16B030EC26FC36B2E
:10218000C46BC56BC66BC76B6000D8F3C8F0B3EC0B
:10219000EAF0A10ED66FFD0ED76F0B0ED86F030EAF
:1021A000D96FDA6FDB6BDC6BDD6BDE6B010EDF6F23
:1021B000F1ECD4F06C0EBC6FFC0EBD6F5A0EBE6F0E
:1021C000010EBF6FC06BC16B060EC26FC36BC46BD9
:1021D000C56BC66BC76B6000D8F3C8F0B3ECEAF010
:1021E000F5D6EB0EE96FFD0EEA6F0A0EEB6F60009D
:1021F00094F2ECF0050EAEECE0F06C0EBC6FFC0E51
:10220000BD6F5A0EBE6F010EBF6FC06BC16B020E69
:10221000C26FC36BC46BC56BC66BC76B6000D8F372
:10222000C8F0B3ECEAF0080ED66FFE0ED76F090EB9
:10223000D86F030ED96F020EDA6FDB6BDC6BDD6BD0
:10224000DE6B010EDF6FF1ECD4F06C0EBC6FFC0E98
:10225000BD6F5A0EBE6F010EBF6FC06BC16B030E18
:10226000C26FC36BC46BC56BC66BC76B6000D8F322
:10227000C8F0B3ECEAF0A10ED66FFD0ED76F0B0ECF
:10228000D86F030ED96FDA6FDB6BDC6BDD6BDE6B47
:10229000010EDF6FF1ECD4F06C0EBC6FFC0EBD6F65
:1022A0005A0EBE6F010EBF6FC06BC16B040EC26FC2
:1022B000C36BC46BC56BC66BC76B6000D8F3C8F04B
:1022C000B3ECEAF0FF0ED66FFD0ED76F090ED86F94
:1022D000030ED96F040EDA6FDB6BDC6BDD6BDE6B2C
:1022E000010EDF6FF1ECD4F06C0EBC6FFC0EBD6F15
:1022F0005A0EBE6F010EBF6FC06BC16B070EC26F6F
:10230000C36BC46BC56BC66BC76B6000D8F3C8F0FA
:10231000B3ECEAF083D6300EE96FFE0EEA6F060EDC
:10232000EB6F600094F2ECF0AEECE0F06C0EBC6F82
:10233000FC0EBD6F5A0EBE6F010EBF6FC06BC16B3E
:10234000020EC26FC36BC46BC56BC66BC76B6000FC
:10235000D8F3C8F0B3ECEAF0080ED66FFE0ED76FD4
:10236000090ED86F030ED96F020EDA6FDB6BDC6BD0
:10237000DD6BDE6B010EDF6FF1ECD4F06C0EBC6F29
:10238000FC0EBD6F5A0EBE6F010EBF6FC06BC16BEE
:10239000030EC26FC36BC46BC56BC66BC76B6000AB
:1023A000D8F3C8F0B3ECEAF0A10ED66FFD0ED76FEC
:1023B0000B0ED86F030ED96FDA6FDB6BDC6BDD6B46
:1023C000DE6B010EDF6FF1ECD4F06C0EBC6FFC0E17
:1023D000BD6F5A0EBE6F010EBF6FC06BC16B040E96
:1023E000C26FC36BC46BC56BC66BC76B6000D8F3A1
:1023F000C8F0B3ECEAF0FF0ED66FFD0ED76F090EF2
:10240000D86F030ED96F040EDA6FDB6BDC6BDD6BFC
:10241000DE6B010EDF6FF1ECD4F06C0EBC6FFC0EC6
:10242000BD6F5A0EBE6F010EBF6FC06BC16B050E44
:10243000C26FC36BC46BC56BC66BC76B6000D8F350
:10244000C8F0B3ECEAF0EB0ED66FFD0ED76F0A0EB4
:10245000D86F030ED96F050EDA6FDB6BDC6BDD6BAB
:10246000DE6B010EDF6FF1ECD4F09EEF86F094513D
:10247000010A01E139D5030A01E1E4D5010A01E1CC
:102480003ED6070A01E1ADD6010A01E144D79EEF2D
:1024900086F0790E111951E100019F052BE1070E1D
:1024A000D66F6000D8F3D7F0010E8DECFFF09A0ED6
:1024B000EA6FFF0EEB6F090EEC6FF7ECFBF09F6B12
:1024C000986BF80E9225D66FD76BFF0ED7232E0E82
:1024D000D86F020ED96FDA6BDB6BDC6BDDECBDF015
:1024E000050ED66F9251F80FD76F070E1AECF9F060
:1024F000080F926F01017A05D8A41200F80E7B250F
:102500000001D66FD76BFF0ED7232E0ED86F020EA9
:10251000D96FDA6BDB6BDC6BDDECBDF0050ED66FD3
:1025200001017B51F80F0001D76F070E1AECF9F08B
:10253000080F926F01017A6B12007A0E111902E0F6
:102540002CEF97F000019F0514E1070ED66F600095
:10255000D8F3D7F0010E8DECFFF0CA0EEA6FFE0E35
:10256000EB6F0F0EEC6FF7ECFBF09F6B010E946FAF
:10257000966F960501E17CD388D3AF0549E10D0E36
:10258000BC6FC30EBD6F440EBE6F020EBF6F110E47
:10259000C06F080EC16F020EC26FC36BC46BC56BF8
:1025A000C66BC76B6000D8F3C8F0B3ECEAF00D0E51
:1025B000BC6FC30EBD6F440EBE6F020EBF6F160E12
:1025C000C06F080EC16F040EC26FC36BC46BC56BC6
:1025D000C66BC76B6000D8F3C8F0B3ECEAF00D0E21
:1025E000BC6FC30EBD6F440EBE6F020EBF6F120EE6
:1025F000C06F080EC16F060EC26FC36BC46BC56B94
:10260000C66BC76B6000D8F3C8F0B3ECEAF097D0A4
:10261000020EAF1949E10D0EBC6FC30EBD6F440E23
:10262000BE6F020EBF6F0F0EC06F080EC16F020E9D
:10263000C26FC36BC46BC56BC66BC76B6000D8F34E
:10264000C8F0B3ECEAF00D0EBC6FC30EBD6F440EC4
:10265000BE6F020EBF6F180EC06F080EC16F040E62
:10266000C26FC36BC46BC56BC66BC76B6000D8F31E
:10267000C8F0B3ECEAF00D0EBC6FC30EBD6F440E94
:10268000BE6F020EBF6F120EC06F080EC16F060E36
:10269000C26FC36BC46BC56BC66BC76B6000D8F3EE
:1026A000C8F0B3ECEAF04BD0030EAF1948E10D0EC1
:1026B000BC6FC30EBD6F440EBE6F020EBF6F0F0E18
:1026C000C06F080EC16F020EC26FC36BC46BC56BC7
:1026D000C66BC76B6000D8F3C8F0B3ECEAF00D0E20
:1026E000BC6FC30EBD6F440EBE6F020EBF6F160EE1
:1026F000C06F080EC16F040EC26FC36BC46BC56B95
:10270000C66BC76B6000D8F3C8F0B3ECEAF00D0EEF
:10271000BC6FC30EBD6F440EBE6F020EBF6F140EB2
:10272000C06F080EC16F060EC26FC36BC46BC56B62
:10273000C66BC76B6000D8F3C8F0B3ECEAF0630E69
:10274000BC6FE50EBD6F070EBE6F020EBF6FC06B94
:10275000500EC16F040EC26FC36BC46BC56BC66BEA
:10276000C76B6000D8F3C8F0B3ECEAF0630EBC6F3F
:10277000E50EBD6F070EBE6F020EBF6FC06B500E31
:10278000C16F060EC26FC36BC46BC56BC66BC76BE4
:102790006000D8F3C8F0B3ECEAF0630EBC6FE50E4E
:1027A000BD6F070EBE6F020EBF6F6B0EC06F500E77
:1027B000C16F020EC26FC36BC46BC56BC66BC76BB8
:1027C0006000D8F3C8F0B3ECEAF05CD2020EAF19A7
:1027D00049E10D0EBC6FC30EBD6F440EBE6F020EFD
:1027E000BF6F0E0EC06F080EC16F020EC26FC36BBB
:1027F000C46BC56BC66BC76B6000D8F3C8F0B3EC95
:10280000EAF00D0EBC6FC30EBD6F440EBE6F020E1C
:10281000BF6F190EC06F080EC16F040EC26FC36B7D
:10282000C46BC56BC66BC76B6000D8F3C8F0B3EC64
:10283000EAF00D0EBC6FC30EBD6F440EBE6F020EEC
:10284000BF6F120EC06F080EC16F060EC26FC36B52
:10285000C46BC56BC66BC76B6000D8F3C8F0B3EC34
:10286000EAF096D0AF0549E10D0EBC6FC30EBD6F07
:10287000440EBE6F020EBF6F100EC06F080EC16F08
:10288000020EC26FC36BC46BC56BC66BC76B6000B7
:10289000D8F3C8F0B3ECEAF00D0EBC6FC30EBD6FF9
:1028A000440EBE6F020EBF6F170EC06F080EC16FD1
:1028B000040EC26FC36BC46BC56BC66BC76B600085
:1028C000D8F3C8F0B3ECEAF00D0EBC6FC30EBD6FC9
:1028D000440EBE6F020EBF6F120EC06F080EC16FA6
:1028E000060EC26FC36BC46BC56BC66BC76B600053
:1028F000D8F3C8F0B3ECEAF04BD0030EAF1948E1BF
:102900000D0EBC6FC30EBD6F440EBE6F020EBF6FC7
:102910000E0EC06F080EC16F020EC26FC36BC46B88
:10292000C56BC66BC76B6000D8F3C8F0B3ECEAF0B8
:102930000D0EBC6FC30EBD6F440EBE6F020EBF6F97
:10294000170EC06F080EC16F040EC26FC36BC46B4D
:10295000C56BC66BC76B6000D8F3C8F0B3ECEAF088
:102960000D0EBC6FC30EBD6F440EBE6F020EBF6F67
:10297000140EC06F080EC16F060EC26FC36BC46B1E
:10298000C56BC66BC76B6000D8F3C8F0B3ECEAF058
:10299000630EBC6FE50EBD6F070EBE6F020EBF6FFC
:1029A000C06B500EC16F020EC26FC36BC46BC56BA0
:1029B000C66BC76B6000D8F3C8F0B3ECEAF0630EE7
:1029C000BC6FE50EBD6F070EBE6F020EBF6FC06B12
:1029D000500EC16F060EC26FC36BC46BC56BC66B66
:1029E000C76B6000D8F3C8F0B3ECEAF0630EBC6FBD
:1029F000E50EBD6F070EBE6F020EBF6F6B0EC06F90
:102A0000500EC16F040EC26FC36BC46BC56BC66B37
:102A1000C76B6000D8F3C8F0B3ECEAF033D1030E13
:102A2000AF1949E10D0EBC6FC30EBD6F440EBE6FF2
:102A3000020EBF6F0E0EC06F080EC16F020EC26F86
:102A4000C36BC46BC56BC66BC76B6000D8F3C8F0B3
:102A5000B3ECEAF00D0EBC6FC30EBD6F440EBE6F3B
:102A6000020EBF6F160EC06F080EC16F040EC26F4C
:102A7000C36BC46BC56BC66BC76B6000D8F3C8F083
:102A8000B3ECEAF00D0EBC6FC30EBD6F440EBE6F0B
:102A9000020EBF6F150EC06F080EC16F060EC26F1B
:102AA000C36BC46BC56BC66BC76B6000D8F3C8F053
:102AB000B3ECEAF096D0AF0549E10D0EBC6FC30E42
:102AC000BD6F440EBE6F020EBF6F100EC06F080EBA
:102AD000C16F020EC26FC36BC46BC56BC66BC76B95
:102AE0006000D8F3C8F0B3ECEAF00D0EBC6FC30E73
:102AF000BD6F440EBE6F020EBF6F160EC06F080E84
:102B0000C16F040EC26FC36BC46BC56BC66BC76B62
:102B10006000D8F3C8F0B3ECEAF00D0EBC6FC30E42
:102B2000BD6F440EBE6F020EBF6F130EC06F080E56
:102B3000C16F060EC26FC36BC46BC56BC66BC76B30
:102B40006000D8F3C8F0B3ECEAF04BD0020EAF1936
:102B500048E10D0EBC6FC30EBD6F440EBE6F020E7A
:102B6000BF6F0E0EC06F080EC16F020EC26FC36B37
:102B7000C46BC56BC66BC76B6000D8F3C8F0B3EC11
:102B8000EAF00D0EBC6FC30EBD6F440EBE6F020E99
:102B9000BF6F180EC06F080EC16F040EC26FC36BFB
:102BA000C46BC56BC66BC76B6000D8F3C8F0B3ECE1
:102BB000EAF00D0EBC6FC30EBD6F440EBE6F020E69
:102BC000BF6F130EC06F080EC16F060EC26FC36BCE
:102BD000C46BC56BC66BC76B6000D8F3C8F0B3ECB1
:102BE000EAF0630EBC6FE50EBD6F070EBE6F020EFE
:102BF000BF6FC06B500EC16F020EC26FC36BC46B50
:102C0000C56BC66BC76B6000D8F3C8F0B3ECEAF0D5
:102C1000630EBC6FE50EBD6F070EBE6F020EBF6F79
:102C2000C06B500EC16F040EC26FC36BC46BC56B1B
:102C3000C66BC76B6000D8F3C8F0B3ECEAF0630E64
:102C4000BC6FE50EBD6F070EBE6F020EBF6F6B0E41
:102C5000C06F500EC16F060EC26FC36BC46BC56BE5
:102C6000C66BC76B6000D8F3C8F0B3ECEAF00AD0CB
:102C70009451010A01E181D4030A01E1A7D5010AB7
:102C800001E1CDD694C095F0966B9E05D8A41200B4
:102C9000950549E10D0EBC6FC30EBD6F440EBE6FAE
:102CA000020EBF6F110EC06F080EC16F020EC26F11
:102CB000C36BC46BC56BC66BC76B6000D8F3C8F041
:102CC000B3ECEAF00D0EBC6FC30EBD6F440EBE6FC9
:102CD000020EBF6F160EC06F080EC16F040EC26FDA
:102CE000C36BC46BC56BC66BC76B6000D8F3C8F011
:102CF000B3ECEAF00D0EBC6FC30EBD6F440EBE6F99
:102D0000020EBF6F120EC06F080EC16F060EC26FAB
:102D1000C36BC46BC56BC66BC76B6000D8F3C8F0E0
:102D2000B3ECEAF097D0020E951949E10D0EBC6F95
:102D3000C30EBD6F440EBE6F020EBF6F0E0EC06F8E
:102D4000080EC16F020EC26FC36BC46BC56BC66B3E
:102D5000C76B6000D8F3C8F0B3ECEAF00D0EBC6F9F
:102D6000C30EBD6F440EBE6F020EBF6F190EC06F53
:102D7000080EC16F040EC26FC36BC46BC56BC66B0C
:102D8000C76B6000D8F3C8F0B3ECEAF00D0EBC6F6F
:102D9000C30EBD6F440EBE6F020EBF6F120EC06F2A
:102DA000080EC16F060EC26FC36BC46BC56BC66BDA
:102DB000C76B6000D8F3C8F0B3ECEAF04BD0030E59
:102DC000951948E10D0EBC6FC30EBD6F440EBE6F6A
:102DD000020EBF6F0E0EC06F080EC16F020EC26FE3
:102DE000C36BC46BC56BC66BC76B6000D8F3C8F010
:102DF000B3ECEAF00D0EBC6FC30EBD6F440EBE6F98
:102E0000020EBF6F160EC06F080EC16F040EC26FA8
:102E1000C36BC46BC56BC66BC76B6000D8F3C8F0DF
:102E2000B3ECEAF00D0EBC6FC30EBD6F440EBE6F67
:102E3000020EBF6F150EC06F080EC16F060EC26F77
:102E4000C36BC46BC56BC66BC76B6000D8F3C8F0AF
:102E5000B3ECEAF09E6B12007B0E111919E1000130
:102E60009F05D8A41200070ED66F6000D8F3D7F0E4
:102E7000010E8DECFFF0910EEA6FFF0EEB6F090E65
:102E8000EC6FF7ECFBF09F6B010E9E6F946F010CE3
:102E90007C0E111901E0E4D000019F0537E1070E17
:102EA000D66F6000D8F3D7F0010E8DECFFF06A0EFC
:102EB000EA6FFF0EEB6F0A0EEC6FF7ECFBF0460EBD
:102EC000D66FFE0ED76F130ED86FD96B020EDA6F66
:102ED000DB6BDC6BDD6BDE6B010EDF6FF1ECD4F0D6
:102EE000590ED66FFE0ED76F110ED86FD96B030E29
:102EF000DA6FDB6BDC6BDD6BDE6B010EDF6FF1EC31
:102F0000D4F09F6B020E946F010E966F960501E14F
:102F10009FD09E0501E19CD012009E0519E10D0E87
:102F2000BC6FC30EBD6F440EBE6F020EBF6F090EA5
:102F3000C06F100EC16F040EC26FC36BC46BC56B44
:102F4000C66BC76B6000D8F3C8F0B3ECEAF018D0DA
:102F50000D0EBC6FC30EBD6F440EBE6F020EBF6F71
:102F6000080EC06F100EC16F040EC26FC36BC46B2E
:102F7000C56BC66BC76B6000D8F3C8F0B3ECEAF062
:102F80000D0EBC6FC30EBD6F440EBE6F020EBF6F41
:102F90001D0EC06F100EC16F060EC26FC36BC46BE7
:102FA000C56BC66BC76B6000D8F3C8F0B3ECEAF032
:102FB0009EEF86F00D0EBC6FC30EBD6F440EBE6F4C
:102FC000020EBF6F070EC06F100EC16F040EC26FEE
:102FD000C36BC46BC56BC66BC76B6000D8F3C8F01E
:102FE000B3ECEAF09E051AE10D0EBC6FC30EBD6F87
:102FF000440EBE6F020EBF6F1F0EC06F100EC16F6A
:10300000060EC26FC36BC46BC56BC66BC76B60002B
:10301000D8F3C8F0B3ECEAF09EEF86F00D0EBC6F6B
:10302000C30EBD6F440EBE6F020EBF6F1E0EC06F8B
:10303000100EC16F060EC26FC36BC46BC56BC66B3F
:10304000C76B6000D8F3C8F0B3ECEAF09EEF86F0EF
:103050009451010A01E161D7030AACE09EEF86F0CA
:10306000810E111959E100019F05D8A41200070E25
:10307000D66F6000D8F3D7F0010E8DECFFF0F00EA4
:10308000EA6FFF0EEB6F060EEC6FF7ECFBF07B0EBA
:10309000D66FFE0ED76F100ED86F060ED96F030EC7
:1030A000DA6FDB6BDC6BDD6BDE6BDF6BF1ECD4F0CE
:1030B000BB0ED66FFE0ED76F0F0ED86F0A0ED96FEC
:1030C000040EDA6FDB6BDC6BDD6BDE6BDF6BF1EC60
:1030D000D4F0DE0ED66FFF0ED76F060ED86F240E1B
:1030E000D96F050EDA6FDB6BDC6BDD6BDE6BDF6BD4
:1030F000F1ECD4F08B0ED66FFE0ED76F100ED86F9A
:10310000080ED96F060EDA6FDB6BDC6BDD6BDE6BE6
:10311000DF6BF1ECD4F0B7D6820E111901E0F4D2D6
:1031200000019F0514E1070ED66F6000D8F3D7F0B9
:10313000010E8DECFFF0540EEA6FFF0EEB6F0B0EDD
:10314000EC6FF7ECFBF09F6B010E9E6F946F960592
:1031500001E1C8D29E0501E1C5D21200AC0EE96FB3
:10316000FD0EEA6F0B0EEB6F600094F2ECF0020EB6
:10317000AEECE0F06C0EBC6FFC0EBD6F5A0EBE6F75
:10318000010EBF6FC06BC16B040EC26FC36BC46B0B
:10319000C56BC66BC76B6000D8F3C8F0B3ECEAF040
:1031A000F50ED66FFD0ED76F0A0ED86F030ED96FCE
:1031B000040EDA6FDB6BDC6BDD6BDE6B010EDF6F39
:1031C000F1ECD4F06C0EBC6FFC0EBD6F660EBE6FE2
:1031D000010EBF6FC06BC16B050EC26FC36BC46BBA
:1031E000C56BC66BC76B6000D8F3C8F0B3ECEAF0F0
:1031F000400ED66FFE0ED76F020ED86F030ED96F3A
:10320000050EDA6FDB6BDC6BDD6BDE6B010EDF6FE7
:10321000F1ECD4F06C0EBC6FFC0EBD6F660EBE6F91
:10322000010EBF6FC06BC16B060EC26FC36BC46B68
:10323000C56BC66BC76B6000D8F3C8F0B3ECEAF09F
:103240003E0ED66FFE0ED76F020ED86F030ED96FEB
:10325000060EDA6FDB6BDC6BDD6BDE6B010EDF6F96
:10326000F1ECD4F06C0EBC6FFC0EBD6F660EBE6F41
:10327000010EBF6FC06BC16B070EC26FC36BC46B17
:10328000C56BC66BC76B6000D8F3C8F0B3ECEAF04F
:103290003C0ED66FFE0ED76F020ED86F030ED96F9D
:1032A000070EDA6FDB6BDC6BDD6BDE6B010EDF6F45
:1032B000F1ECD4F09EEF86F0F50EE96FFD0EEA6FAB
:1032C0000A0EEB6F600094F2ECF0030EAEECE0F04F
:1032D0006C0EBC6FFC0EBD6F5A0EBE6F010EBF6F41
:1032E000C06BC16B020EC26FC36BC46BC56BC66B88
:1032F000C76B6000D8F3C8F0B3ECEAF0AC0ED66F41
:10330000FD0ED76F0B0ED86F030ED96F020EDA6F5A
:10331000DB6BDC6BDD6BDE6B010EDF6FF1ECD4F091
:103320006C0EBC6FFC0EBD6F5A0EBE6F010EBF6FF0
:10333000C06BC16B050EC26FC36BC46BC56BC66B34
:10334000C76B6000D8F3C8F0B3ECEAF0400ED66F5C
:10335000FE0ED76F020ED86F030ED96F050EDA6F0F
:10336000DB6BDC6BDD6BDE6B010EDF6FF1ECD4F041
:1033700051D7400EE96FFE0EEA6F020EEB6F600050
:1033800094F2ECF0040EAEECE0F06C0EBC6FFC0EB0
:10339000BD6F5A0EBE6F010EBF6FC06BC16B020EC8
:1033A000C26FC36BC46BC56BC66BC76B6000D8F3D1
:1033B000C8F0B3ECEAF0AC0ED66FFD0ED76F0B0E73
:1033C000D86F030ED96F020EDA6FDB6BDC6BDD6B2F
:1033D000DE6B010EDF6FF1ECD4F06C0EBC6FFC0EF7
:1033E000BD6F5A0EBE6F010EBF6FC06BC16B030E77
:1033F000C26FC36BC46BC56BC66BC76B6000D8F381
:10340000C8F0B3ECEAF0F50ED66FFD0ED76F0A0EDA
:10341000D86F030ED96FDA6FDB6BDC6BDD6BDE6BA5
:10342000010EDF6FF1ECD4F06C0EBC6FFC0EBD6FC3
:103430005A0EBE6F010EBF6FC06BC16B060EC26F1E
:10344000C36BC46BC56BC66BC76B6000D8F3C8F0A9
:10345000B3ECEAF0F5D63E0EE96FFE0EEA6F020E0F
:10346000EB6F600094F2ECF0050EAEECE0F06C0E49
:10347000BC6FFC0EBD6F5A0EBE6F010EBF6FC06BEE
:10348000C16B020EC26FC36BC46BC56BC66BC76BDF
:103490006000D8F3C8F0B3ECEAF0AC0ED66FFD0EC6
:1034A000D76F0B0ED86F030ED96F020EDA6FDB6B7E
:1034B000DC6BDD6BDE6B010EDF6FF1ECD4F06C0EBC
:1034C000BC6FFC0EBD6F5A0EBE6F010EBF6FC06B9E
:1034D000C16B030EC26FC36BC46BC56BC66BC76B8E
:1034E0006000D8F3C8F0B3ECEAF0F50ED66FFD0E2D
:1034F000D76F0A0ED86F030ED96FDA6FDB6BDC6BF8
:10350000DD6BDE6B010EDF6FF1ECD4F06C0EBC6F87
:10351000FC0EBD6F5A0EBE6F010EBF6FC06BC16B4C
:10352000040EC26FC36BC46BC56BC66BC76B600008
:10353000D8F3C8F0B3ECEAF0400ED66FFE0ED76FAA
:10354000020ED86F030ED96F040EDA6FDB6BDC6BE3
:10355000DD6BDE6B010EDF6FF1ECD4F06C0EBC6F37
:10356000FC0EBD6F5A0EBE6F010EBF6FC06BC16BFC
:10357000070EC26FC36BC46BC56BC66BC76B6000B5
:10358000D8F3C8F0B3ECEAF083D63C0EE96FFE0E38
:10359000EA6F020EEB6F600094F2ECF0060EAEECF8
:1035A000E0F06C0EBC6FFC0EBD6F5A0EBE6F010ECC
:1035B000BF6FC06BC16B020EC26FC36BC46BC56BB8
:1035C000C66BC76B6000D8F3C8F0B3ECEAF0AC0E82
:1035D000D66FFD0ED76F0B0ED86F030ED96F020E8C
:1035E000DA6FDB6BDC6BDD6BDE6B010EDF6FF1EC3A
:1035F000D4F06C0EBC6FFC0EBD6F5A0EBE6F010E88
:10360000BF6FC06BC16B030EC26FC36BC46BC56B66
:10361000C66BC76B6000D8F3C8F0B3ECEAF0F50EE8
:10362000D66FFD0ED76F0A0ED86F030ED96FDA6F03
:10363000DB6BDC6BDD6BDE6B010EDF6FF1ECD4F06E
:103640006C0EBC6FFC0EBD6F5A0EBE6F010EBF6FCD
:10365000C06BC16B040EC26FC36BC46BC56BC66B12
:10366000C76B6000D8F3C8F0B3ECEAF0400ED66F39
:10367000FE0ED76F020ED86F030ED96F040EDA6FED
:10368000DB6BDC6BDD6BDE6B010EDF6FF1ECD4F01E
:103690006C0EBC6FFC0EBD6F5A0EBE6F010EBF6F7D
:1036A000C06BC16B050EC26FC36BC46BC56BC66BC1
:1036B000C76B6000D8F3C8F0B3ECEAF03E0ED66FEB
:1036C000FE0ED76F020ED86F030ED96F050EDA6F9C
:1036D000DB6BDC6BDD6BDE6B010EDF6FF1ECD4F0CE
:1036E0009EEF86F09451010A01E138D5030A01E109
:1036F000E3D5010A01E13DD6070A01E1ACD6010A92
:1037000001E143D79EEF86F0830E111901E017D334
:1037100000019F0531E1070ED66F6000D8F3D7F0A6
:10372000010E8DECFFF0330EEA6FFF0EEB6F0B0E08
:10373000EC6FF7ECFBF0F60ED66FFF0ED76F050EB1
:10374000D86FD96B020EDA6FDB6BDC6BDD6BDE6B77
:10375000DF6B68ECF1F09A0503E1916B030E02D088
:10376000010E916F946F9F6B3550361003E1366AEE
:10377000010E356E010E966F960501E105D213D24A
:10378000630EBC6FE50EBD6F070EBE6F020EBF6FFE
:10379000C06B450EC16F040EC26FC36BC46BC56BAB
:1037A000C66BC76B6000D8F3C8F0B3ECEAF0630EE9
:1037B000BC6FE50EBD6F070EBE6F020EBF6F6B0EC6
:1037C000C06F450EC16F020EC26FC36BC46BC56B79
:1037D000C66BC76B6000D8F3C8F0B3ECEAF06000CA
:1037E000C8F1D6F06000CCF1D7F01E0ED86F020EF3
:1037F000D96FDA6BDB6BDC6BDDECBDF0B65118E139
:103800000D0EBC6FC30EBD6F440EBE6F020EBF6FB8
:103810000A0EC06FC16B040EC26FC36BC46BC56B65
:10382000C66BC76B6000D8F3C8F0B3ECEAF017D0F2
:103830000D0EBC6FC30EBD6F440EBE6F020EBF6F88
:103840000C0EC06FC16B040EC26FC36BC46BC56B33
:10385000C66BC76B6000D8F3C8F0B3ECEAF0910513
:1038600018E10D0EBC6FC30EBD6F440EBE6F020E8D
:10387000BF6F040EC06FC16B060EC26FC36BC46B0B
:10388000C56BC66BC76B6000D8F3C8F0B3ECEAF049
:1038900017D00D0EBC6FC30EBD6F440EBE6F020E6F
:1038A000BF6F1A0EC06FC16B060EC26FC36BC46BC5
:1038B000C56BC66BC76B6000D8F3C8F0B3ECEAF019
:1038C000B00506E15A0ED66F200EDAECEEF066D1A6
:1038D000020EB01906E15A0ED66F200EDAECEEF0A9
:1038E0005DD1030EB01901E059D15A0ED66F200EEA
:1038F000DAECEEF053D1630EBC6FE50EBD6F070E30
:10390000BE6F020EBF6FC06B450EC16F020EC26F5D
:10391000C36BC46BC56BC66BC76B6000D8F3C8F0D4
:10392000B3ECEAF0630EBC6FE50EBD6F070EBE6F21
:10393000020EBF6F6B0EC06F450EC16F040EC26FDB
:10394000C36BC46BC56BC66BC76B6000D8F3C8F0A4
:10395000B3ECEAF06000C8F1D6F06000CCF1D7F02B
:103960001E0ED86F020ED96FDA6BDB6BDC6BDDECF1
:10397000BDF0B65118E10D0EBC6FC30EBD6F440E05
:10398000BE6F020EBF6F0B0EC06FC16B040EC26F15
:10399000C36BC46BC56BC66BC76B6000D8F3C8F054
:1039A000B3ECEAF017D00D0EBC6FC30EBD6F440E22
:1039B000BE6F020EBF6F0D0EC06FC16B040EC26FE3
:1039C000C36BC46BC56BC66BC76B6000D8F3C8F024
:1039D000B3ECEAF0910518E10D0EBC6FC30EBD6F9C
:1039E000440EBE6F020EBF6F040EC06FC16B060E99
:1039F000C26FC36BC46BC56BC66BC76B6000D8F37B
:103A0000C8F0B3ECEAF017D00D0EBC6FC30EBD6F5B
:103A1000440EBE6F020EBF6F1A0EC06FC16B060E52
:103A2000C26FC36BC46BC56BC66BC76B6000D8F34A
:103A3000C8F0B3ECEAF0780ED66FDAECEEF0AED068
:103A4000630EBC6FE50EBD6F070EBE6F020EBF6F3B
:103A5000C06B450EC16F020EC26FC36BC46BC56BEA
:103A6000C66BC76B6000D8F3C8F0B3ECEAF0630E26
:103A7000BC6FE50EBD6F070EBE6F020EBF6FC06B51
:103A8000450EC16F040EC26FC36BC46BC56BC66BB2
:103A9000C76B6000D8F3C8F0B3ECEAF06000C8F17F
:103AA000D6F06000CCF1D7F01E0ED86F020ED96FA1
:103AB000DA6BDB6BDC6BDDECBDF0B65118E10D0EA3
:103AC000BC6FC30EBD6F440EBE6F020EBF6F0A0EF9
:103AD000C06FC16B040EC26FC36BC46BC56BC66B8A
:103AE000C76B6000D8F3C8F0B3ECEAF017D00D0E46
:103AF000BC6FC30EBD6F440EBE6F020EBF6F0C0EC7
:103B0000C06FC16B040EC26FC36BC46BC56BC66B59
:103B1000C76B6000D8F3C8F0B3ECEAF0910518E188
:103B20000D0EBC6FC30EBD6F440EBE6F020EBF6F95
:103B3000050EC06FC16B060EC26FC36BC46BC56B45
:103B4000C66BC76B6000D8F3C8F0B3ECEAF017D0CF
:103B50000D0EBC6FC30EBD6F440EBE6F020EBF6F65
:103B60001B0EC06FC16B060EC26FC36BC46BC56BFF
:103B7000C66BC76B6000D8F3C8F0B3ECEAF0780E00
:103B8000D66FDAECEEF00AD09451010A01E1F8D5D3
:103B9000030A01E1B0D6010A01E152D794C095F0C1
:103BA000966B9E6B1BD00101630518E100017051FB
:103BB000711103E1716B010E706F6000C0F1D6F0FE
:103BC0006000C4F1D7F01E0ED86F020ED96FDA6B09
:103BD000DB6BDC6BDDECBDF00101636B00019E056E
:103BE00001E0A3D08C0530E16000C0F1D6F06000A8
:103BF000C4F1D7F01E0ED86F020ED96FDA6BDB6BF3
:103C0000DC6BDDECBDF070C072F071C073F09151EF
:103C100001E08AD00D0EBC6FC30EBD6F440EBE6FA7
:103C2000020EBF6F040EC06FC16B060EC26FC36B76
:103C3000C46BC56BC66BC76B6000D8F3C8F0B3EC40
:103C4000EAF0010E916F70D0020E95193AE1010170
:103C500062051BE10D0E0001BC6FC30EBD6F440E6B
:103C6000BE6F020EBF6F0D0EC06FC16B040EC26F30
:103C7000C36BC46BC56BC66BC76B6000D8F3C8F071
:103C8000B3ECEAF0010EB66F19D00D0E0001BC6F57
:103C9000C30EBD6F440EBE6F020EBF6F0B0EC06F22
:103CA000C16B040EC26FC36BC46BC56BC66BC76BB5
:103CB0006000D8F3C8F0B3ECEAF0B66B9151AAE01B
:103CC00033D0030E951930E1910517E10D0EBC6F4D
:103CD000C30EBD6F440EBE6F020EBF6F060EC06FE7
:103CE000C16BC26FC36BC46BC56BC66BC76B600027
:103CF000D8F3C8F0B3ECEAF017D00D0EBC6FC30ECA
:103D0000BD6F440EBE6F020EBF6F1C0EC06FC16B45
:103D1000060EC26FC36BC46BC56BC66BC76B60000E
:103D2000D8F3C8F0B3ECEAF09E6B410EBB6F140EF3
:103D3000BC6F985198ECF9F00101636F1200840E8A
:103D4000111901E005D2360E0A6F1B0E0E6F5F0EC1
:103D50000D6F00019F0538E1070ED66F6000D8F3A4
:103D6000D7F0010E8DECFFF0490EEA6FFF0EEB6FFE
:103D70000B0EEC6FF7ECFBF0A30ED66FFF0ED76FB8
:103D8000080ED86FD96B020EDA6FDB6BDC6BDD6B64
:103D9000DE6BDF6B68ECF1F0CC0ED66FFF0ED76FE9
:103DA000060ED86FD96B040EDA6FDB6BDC6BDD6B44
:103DB000DE6BDF6B68ECF1F09F6B010E9E6F946F12
:103DC000966F0101506F4F6F0001960501E1FFD022
:103DD0000CD1630EBC6FE50EBD6F070EBE6F020EF9
:103DE000BF6FC06B600034FCC1F0040EC26FC36BC8
:103DF000C46BC56BC66BC76B6000D8F3C8F0B3EC7F
:103E0000EAF0630EBC6FE50EBD6F070EBE6F020ECB
:103E1000BF6F6B0EC06F600034FCC1F0020EC26F4A
:103E2000C36BC46BC56BC66BC76B6000D8F3C8F0BF
:103E3000B3ECEAF084511AE1890EBC6FEE0EBD6F4F
:103E4000320EBE6F020EBF6F010EC06F600038FCF5
:103E5000C1F0060EC26FC36BC46BC56BC66BC76B7C
:103E60006000D8F3C8F0B3ECEAF0BAD0890EBC6FAA
:103E7000EE0EBD6F320EBE6F020EBF6F040EC06F2E
:103E8000600038FCC1F0060EC26FC36BC46BC56B1B
:103E9000C66BC76B6000D8F3C8F0B3ECEAF0A0D0F3
:103EA000630EBC6FE50EBD6F070EBE6F020EBF6FD7
:103EB000C06B600034FCC1F0C26FC36BC46BC56BD8
:103EC000C66BC76B6000D8F3C8F0B3ECEAF0630EC2
:103ED000BC6FE50EBD6F070EBE6F020EBF6F6B0E9F
:103EE000C06F600034FCC1F0040EC26FC36BC46BC2
:103EF000C56BC66BC76B6000D8F3C8F0B3ECEAF0D3
:103F000084519AE0B3D7630EBC6FE50EBD6F070E08
:103F1000BE6F020EBF6FC06B600034FCC1F0C26F99
:103F2000C36BC46BC56BC66BC76B6000D8F3C8F0BE
:103F3000B3ECEAF0630EBC6FE50EBD6F070EBE6F0B
:103F4000020EBF6FC06B600034FCC1F0040EC26F84
:103F5000C36BC46BC56BC66BC76B6000D8F3C8F08E
:103F6000B3ECEAF0845119E1890EBC6FEE0EBD6F1F
:103F7000320EBE6F020EBF6FC06F600038FCC1F022
:103F8000060EC26FC36BC46BC56BC66BC76B60009C
:103F9000D8F3C8F0B3ECEAF023D0890EBC6FEE0E74
:103FA000BD6F320EBE6F020EBF6F050EC06F600098
:103FB00038FCC1F0060EC26FC36BC46BC56BC66B19
:103FC000C76B6000D8F3C8F0B3ECEAF009D09451A5
:103FD000010A01E1FED6030A01E162D7010A93E07A
:103FE00094C095F0966B9E6B38D0010150051AE194
:103FF0003150321003E1326A010E316E6000C4F0BC
:10400000D6F06000C8F0D7F0600028FCD8F0020EAF
:104010000001D96FDA6BDB6BDC6BDDECBDF001010D
:10402000506B1BD04F0519E12F50301003E1306A5F
:10403000010E2F6E6000BCF0D6F06000C0F0D7F02B
:10404000600028FCD8F0040E0001D96FDA6BDB6B3E
:10405000DC6BDDECBDF001014F6B00019E055FE103
:10406000830512E16000C4F0D6F06000C8F0D7F01C
:10407000600028FCD8F0020ED96FDA6BDB6BDC6BCA
:10408000DDECBDF0986B4AD0820511E16000BCF018
:10409000D6F06000C0F0D7F0600028FCD8F0040E25
:1040A000D96FDA6BDB6BDC6BDDECBDF0EBD7030EAD
:1040B000951934E184511AE1890EBC6FEE0EBD6F83
:1040C000320EBE6F020EBF6F030EC06F600038FC71
:1040D000C1F0060EC26FC36BC46BC56BC66BC76BFA
:1040E0006000D8F3C8F0B3ECEAF018D0890EBC6FCA
:1040F000EE0EBD6F320EBE6F020EBF6F060EC06FAA
:10410000600038FCC1F0C26FC36BC46BC56BC66B7B
:10411000C76B6000D8F3C8F0B3ECEAF09E6B830580
:104120000AE1410EBB6F140EBC6F985198ECF9F088
:104130000101506F12008205D8A41200410EBB6F1E
:10414000140EBC6F985198ECF9F001014F6F1200FA
:10415000110501E0B5D000019F051DE1030EBC6F04
:10416000DF0EBD6F660EBE6F040EBF6F010EC06F17
:10417000650EC16FC26BC36BC46BC56BC66BC76B7F
:104180006000D8F3C8F0B3ECEAF0010E436E010111
:10419000C56F00019F6B060E0101C465060C650E1C
:1041A000436002D0432A35D0030E0001BC6FDF0EFE
:1041B000BD6F660EBE6F040EBF6F020EC06F160E8F
:1041C000C16F040EC26FC36BC46BC56BC66BC76B8C
:1041D0006000D8F3C8F0B3ECEAF08C0EBC6FF70EB9
:1041E000BD6F0F0EBE6F020EBF6F0A0EC06F590E6D
:1041F000C16F060EC26FC36BC46BC56BC66BC76B5A
:104200006000D8F3C8F0B3ECEAF00101C56B010E11
:10421000C36F3A0E436415D0EE0E0001D66F020E46
:10422000D76F050ED86F43506508D96F040EDA6F4B
:10423000DB6BDC6BDD6BDE6B010EDF6FF1ECD4F062
:1042400024D0110E0001D66FFE0ED76F080ED86F66
:10425000D96B040EDA6FDB6BDC6BDD6BDE6B010E92
:10426000DF6FF1ECD4F0EE0ED66F020ED76F050EB5
:10427000D86F2A0ED96F040EDA6FDB6BDC6BDD6B47
:10428000DE6B010EDF6FF1ECD4F0030EBC6FDF0EBE
:10429000BD6F660EBE6F040EBF6F010EC06F435040
:1042A0006508C16FC26BC36BC46BC56BC66BC76B54
:1042B0006000D8F3C8F0B3ECEAF00101C46B12005F
:1042C000030E111942E100019F0517E181050BE181
:1042D000600010F1D6F0D76B100ED86F020ED96FB8
:1042E00042ECD1F009D0D76BD66B100ED86F020E0E
:1042F000D96F050E42ECD1F09F6B01018105D8A466
:10430000120000018105D8A41200630EBC6FE50EF7
:10431000BD6F070EBE6F020EBF6F4450600FC06FBF
:10432000290EC16F050EC26FC36BC46B010EC56F42
:10433000C66BC76B6000D8F3C8F0B3ECEAF060005E
:1043400010F182F10101816B1200040E11193FE19D
:10435000100E056F020E066F00019F050EE1600052
:104360004CF2D6F0D76B600014FCD8F0600018FC5B
:10437000D9F0040E42ECD1F09F6B01017F05D8A467
:104380001200630E0001BC6FE50EBD6F070EBE6F1D
:10439000020EBF6F9351600FC06F03010551190FDB
:1043A0000001C16F03010651030F0001C26FC36B0F
:1043B000C46B010EC56FC66BC76B6000D8F3C8F045
:1043C000B3ECEAF093C080F101017F6B1200050E9F
:1043D000111901E093D0100E0B6F020E0C6F096FD4
:1043E000090E046F00019F050DE1D76B1E0ED66FFD
:1043F00060002CFCD8F0600030FCD9F0030E42ECD9
:10440000D1F09F6B01017F05D8A412000A0E0001B4
:10441000BF6F93517AEC01F0600F0301096F0A0E30
:104420000001BB6F935166EC02F0600F0301046F53
:10443000600E091922E0630E0001BC6FE50EBD6F2E
:10444000070EBE6F020EBF6F600024FCC0F00301B8
:104450000B51150F0001C16F03010C51030F000137
:10446000C26FC36BC46B010EC56FC66BC76B6000B8
:10447000D8F3C8F0B3ECEAF020D0630E0001BC6FB3
:10448000E50EBD6F070EBE6F020EBF6F6C0EC06FE4
:1044900003010B51150F0001C16F03010C51030FF4
:1044A0000001C26FC36BC46B010EC56FC66BC76BD7
:1044B0006000D8F3C8F0B3ECEAF0630EBC6FE50E11
:1044C000BD6F070EBE6F020EBF6F600010FCC0F024
:1044D00003010B511E0F0001C16F03010C51030FAB
:1044E0000001C26FC36BC46B010EC56FC66BC76B97
:1044F0006000D8F3C8F0B3ECEAF064D7060E1119E7
:10450000D8A41200100E076F020E086F00019F055D
:104510000EE1600008F1D6F0D76B60001CFCD8F00B
:10452000600020FCD9F00D0E42ECD1F09F6B010130
:104530007805D8A41200630E0001BC6FE50EBD6FB4
:10454000070EBE6F020EBF6F4250600FC06F0301B7
:104550000751190F0001C16F03010851030F00013A
:10456000C26FC36BC46B010EC56FC66BC76B6000B7
:10457000D8F3C8F0B3ECEAF0600008F179F101017A
:10458000786B1200DAECF8F0F1ECE7F00001BC6BAC
:10459000BB6B73EC03F09E0A07E00001BC6BBB6BC6
:1045A0009E0EBD6FAFECFFF09E0EA4ECFEF0FCEC97
:1045B00003F0210E3A01136F3D017399D28ED28C14
:1045C000010E44ECFFF0F66FF651C3ECF5F0010E6E
:1045D0000001A26F516EC682200EFAEC02F00101BA
:1045E000E46FFAEC03F045ECCFF02FEC03F00001A0
:1045F000CA6B6000E4F0CBF06000E8F0CCF0020E93
:10460000CE6FCD6F040ED06FCF6F090E83ECC8F064
:10461000600028F339F060002CF33AF0010E01013C
:10462000BD6F0001905102E079ECFEF00001905165
:1046300002E094ECFCF07AEC02F0DDEC03F0F6EC36
:10464000E4F00001905102E0D2ECF2F022ECFEF036
:1046500060ECFCF058ECE9F0BDECE5F05FEC01F04B
:1046600001016C051AE1040E0001A21916E0030E07
:10467000A21913E0A20511E0050EA2190EE0905157
:104680000CE0B3510AE1AC5108E1A2C0A1F0050E63
:10469000A26F010E9F6F0101CA6F515002E1F4EC4D
:1046A000FDF00101B4510CE00001905109E1010E4F
:1046B0000101876F6D0E0001A21902E00101B46BC8
:1046C0000201A251A31103E0A207D8A0A307010190
:1046D000870529E10001A20526E00201A251A311EC
:1046E00022E1000EA36F400EA26F6000B0F2EAF06C
:1046F0006000CCF2EBF06000B4F2ECF06000C8F5C2
:10470000EDF0600064F2EEF0600078FAEFF0600027
:104710007CFAF0F0600044F6F1F0010170512DECEC
:10472000E4F00101876F0A0E0001A21901E0EAD24C
:10473000990509E1996B7AC09EF27BC09FF2010E48
:104740000101876F576B0001AD0503E0AE0501E085
:10475000B6D00101605159E1000178517A1903E1A5
:1047600079517B1948E00101226B236B010E000196
:10477000B26F3DD0DDEC03F0000178517A190BE106
:1047800079517B1908E10101B26B226B236B0001A7
:10479000B26B010E9F6F0101235103E1C80E225D30
:1047A00026E30001D76BD66B100ED86F020ED96FBF
:1047B000060E42ECD1F07A51351804E17B513618DF
:1047C00001E19A6B010E0101B26F226B236B0001B4
:1047D000B26B010E9F6F410E0001F46FF00EF36F8C
:1047E000330EE82EFED7F32FFCD7F42FFAD70001B3
:1047F000B20504E1BFD70101B26B616B00017A51D0
:104800007B1103E1010E0101606F01015F5157E16E
:104810003550361002E1010E5F6F000172513518FC
:1048200003E1735136184BE00101226B236B010E3B
:104830000001B26F41D0DDEC03F000017251351878
:1048400011E1735136180EE178517A190BE1795163
:104850007B1908E10101B26B226B236B0001B26B83
:10486000010E9F6F0101235103E1640E225D24E3D9
:104870000001D76BD66B100ED86F020ED96F060EE3
:1048800042ECD1F09A6B6000C8F135F06000CCF1D9
:1048900036F00101226B236B0001B26B010E9F6F9A
:1048A000410E0001F46FF00EF36F330EE82EFED7C9
:1048B000F32FFCD7F42FFAD70001B205BCE00101B9
:1048C000B20503E00001860504E1010E0101856FD8
:1048D00008D00101B25105E10001865102E1010158
:1048E000856B5A0E0001A61904E05A0E59ECF9F036
:1048F000A66FAF51B01904E0AF5164ECEFF0B06FA8
:1049000048502FE0A5512CE1C86B100EC76F26EC64
:1049100002F0000925E16000DCF2BBF03F5058ECEA
:10492000F8F08F6F850518E1120E8F6501D007D062
:10493000030E8F6105D0010E3F6402D0020E8F6F0F
:10494000050E8F6109D0020E8E6106D08D6F8DC06D
:104950008EF0010E0101676F010E01016B6F01D036
:10496000486A010169510001B71910E0010169515C
:10497000EDEC03F0B76F010E0101686F0001B75154
:10498000B61901016A6F5A6B010E596F0001A50536
:1049900012E1010E0101D16F355103E13D0E345D8D
:1049A0000AE30B0E0001A26F0101D16B346B356B72
:1049B000010E00019F6F0001A4051CE101013551AA
:1049C00019E13D0E345D16E2D16B346B356B47A0B7
:1049D00005D000018F6B010E01016B6F47A20AD059
:1049E0003F5008E10001B751010A0101696F5A6B9C
:1049F000010E596F0001C86B100EC76F70EC00F00C
:104A0000000905E0AA5103E1010E0101CC6F00018C
:104A1000C86B100EC76F8FEC00F0000904E00101B5
:104A2000CC6B306B316B0001A90510E101013151F4
:104A300003E1330E305D0AE30C0E0001A26F0101A9
:104A4000CC6B306B316B010E00019F6F01012D515A
:104A500003E1960E2C5D19E3010E00019F6F010129
:104A6000C96B2C6B2D6B0001870503E1010E010161
:104A7000586F0001850503E1010E0101516F00012E
:104A8000860503E1010E0101536FCDECDCF001015D
:104A90008F5101E08F6B0001C86B100EC76F70EC77
:104AA00000F0E80607E0C86B100EC76F8FEC00F04F
:104AB000E8061CE16000A4F2CAF0600084F6CBF0C6
:104AC000600054F6CCF0CD6B0A0E56ECD8F0A96F0E
:104AD00060002CF1CAF060007CF6CBF060004CF670
:104AE000CCF0CD6B0C0E56ECD8F04B6EC86B200E94
:104AF000C76F70EC00F0E80607E0C86B200EC76FC8
:104B00008FEC00F0E8061CE16000A0F2CAF0600043
:104B100080F6CBF0600050F6CCF0CD6B0B0E56EC6F
:104B2000D8F0A86F60009CF2CAF0600078F6CBF075
:104B3000600048F6CCF0CD6B0D0E56ECD8F0A76FA8
:104B4000A8050AE107ECEAF005D0DDEC03F085ECFE
:104B5000E2F0506E5050F9E00001AF0504E1A751BA
:104B6000B2EC02F006D0020EAF1905E1A751B2EC8B
:104B700002F03D6E16D0030EAF1913E18851B2EC6E
:104B800002F03D6E890504E1010E0101556F02D06E
:104B90000101556B000186510101551902E0010E1A
:104BA000546F000185513D180FE03D0405E18EC0B2
:104BB00066F1010E8D6F02D066C18DF08DC08EF052
:104BC000010E0101676F526F0101906B0001A0059A
:104BD0000FE1600080F2CAF0CB6BCC6BCD6B140E92
:104BE00056ECD8F0A06FA05118E1A1C0A2F00AD0F5
:104BF0000001C86B800EC76F8FEC00F0E80605E17E
:104C0000640EA26F010E9F6F06D00001C86B800E6C
:104C1000C76F26EC02F00101906F020E0001C86F11
:104C2000C76B8FEC00F0E80607E0020EC86FC76B99
:104C300070EC00F0E80613E16000A8F2CAF0010E83
:104C4000CB6FCC6FCD6B0E0E56ECD8F0AA6F030E67
:104C5000B01902E0AAC091F1010E0101876F0101B4
:104C6000405102E085ECE2F00001C86B400EC76FD6
:104C700070EC00F0E80609E1010E0101D06F0001BF
:104C80007E6B7F6B010E0101576F0001C86B400EF8
:104C9000C76F26EC02F0E80613E17F5103E1320E04
:104CA0007E5D0EE30101576B0001905109E007ECB6
:104CB000EAF0A2C0A1F0040E0001A26F010E9F6FE6
:104CC000C86B400EC76F8FEC00F0E80610E17F5113
:104CD0000EE1320E7E5D0BE20101D06B00017E6BB6
:104CE0007F6B0101570503E1010E5A1B596F87C005
:104CF00084F10001800502E022EFB9F0A2C0A1F02A
:104D00007DEFB7F00B0EA2192BE1995108E1010ECE
:104D1000996F7AC09EF27BC09FF20101876F1E0ED1
:104D20000001A61904E01E0E59ECF9F0A66F4850D8
:104D300007E08E5108EC01F08D6F010E0101676FE5
:104D40000001A40509E10A0EA26F0101D16B346BC9
:104D5000356B010E00019F6F8005D0E022EFB9F0A6
:104D60000C0EA21901E0F1D0995114E1010E996FD6
:104D70007AC09EF27BC09FF20101876F0001C86B71
:104D8000100EC76F26EC02F0000904E10A0EA26FB4
:104D9000010E9F6FDC0EA61904E0DC0E59ECF9F051
:104DA000A66F485011E06000D8F1BBF06000DCF164
:104DB000BCF016ECF8F06000ECF276F06000F0F277
:104DC00077F0010E0101656F00017651335C775178
:104DD000345809E26000CCF076F06000D0F077F053
:104DE000010E0101656F00017651771105E1776BC6
:104DF000010E766F0101656F0001CA6BCB6BCC6B46
:104E0000CD6B120E56ECD8F0E80607E174C076F0D0
:104E100075C077F0010E0101656F0001CA6BCB6BA5
:104E2000CC6BCD6B130E56ECD8F0E80609E16000B0
:104E3000DCF076F06000E0F077F0010E0101656FC4
:104E40000001C86B100EC76F8FEC00F0000942E044
:104E5000A96B986B76517A1903E177517B1925E09C
:104E60006000D0F137F06000D4F138F07AC074F00F
:104E70007BC075F08B6B8A6B896B886B01015E6BF5
:104E80005D6B5C6B5B6B0001870504E101015A6B94
:104E9000010E596F00018F6B010E01016B6F000154
:104EA0008D6F0101676F616B606B78C09EF279C096
:104EB0009FF2355000017A1904E136507B1901E167
:104EC0009A6B0A0EA26F010E9F6F905103E1050EBF
:104ED00059ECE3F00001C86B100EC76F70EC00F0E6
:104EE000E80607E0C86B100EC76F8FEC00F0E8060D
:104EF0000EE16000A4F2CAF0600084F6CBF060001E
:104F000054F6CCF0CD6B0A0E56ECD8F0A96FC86BF6
:104F1000200EC76F70EC00F0E80608E0C86B200EAA
:104F2000C76F8FEC00F0E80601E016D76000A0F232
:104F3000CAF0600080F6CBF0600050F6CCF0CD6B8C
:104F40000B0E56ECD8F0A86F07D7640EA21979E1C2
:104F5000995108E1010E996F7AC09EF27BC09FF2D1
:104F60000101876F1E0E0001A61904E01E0E59EC08
:104F7000F9F0A66F485009E0600088F2BBF0955147
:104F80002CECFCF0946F010E966FA30502E1010E6C
:104F90009E6FA4050EE01BD0650E09D06E0E07D0E3
:104FA000820E05D0780E03D06D0E01D0640EA26F74
:104FB0000CD09551010AF0E0030AF0E0010AF0E09C
:104FC000070AF0E0010AF0E0F1D7010E9F6FC86B0D
:104FD000400EC76F70EC00F0E80606E1010E01011B
:104FE000D06F00017E6B7F6BC86B400EC76F26ECE5
:104FF00002F0E8060EE17F5103E1510E7E5D09E308
:105000000A0EA26F010E9F6F0101D06B00017E6B33
:105010007F6BC86B400EC76F8FEC00F0E80601E0B5
:105020009BD67F510DE1510E7E5D01E395D60A0EB0
:10503000A26F010E9F6F0101D06B00017E6B7F6B31
:105040008BD6650EA21901E096D1995108E1010EA7
:10505000996F7AC09EF27BC09FF20101876FDC0ED0
:105060000001A61904E0DC0E59ECF9F0A66F4850D7
:1050700011E06000D8F1BBF06000DCF1BCF016EC90
:10508000F8F06000ECF276F06000F0F277F0010EDC
:105090000101656F0001A30503E1010E9E6F986B8E
:1050A000A40540E176517A1903E177517B1925E097
:1050B0006000D0F137F06000D4F138F07AC074F0BD
:1050C0007BC075F08B6B8A6B896B886B01015E6BA3
:1050D0005D6B5C6B5B6B0001870504E101015A6B42
:1050E000010E596F00018F6B010E01016B6F000102
:1050F0008D6F0101676F616B606B78C09EF279C044
:105100009FF2355000017A1904E136507B1901E114
:105110009A6B0A0EA26F010E9F6F905103E1050E6C
:1051200059ECE3F00001CA6BCB6BCC6BCD6B120E6C
:1051300056ECD8F0E80607E174C076F075C077F059
:10514000010E0101656F0001CA6BCB6BCC6BCD6B9F
:10515000130E56ECD8F0E80609E16000DCF076F0BA
:105160006000E0F077F0010E0101656F0001CA6B8D
:10517000CB6BCC6BCD6B0F0E56ECD8F0E8066CE128
:10518000030EB01920E16000D8F1C7F06000DCF137
:10519000C8F05A0EC96F58ECEBF0F36F060EF361CE
:1051A00005D00A0E7627000E772304D03C0E765FDA
:1051B000000E775B775103E13E0E765D4AE3776B35
:1051C0003D0E766F46D0020E0001B0190FE160006F
:1051D000D8F1C7F06000DCF1C8F05A0EC96F58EC86
:1051E000EBF0F36F090EF3611BD02AD00001B0057C
:1051F00033E16000D8F1C7F06000DCF1C8F0540E74
:10520000C96F58ECEBF000090DE16000D8F1C7F070
:105210006000DCF1C8F05A0EC96F58ECEBF0E1D732
:105220005A0E14D06000D8F1C7F06000DCF1C8F06D
:105230005A0EC96F58ECEBF0F36F020EF36105D014
:105240000A0E7627000E772304D0140E765F000E28
:10525000775B010E0101656F0001CA6BCB6BCC6BF4
:10526000CD6B100E56ECD8F0E8062DE1020EB01909
:105270002AE0B00528E16000D8F1C7F06000DCF159
:10528000C8F0540EC96F58ECEBF0000915E160004E
:10529000D8F1C7F06000DCF1C8F0480EC96F58ECD7
:1052A000EBF0F36F090EF36105D0640E7627000E64
:1052B000772306D0840E01D0E80E765F030E775B6D
:1052C000010E0101656F00017651335C775134584E
:1052D00009E26000CCF076F06000D0F077F0010ECB
:1052E0000101656F00017651771105E1776B010EC1
:1052F000766F0101656F0001C86B400EC76F70ECDF
:1053000000F0E8060BE1986B010E0101D06F00017F
:105310007E6B7F6B7AC076F07BC077F0C86B400EF7
:10532000C76F26EC02F0E8060EE17F5103E1510E53
:105330007E5D09E30A0EA26F010E9F6F0101D06B23
:1053400000017E6B7F6BC86B400EC76F8FEC00F067
:10535000E80601E001D57F510DE1510E7E5D01E3CC
:10536000FBD4640EA26F0101D06B00017E6B7F6BDA
:10537000010EF1D4F1D46E0EA21974E1995108E135
:10538000010E996F7AC09EF27BC09FF20101876F78
:105390001E0E0001A61904E01E0E59ECF9F0A66FCE
:1053A000485009E0600088F2BBF095512CECFCF00D
:1053B000946F010E966FA30502E1010E9E6FA40586
:1053C00014E021D06F0EA26F030EE4EC03F018D0AE
:1053D0006F0E0001A26F010EE4EC03F011D0700E0D
:1053E0000001A26F0DD0640EFCD79551010AEAE0CE
:1053F000030AEEE0010AF3E0070AD8A4010AF3D792
:10540000010E00019F6FC86B400EC76F70EC00F07B
:10541000E80606E1010E0101D06F00017E6B7F6B93
:10542000C86B400EC76F26EC02F0E8060EE17F5114
:1054300003E1510E7E5D09E30A0EA26F010E9F6F1C
:105440000101D06B00017E6B7F6BC86B400EC76F94
:105450008FEC00F0E80601E07FD47F5102E173EFAA
:10546000B7F07AD46F0EA21901E0BCD2995108E1CD
:10547000010E996F7AC09EF27BC09FF20101876F87
:10548000080E3F6403D000018F6F3F6E010E0001D4
:105490008D6F8E6F9C5109E19B5107E11E0EA6197D
:1054A00004E01E0E59ECF9F011D09C0507E1A00EA6
:1054B000A61904E0A00E59ECF9F008D09B0507E10D
:1054C000DC0EA61904E0DC0E59ECF9F0A66F48508A
:1054D00033E09C5112E19B5110E1600088F2BBF077
:1054E00095512CECFCF0946F9D0504E1020E94653F
:1054F00001D0946F010E966F1FD09C0509E16C518D
:10550000AEEC00F06C6F6D6B010E01014E6F14D0AC
:1055100000019B0511E16000A0F1BBF06000A4F167
:10552000BCF0D2ECF9F06000ECF268F06000F0F250
:1055300069F0010E01014D6F0001A30503E1986BB5
:10554000010E9E6FA4055BE19C5150E19B5133E03D
:105550004DD0010E9C6F466A9B6B08D09D0509E0FB
:10556000010E9B6F0101866B00019C6B010E986F11
:1055700046D0460444E1010E0101AA6F0001AB6B65
:1055800012D046043CE10101860539E100019D0588
:105590000AE06E51C5ECFDF00101AA6F00016E51E9
:1055A000B1ECF6F0AB6F0101B16B6F0E0001A26FB1
:1055B000010E9F6F24D09551010ACBE0030ACEE083
:1055C000010ADFE01CD09C6B010E466E6CC06EF0D1
:1055D0006DC06FF011D09D050FE09B6B010E0101B6
:1055E000866F68C06AF069C06BF006D00001955103
:1055F000010AE9E0030AEFE0010E0001966F0101E4
:10560000AA0503E00001AB0506E10101B15103E188
:10561000010E0001B26F0001B20548E04AD0DDEC96
:1056200003F000016E5102019C1917E100016F5156
:1056300002019D1912E100016A5102019A190DE15E
:1056400000016B5102019B1908E10101B16B226B52
:10565000236B0001B26B010E9F6F0101235103E127
:10566000C80E225D23E30001D76BD66B100ED86FF6
:10567000020ED96F0B0E42ECD1F0010E0101B16F99
:10568000AA6B0001AB6B0101226B236B0001B26BB3
:10569000010E9F6F410E0001F46FF00EF36F330E99
:1056A000E82EFED7F32FFCD7F42FFAD70001B2056E
:1056B000B6E0600080F2CAF0CB6BCC6BCD6B140E01
:1056C00056ECD8F0A06FA00506E1A2C0A1F00A0E2A
:1056D000A26F010E9F6FCA6BCB6BCC6BCD6B0F0EA5
:1056E00056ECD8F0E80601E0D8D0030EB0191BE163
:1056F0009B0504E1696B010E686F4BD000019C5162
:1057000001E1CBD06000B0F1C7F06000B4F1C8F0A7
:105710005A0EC96F58ECEBF0F36F070EF36101D02E
:10572000B0D0460EB4D0020E0001B01947E19B057F
:1057300033E16000A0F1C7F06000A4F1C8F0480EAA
:10574000C96F58ECEBF0F36F020EF36111D06000FB
:10575000A0F1C7F06000A4F1C8F05A0EC96F58EC70
:10576000EBF0F36F090EF36101D054D05A0E58D00C
:105770006000A0F1C7F06000A4F1C8F05A0EC96F34
:1057800058ECEBF0F36F030EF36101D043D01E0E23
:1057900047D001014D6F81D000019C517EE0600037
:1057A000B0F1C7F06000B4F1C8F05A0EC96F58EC00
:1057B000EBF0F36F090EF36154D063D00001B00534
:1057C0006CE19B0532E16000A0F1C7F06000A4F13C
:1057D000C8F0480EC96F58ECEBF0F36F020EF3619E
:1057E0000BD06000A0F1C7F06000A4F1C8F05A0E21
:1057F000C96F58ECEBF0B5D76000A0F1C7F06000BE
:10580000A4F1C8F05A0EC96F58ECEBF0F36F050E17
:10581000F36105D00A0E6827000E692304D0320E0A
:10582000685F000E695B010EB4D700019C5135E042
:105830006000B0F1C7F06000B4F1C8F0480EC96F65
:1058400058ECEBF0F36F020EF3610DD06000B0F195
:10585000C7F06000B4F1C8F05A0EC96F58ECEBF015
:10586000A8D75A0E14D06000B0F1C7F06000B4F1B0
:10587000C8F05A0EC96F58ECEBF0F36F050EF361E8
:1058800005D00A0E6C27000E6D2304D0320E6C5F1B
:10589000000E6D5B010E01014E6F0001CA6BCB6BF8
:1058A000CC6BCD6B100E56ECD8F0E8064EE1B0058F
:1058B0002FE19B050FE16000A0F1C7F06000A4F1AB
:1058C000C8F0480EC96F58ECEBF0F36F020EF361AD
:1058D00035D02FD000019C5138E06000B0F1C7F006
:1058E0006000B4F1C8F0480EC96F58ECEBF0F36FEC
:1058F000020EF36105D0640E6C27000E6D2304D0F8
:10590000C80E6C5F000E6D5B010E01014E6F1DD065
:10591000020E0001B01919E19B0517E16000A0F12A
:10592000C7F06000A4F1C8F0480EC96F58ECEBF066
:10593000CCD7640E6827000E692304D0C80E685FB8
:10594000000E695B010E01014D6F3E500001F36FC7
:10595000F46B6C51F35D6D51F45904E26000F8F0A2
:105960006CF06D6B68510101085D00016951010126
:10597000095904E208C168F009C169F00001C86B67
:10598000400EC76F70EC00F0E80609E1986B010E5D
:105990000101D06F00017E6B7F6B9B6B9C6BC86BB2
:1059A000400EC76F26EC02F0E8060EE17F5103E1DE
:1059B000510E7E5D09E30A0EA26F010E9F6F010179
:1059C000D06B00017E6B7F6BC86B400EC76F8FEC96
:1059D00000F0E80602E0ACEFA6F07F5101E1CAD189
:1059E000ACEFA6F0700EA21901E0CED1995108E1FA
:1059F000010E996F7AC09EF27BC09FF20101876F02
:105A000000018F6B3F6ADC0EA61904E0DC0E59EC36
:105A1000F9F0A66F485011E0600098F1BBF060000B
:105A20009CF1BCF016ECF8F06000ECF266F060005F
:105A3000F0F267F0010E01014C6F0001A30503E1D4
:105A4000986B010E9E6FA40523E166517A1903E15C
:105A500067517B191BE08B6B8A6B896B886B01012B
:105A60005E6B5D6B5C6B5B6B0001870504E10101A4
:105A70005A6B010E596F010E00018D6F8E6F66C05B
:105A800000F167C001F10101AB6FB16B00019A6BCE
:105A90000101AB0505E1B15103E1010E0001B26F57
:105AA0000001B2054DE04FD0DDEC03F001010051E3
:105AB00002191EE1015103191BE1B16B02C176F01D
:105AC00003C177F002C178F003C179F06000E0F122
:105AD000BBF06000E4F1BCF0E3ECF1F00101AB6B72
:105AE000226B236B0001B26B0A0EA26F010E9F6F37
:105AF0000101235103E1C80E225D22E30001D76BAF
:105B0000D66B100ED86F020ED96F0B0E42ECD1F08F
:105B1000010E0101B16FAB6B226B236B0001B26B05
:105B20000A0EA26F010E9F6F410E0001F46FF00E7E
:105B3000F36F330EE82EFED7F32FFCD7F42FFAD7EE
:105B40000001B205B1E0CA6BCB6BCC6BCD6B120E12
:105B500056ECD8F0E80607E174C066F075C067F04F
:105B6000010E01014C6F0001CA6BCB6BCC6BCD6B8E
:105B7000130E56ECD8F0E80609E16000DCF066F0A0
:105B80006000E0F067F0010E01014C6F0001CA6B8C
:105B9000CB6BCC6BCD6B0F0E56ECD8F0E8066CE1FE
:105BA000030EB01920E1600098F1C7F060009CF18D
:105BB000C8F05A0EC96F58ECEBF0F36F060EF361A4
:105BC00005D00A0E6627000E672304D03C0E665FE0
:105BD000000E675B675103E13E0E665D4AE3676B4B
:105BE0003D0E666F46D0020E0001B0190FE1600055
:105BF00098F1C7F060009CF1C8F05A0EC96F58ECDC
:105C0000EBF0F36F090EF3611BD02AD00001B00551
:105C100033E1600098F1C7F060009CF1C8F0540EC9
:105C2000C96F58ECEBF000090DE1600098F1C7F086
:105C300060009CF1C8F05A0EC96F58ECEBF0E1D748
:105C40005A0E14D0600098F1C7F060009CF1C8F0C3
:105C50005A0EC96F58ECEBF0F36F020EF36105D0EA
:105C60000A0E6627000E672304D0140E665F000E2E
:105C7000675B010E01014C6F0001CA6BCB6BCC6BF3
:105C8000CD6B100E56ECD8F0E8062DE1020EB019DF
:105C90002AE0B00528E1600098F1C7F060009CF1AF
:105CA000C8F0540EC96F58ECEBF0000915E1600024
:105CB00098F1C7F060009CF1C8F0480EC96F58EC2D
:105CC000EBF0F36F090EF36105D0640E6627000E4A
:105CD000672306D0840E01D0E80E665F030E675B73
:105CE000010E01014C6F00016651335C675134585D
:105CF00009E26000CCF066F06000D0F067F0010EC1
:105D000001014C6F00016651671105E1676B010EDF
:105D1000666F01014C6F0001C86B400EC76F70ECDD
:105D200000F0E80607E1986B010E0101D06F000159
:105D30007E6B7F6BC86B400EC76F26EC02F0E806E7
:105D40000EE17F5103E1510E7E5D09E30A0EA26F61
:105D5000010E9F6F0101D06B00017E6B7F6BC86BE2
:105D6000400EC76F8FEC00F0E80602E0ACEFA6F043
:105D70007F5108E1510E7E5D02E3ACEFA6F06E0E9E
:105D800018EFA8F0ACEFA6F0780EA2196EE19951C9
:105D900008E1010E996F7AC09EF27BC09FF201016B
:105DA000876F1E0E0001A61904E01E0E59ECF9F0D3
:105DB000A66F485009E0600088F2BBF095512CECCA
:105DC000FCF0946F010E966FA30502E1010E9E6F29
:105DD000A4050CE019D0790E07D07A0E05D07C0E00
:105DE00003D0810E01D0780EA26F0CD09551010A1C
:105DF000F2E0030AF2E0010AF6E0070AF0E0010A25
:105E0000F0E0F1D7010E9F6FC86B400EC76F70ECCA
:105E100000F0E80606E1010E0101D06F00017E6B83
:105E20007F6BC86B400EC76F26EC02F0E8060EE1F0
:105E30007F5103E1510E7E5D09E30A0EA26F010E50
:105E40009F6F0101D06B00017E6B7F6BC86B400EB2
:105E5000C76F8FEC00F0E80602E0ACEFA6F07F51D0
:105E600002E173EFB7F0ACEFA6F0790EA21965E18D
:105E7000995108E1010E996F7AC09EF27BC09FF2A2
:105E80000101876F1E0E0001A61904E01E0E59ECD9
:105E9000F9F0A66F485008E001017B5110EC00F0CA
:105EA00001017B6F010E7A6F0001A40504E1780EF9
:105EB000A26F010E9F6F600080F2CAF0CB6BCC6BBB
:105EC000CD6B140E56ECD8F0A06FA00506E1A2C071
:105ED000A1F00A0EA26F010E9F6FC86B400EC76F34
:105EE00070EC00F0E80606E1010E0101D06F000140
:105EF0007E6B7F6BC86B400EC76F26EC02F0E80626
:105F00000EE17F5103E1510E7E5D09E30A0EA26F9F
:105F1000010E9F6F0101D06B00017E6B7F6BC86B20
:105F2000400EC76F8FEC00F0E80602E0ACEFA6F081
:105F30007F5101E1ACD3ACEFA6F07A0EA21901E0DB
:105F4000ABD0995108E1010E996F7AC09EF27BC0E7
:105F50009FF20101876F1E0E0001A61904E01E0EBC
:105F600059ECF9F0A66F485009E0600088F2BBF0E8
:105F700095512CECFCF0946F010E966FA30502E195
:105F8000010E9E6FA40508E00FD0020E03D0030E91
:105F900001D0010EAF6F08D09551010AFAE0030A53
:105FA000F4E0010AF4E0F5D7AF51B01932E08F6B9D
:105FB000010E01016B6F00018D6F0101676F000120
:105FC000AF5164ECEFF0B06F8B6B8A6B896B886BB1
:105FD00001015E6B5D6B5C6B5B6B0001A96BA86B79
:105FE0004B6AA76B0101916B0001870504E1010178
:105FF0005A6B010E596F0001860504E10101556BD2
:10600000010E546F0001850504E13D6A010E010196
:10601000526F600080F2CAF00001CB6BCC6BCD6B8D
:10602000140E56ECD8F0A06FA00506E1A2C0A1F0B6
:106030000A0EA26F010E9F6FC86B400EC76F70EC07
:1060400000F0E80606E1010E0101D06F00017E6B51
:106050007F6BC86B400EC76F26EC02F0E8060EE1BE
:106060007F5103E1510E7E5D09E30A0EA26F010E1E
:106070009F6F0101D06B00017E6B7F6BC86B400E80
:10608000C76F8FEC00F0E80602E0ACEFA6F07F519E
:1060900001E1FDD2ACEFA6F07B0EA2193BE19951D4
:1060A00008E1010E996F7AC09EF27BC09FF2010158
:1060B000876F0001C86B400EC76F70EC00F0E806F8
:1060C00006E1010E0101D06F00017E6B7F6BC86B92
:1060D000400EC76F26EC02F0E8060EE17F5103E1A7
:1060E000510E7E5D09E30A0EA26F010E9F6F010142
:1060F000D06B00017E6B7F6BC86B400EC76F8FEC5F
:1061000000F0E80602E0ACEFA6F07F5101E1BFD25B
:10611000ACEFA6F07C0EA21901E02AD2995108E159
:10612000010E996F7AC09EF27BC09FF20101876FCA
:106130001E0E0001A61904E01E0E59ECF9F0A66F20
:10614000485009E0600088F2BBF095512CECFCF05F
:10615000946F010E966FA30502E1010E9E6FA405D8
:1061600001E1CDD1D4D1780EA26F010E9F6FCFD1B6
:106170004F6A010E4E6E5A6A5B6ABED1DDEC03F0C7
:106180000001B25175E1070ED66F6000D8F3D7F069
:10619000020E8DECFFF0D76BD66B100ED86F030E8E
:1061A000D96F0A0E42ECD1F0420EBC6FFD0EBD6FEE
:1061B000070EBE6F010EBF6FC06F1E0EC16F060EC1
:1061C000C26FC36BC46BC56BC66BC76B6000D8F383
:1061D000C8F0B3ECEAF0420EBC6FFD0EBD6F070EC7
:1061E000BE6F010EBF6FC06F250EC16F060EC26F6E
:1061F000C36BC46BC56BC66BC76B6000D8F3C8F0CC
:10620000B3ECEAF0420EBC6FFD0EBD6F070EBE6F21
:10621000010EBF6FC06F2C0EC16F060EC26FC36B35
:10622000C46BC56BC66BC76B6000D8F3C8F0B3EC2A
:10623000EAF0420EBC6FFD0EBD6F070EBE6F010E81
:10624000BF6FC06F330EC16F060EC26FC36BC46BDE
:10625000C56BC66BC76B6000D8F3C8F0B3ECEAF04F
:10626000F56B010E0101C56FB56B010E0001B26F38
:106270001D0E0101C465CED0C46B0001F52BF505E0
:1062800030E1420EBC6FFD0EBD6F070EBE6F010EFA
:10629000BF6FC06F330EC16F060EC26FC36BC46B8E
:1062A000C56BC66BC76B6000D8F3C8F0B3ECEAF0FF
:1062B000420EBC6FFD0EBD6F070EBE6F010EBF6FAD
:1062C000020EC06F1E0EC16F060EC26FC36BC46B91
:1062D000C56BC66BC76B6000D8F3C8F0B3ECEAF0CF
:1062E00099D0020EF51930E1420EBC6FFD0EBD6F64
:1062F000070EBE6F010EBF6FC06F1E0EC16F060E80
:10630000C26FC36BC46BC56BC66BC76B6000D8F341
:10631000C8F0B3ECEAF0420EBC6FFD0EBD6F070E85
:10632000BE6F010EBF6F020EC06F250EC16F060E4D
:10633000C26FC36BC46BC56BC66BC76B6000D8F311
:10634000C8F0B3ECEAF066D0030EF51930E1420E66
:10635000BC6FFD0EBD6F070EBE6F010EBF6FC06F2D
:10636000250EC16F060EC26FC36BC46BC56BC66BC7
:10637000C76B6000D8F3C8F0B3ECEAF0420EBC6F14
:10638000FD0EBD6F070EBE6F010EBF6F020EC06F18
:106390002C0EC16F060EC26FC36BC46BC56BC66B90
:1063A000C76B6000D8F3C8F0B3ECEAF033D0040E4A
:1063B000F51930E1420EBC6FFD0EBD6F070EBE6FCA
:1063C000010EBF6FC06F2C0EC16F060EC26FC36B84
:1063D000C46BC56BC66BC76B6000D8F3C8F0B3EC79
:1063E000EAF0420EBC6FFD0EBD6F070EBE6F010ED0
:1063F000BF6F020EC06F330EC16F060EC26FC36B4C
:10640000C46BC56BC66BC76B6000D8F3C8F0B3EC48
:10641000EAF0F56B4F043EE10101C56BC46B226BE2
:10642000236B0001B26B4E6A0101B56B616B070E05
:106430000001D66F6000D8F3D7F0040E8DECFFF0AA
:10644000D76BD66B100ED86F020ED96F0C0E42ECC4
:10645000D1F07A0E0001F46FC10EF36F810EE82EB9
:10646000FED7F32FFCD7F42FFAD700D00A0E000185
:10647000A26F010E9F6F905107E0030E59ECE3F0FD
:10648000040E59ECE3F006D0010E59ECE3F0020ED5
:1064900059ECE3F0DC0E0101225D050E23592CE3DB
:1064A000C56BC46B226B236B0001B26B4E6A010E8D
:1064B0000101B56F070E0001D66F6000D8F3D7F069
:1064C000040E8DECFFF0D76BD66B100ED86F020E5A
:1064D000D96F0B0E42ECD1F07A0E0001F46FC10EB1
:1064E000F36F810EE82EFED7F32FFCD7F42FFAD7E7
:1064F00000D0010E00019F6F4E0409E13FD600015C
:106500009551010A01E12FD6030A01E131D60001BC
:10651000C86B400EC76F70EC00F0E80606E1010E94
:106520000101D06F00017E6B7F6BC86B400EC76F9F
:1065300026EC02F0E8060EE17F5103E1510E7E5D8C
:1065400009E30A0EA26F010E9F6F0101D06B0001DB
:106550007E6B7F6BC86B400EC76F8FEC00F0E80658
:1065600002E0ACEFA6F07F5101E191D0ACEFA6F0D4
:10657000810EA21901E095D0995108E1010E996FA1
:106580007AC09EF27BC09FF20101876F0001A305D4
:1065900003E1010E0101AE6F0001A4054AE1010112
:1065A000AE0547E16BECDBF00009FCE0070E0001F3
:1065B000C36F0D0E42EC01F0070E0001C36F0F0E0A
:1065C00042EC01F0070E0001C36F0E0E42EC01F029
:1065D000070E0001C36F100E42EC01F045ECCFF046
:1065E000410E0001F46FF00EF36F330EE82EFED76C
:1065F000F32FFCD7F42FFAD7020E0001C36F0D0E54
:1066000042EC01F0020E0001C36F0F0E42EC01F0EC
:10661000030E0001C36F0E0E42EC01F0030E0001E9
:10662000C36F100E42EC01F00A0E0001A26F010EC2
:106630009F6F0001C86B400EC76F70EC00F0E8065A
:1066400006E1010E0101D06F00017E6B7F6BC86B0C
:10665000400EC76F26EC02F0E8060EE17F5103E121
:10666000510E7E5D09E30A0EA26F010E9F6F0101BC
:10667000D06B00017E6B7F6BC86B400EC76F8FECD9
:1066800000F0E80602E0ACEFA6F07F5108E1510E01
:106690007E5D02E3ACEFA6F0780E18EFA8F0ACEF49
:1066A000A6F0820EA21967E1995108E1010E996FD7
:1066B0007AC09EF27BC09FF20101876F1E0E00011F
:1066C000A61904E01E0E59ECF9F0A66F485009E037
:1066D000600088F2BBF095512CECFCF0946F010E39
:1066E000966FA30502E1010E9E6FA4050CE013D086
:1066F000830E07D0840EA26F8F6B3F6A9A6B09D00E
:10670000820EA26F06D09551010AF2E0030AF2E070
:10671000F7D7010E9F6FC86B400EC76F70EC00F08B
:10672000E80606E1010E0101D06F00017E6B7F6B70
:10673000C86B400EC76F26EC02F0E8060EE17F51F1
:1067400003E1510E7E5D09E30A0EA26F010E9F6FF9
:106750000101D06B00017E6B7F6BC86B400EC76F71
:106760008FEC00F0E80602E0ACEFA6F07F5101E10B
:10677000BAD3ACEFA6F0830EA21901E0D1D19951A2
:1067800008E1010E996F7AC09EF27BC09FF2010171
:10679000876F00018C0507E1DC0EA61904E0DC0E12
:1067A00059ECF9F008D08C5107E11E0EA61904E04F
:1067B0001E0E59ECF9F0A66F48501EE08C0512E150
:1067C0006000C0F1BBF06000C4F1BCF016ECF8F062
:1067D0006000ECF270F06000F0F271F0010E010167
:1067E000636F0AD0600088F2BBF0000195512CEC79
:1067F000FCF0946F010E966F0001A30503E1986B06
:10680000010E9E6FA40566E18C5155E05DD0010E2E
:106810008C6F9A6B010E986F916F5CD0B651010A24
:106820000101626F62C1B6F00001B751B6190101F2
:106830006A6F010E0001916F9E6F986B4BD09105AE
:106840002DE17A51701903E17B51711903E0010EBA
:106850009A6F01D09A6B7051351803E17151361857
:106860001EE09A051CE18B6B8A6B896B886B0101BA
:106870005E6B5D6B5C6B5B6B0001870504E1010186
:106880005A6B010E596F00018F6B010E01016B6F86
:1068900000018D6F0101676F5F6B01D09A6B000182
:1068A000986B0A0EA26F010E9F6F905113E1060EB6
:1068B00059ECE3F00FD000019551010AA8E0030A5A
:1068C000ADE0010ABCE006D0950502E18C6B986B47
:1068D000010E966F600080F2CAF00001CB6BCC6BAA
:1068E000CD6B140E56ECD8F0A06FA00506E1A2C047
:1068F000A1F00A0EA26F010E9F6F8C0501E0C4D0BB
:10690000CA6BCB6BCC6BCD6B120E56ECD8F0E80695
:1069100007E174C070F075C071F0010E0101636F82
:106920000001CA6BCB6BCC6BCD6B130E56ECD8F061
:10693000E80609E16000DCF070F06000E0F071F062
:10694000010E0101636F0001CA6BCB6BCC6BCD6B89
:106950000F0E56ECD8F0E80660E1030EB01903E024
:10696000020EB01920E16000C0F1C7F06000C4F170
:10697000C8F05A0EC96F58ECEBF0F36F060EF361D6
:1069800005D00A0E7027000E712304D03C0E705FF4
:10699000000E715B715103E13E0E705D3BE3716B64
:1069A0003D0E706F37D00001B00537E16000C0F1D7
:1069B000C7F06000C4F1C8F0540EC96F58ECEBF09A
:1069C000000911E16000C0F1C7F06000C4F1C8F037
:1069D0005A0EC96F58ECEBF0F36F090EF36101D05A
:1069E00010D05A0E14D06000C0F1C7F06000C4F19E
:1069F000C8F05A0EC96F58ECEBF0F36F020EF3615A
:106A000005D00A0E7027000E712304D0140E705F9B
:106A1000000E715B010E0101636F0001CA6BCB6B4D
:106A2000CC6BCD6B100E56ECD8F0E8062DE1020EC3
:106A3000B0192AE0B00528E16000C0F1C7F060009D
:106A4000C4F1C8F0540EC96F58ECEBF0000915E121
:106A50006000C0F1C7F06000C4F1C8F0480EC96F13
:106A600058ECEBF0F36F090EF36105D0640E70275C
:106A7000000E712306D0840E01D0E80E705F030E65
:106A8000715B010E0101636F0001705101010A5D2C
:106A90000001715101010B5906E20AC170F00BC1EE
:106AA00071F0010E636F00017051711105E1716B9E
:106AB000010E706F0101636F0001C86B400EC76F5C
:106AC00070EC00F0E80609E1986B010E0101D06F4F
:106AD00000017E6B7F6B9A6B8C6BC86B400EC76F2F
:106AE00026EC02F0E8060EE17F5103E1510E7E5DD7
:106AF00009E30A0EA26F010E9F6F0101D06B000126
:106B00007E6B7F6BC86B400EC76F8FEC00F0E806A2
:106B100002E0ACEFA6F07F5101E1A0D1ACEFA6F00E
:106B2000840EA21901E0A4D1995108E1010E996FD8
:106B30007AC09EF27BC09FF20101876F000183053E
:106B400002E0820507E1C80EA61904E0C80E59EC60
:106B5000F9F006D01E0EA61904E01E0E59ECF9F04D
:106B6000A66F485036E083510CE182510AE1600083
:106B700088F2BBF095512CECFCF0946F010E966FEF
:106B800028D0830512E16000C4F0BBF06000C8F0BB
:106B9000BCF016ECF8F06000ECF231F06000F0F2BE
:106BA00032F0010E0101506F14D00001820511E195
:106BB0006000BCF0BBF06000C0F0BCF016ECF8F078
:106BC0006000ECF22FF06000F0F230F0010E0101F5
:106BD0004F6F0001A30503E1986B010E9E6FA405A2
:106BE00001E08DD0835101E082D0825141E07FD01D
:106BF000010E836F826B03D0010E826F836B010ED7
:106C0000986F7DD084511CE1AE5102E1AD512DE071
:106C1000010E0101BB6F00018D6B8E6B8F6B3F6AA4
:106C20000101696B0001B76B06C176F007C177F00F
:106C300006C178F007C179F0010E3C6E846F15D063
:106C40003C0413E0846B0101BB6B1C6B1D6B010EDC
:106C500000018D6F8E6F8F6B3F6A0101696B0001C0
:106C6000B76B0A0EA26F010E9F6F010E000146D096
:106C70009551010ABDE0030ABFE0010AC3E03FD01D
:106C8000836B6000C4F006F16000C8F007F10101F9
:106C90000451065D05510759E8E331282F6E000EB7
:106CA0003220306E6000BCF004F16000C0F005F1ED
:106CB000010E4F6FDAD7826B6000BCF004F1600008
:106CC000C0F005F101010451065D05510759CDE3FE
:106CD000FF0E2F24316EFF0E3020326E6000C4F0A4
:106CE00006F16000C8F007F1010E506FBED7000139
:106CF0009551010AC5E0030ADEE0B7D7966FAE51A1
:106D000002E1AD5172E084055FE13C040DE1010157
:106D10001D5103E10A0E1C5D07E31C6B1D6B020E87
:106D20003C6E0C0E000112D0020E3C1812E1010163
:106D30001D5103E1640E1C5D0CE31C6B1D6B030E07
:106D40003C6E010E696F0001B76F080E8F6F3F6ECA
:106D50003BD0030E3C180EE101011D5103E18C0EE6
:106D60001C5D08E31C6B1D6B040E3C6E00018F6BF9
:106D70003F6A2AD0040E3C1827E101011D5103E1AE
:106D8000280E1C5D21E31C6B1D6B696B0001B76B4A
:106D9000010104510001785D01010551000179599B
:106DA00009E2010E3C6E764B772B76C078F077C007
:106DB00079F00AD0846B0101BB6B1C6B1D6B010E5B
:106DC00000018D6F8E6F966F00017A5102019E193E
:106DD00005E100017B5102019F1907E07AC09EF294
:106DE0007BC09FF2010E0101876F0001C86B400E4E
:106DF000C76F70EC00F0E80611E1846B0101BB6B1A
:106E00001C6B1D6B00018F6B3F6A826B836B986BF1
:106E1000010E0101D06F00017E6B7F6BC86B400ECD
:106E2000C76F26EC02F0E8060EE17F5103E1510E38
:106E30007E5D09E30A0EA26F010E9F6F0101D06B08
:106E400000017E6B7F6BC86B400EC76F8FEC00F04C
:106E5000E80602E0ACEFA6F07F5108E1510E7E5D3E
:106E600002E3ACEFA6F0820E18EFA8F0ACEFA6F0AC
:106E70006D0EA21945E1995108E1010E996F7AC092
:106E80009EF27BC09FF20101876F0001C86B400E2C
:106E9000C76F70EC00F0E80606E1010E0101D06F4B
:106EA00000017E6B7F6BC86B400EC76F26EC02F053
:106EB000E8060EE17F5103E1510E7E5D09E30A0E03
:106EC000A26F010E9F6F0101D06B00017E6B7F6B83
:106ED000C86B400EC76F8FEC00F0E80602E0ACEF25
:106EE000A6F07F5108E1510E7E5D02E3ACEFA6F003
:106EF000640E18EFA8F0ACEFA6F0030EA26FA0D1BD
:106F0000A2056BE10F0E926FC86B800EC76F26EC67
:106F100002F0516E0101255103E18C0E245D1EE348
:106F200051501CE1C36B246B256B0A0E0001A26F4C
:106F3000010E9F6FBC6B070EBB6F73EC03F05A0A18
:106F400007E10001BC6B080EBB6F73EC03F001D0CE
:106F50000D0E0001926F010E0101B66F0001800558
:106F600006E1A2C0A1F0030EA26F010E9F6FC86BD5
:106F7000400EC76F70EC00F0E80606E1010E01015B
:106F8000D06F00017E6B7F6BC86B400EC76F26EC25
:106F900002F0E8060EE17F5103E1320E7E5D09E367
:106FA000040EA26F0A0EA16F010E9F6F7F6B630E1E
:106FB0007E6FC86B400EC76F8FEC00F0E80601E0F3
:106FC00041D17F5103E1320E7E5DD8B03BD101014A
:106FD000D06B00017E6B7F6BF0D0030E0001A21915
:106FE00021E10101325140080001C06F010133511C
:106FF000D8A0E82A01080001C16FC36B640EC26FFC
:107000001DECFFF0C051446E0101821902E0010E37
:10701000816F0001805101E015D1810501E012D19D
:107020003DD00CD1040EA2193DE17E514008C06F45
:107030007F51D8A0E82A0108C16FC36B640EC26FEC
:107040001DECFFF0C051936F0101805100019319B5
:1070500008E0410E7E5D010E7F5903E2010E010141
:107060007F6F0001C86B400EC76F26EC02F0E80688
:107070000DE1400E7E5D010E7F5904E207D085ECE4
:10708000E2F0506E5050FBE0F1EC03F00001C86BF1
:10709000400EC76F8FEC00F0E806C0D7A251A119CF
:1070A000C0E1C9D0050EA21901E08DD00B0ECA6F48
:1070B000B80EC96F8CECFBF001016C5102E06D055C
:1070C0000BE10001A251A11903E10A0EA26F02D047
:1070D000A1C0A2F0010E9F6F0001C86B100EC76F18
:1070E00070EC00F0E80607E0C86B100EC76F8FEC7D
:1070F00000F0E8060EE16000A4F2CAF0600084F639
:10710000CBF0600054F6CCF0CD6B0A0E56ECD8F004
:10711000A96FC86B200EC76F70EC00F0E80607E09F
:10712000C86B200EC76F8FEC00F0E8060EE1600020
:10713000A0F2CAF0600080F6CBF0600050F6CCF010
:10714000CD6B0B0E56ECD8F0A86F800506E1A2C0FF
:10715000A1F0030EA26F010E9F6FC86B400EC76FA8
:1071600070EC00F0E80606E1010E0101D06F0001AD
:107170007E6B7F6BC86B400EC76F26EC02F0E80693
:107180000EE17F5103E1320E7E5D09E3A2C0A1F062
:10719000040EA26F010E9F6F7F6B630E7E6FC86B34
:1071A000400EC76F8FEC00F0E8064CE17F514AE1DA
:1071B000320E7E5D01E20BD745D0000E0101256F36
:1071C0008C0E246F3FD0060E0001A2193BE1E00EA9
:1071D00001011E5D2E0E1F592CE32F0E1E5D310E78
:1071E0001F5912E21E512E080001C06F01011F51EC
:1071F000D8A0E82A31080001C16FC36B640EC26FCA
:107200001DECFFF0C051426E01017951421802E0BD
:10721000010E786F795116E1425014E107ECEAF063
:1072200003D085ECE2F0506E5050FBE0F1EC03F03F
:1072300009D0000133D70A0EA26F02D0A1C0A2F07C
:10724000010E9F6F0001A2512BECB9F0A25100EC8E
:1072500080F011EFA3F0DA6F3B502AE16E0E0001CF
:10726000DA1918E06F0EDA1915E0700EDA1912E06B
:10727000780EDA190FE0790EDA190CE07A0EDA19C5
:1072800009E07B0EDA1906E07C0EDA1903E0810EC4
:10729000DA1907E1600028F1C9F0020E2BECDEF0EC
:1072A0000DD0600028F1C9F0010E2BECDEF006D005
:1072B000600028F1C9F0030E2BECDEF00A0E00018D
:1072C000A21901E005D3AA5101E0AAD1AF0501E05E
:1072D0008AD060002CF2CAF0600060F4CBF060004D
:1072E00064F4CCF0020ECE6FCD6F040ED06FCF6F72
:1072F000010E83ECC8F0600028F318F160002CF355
:1073000019F1600028F2CAF0600058F4CBF0600078
:107310005CF4CCF0020ECE6FCD6F040ED06FCF6F49
:10732000020E83ECC8F0600028F316F160002CF325
:1073300017F1600024F2CAF0600050F4CBF0600056
:1073400054F4CCF0020ECE6FCD6F040ED06FCF6F21
:10735000030E83ECC8F0600028F314F160002CF3F6
:1073600015F1600020F2CAF0600048F4CBF0600034
:107370004CF4CCF0020ECE6FCD6F040ED06FCF6FF9
:1073800083ECC8F0600028F312F160002CF313F1D5
:107390006000A4F2CAF0600040F4CBF0600044F456
:1073A000CCF0020ECE6FCD6F040ED06FCF6F050EF6
:1073B00083ECC8F0600028F310F160002CF311F1A9
:1073C0006000A0F2CAF0600038F4CBF060003CF43A
:1073D000CCF0020ECE6FCD6F040ED06FCF6F060EC5
:1073E00083ECC8F005D2020EAF1901E08AD060002C
:1073F0002CF2CAF0600060F4CBF0600064F4CCF0D2
:10740000020ECE6FCD6F040ED06FCF6F010E83ECE6
:10741000C8F0600028F318F160002CF319F1600047
:1074200028F2CAF0600058F4CBF060005CF4CCF0B5
:10743000020ECE6FCD6F040ED06FCF6F020E83ECB5
:10744000C8F0600028F316F160002CF317F160001B
:1074500024F2CAF0600050F4CBF0600054F4CCF099
:10746000020ECE6FCD6F040ED06FCF6F030E83EC84
:10747000C8F0600028F314F160002CF315F16000EF
:1074800020F2CAF0600048F4CBF060004CF4CCF07D
:10749000020ECE6FCD6F040ED06FCF6F83ECC8F0AD
:1074A000600028F312F160002CF313F16000A4F2E5
:1074B000CAF0600040F4CBF0600044F4CCF0020E5F
:1074C000CE6FCD6F040ED06FCF6F050E83ECC8F07A
:1074D000600028F310F160002CF311F16000A0F2BD
:1074E000CAF0600038F4CBF060003CF4CCF0020E3F
:1074F000CE6FCD6F040ED06FCF6F060E83ECC8F049
:1075000077D1030EAF1901E079D160002CF2CAF0F7
:10751000600060F4CBF0600064F4CCF0020ECE6F3B
:10752000CD6F040ED06FCF6F010E83ECC8F06000FA
:1075300028F318F160002CF319F1600028F2CAF06A
:10754000600058F4CBF060005CF4CCF0020ECE6F1B
:10755000CD6F040ED06FCF6F020E83ECC8F06000C9
:1075600028F316F160002CF317F1600024F2CAF042
:10757000600050F4CBF0600054F4CCF0020ECE6FFB
:10758000CD6F040ED06FCF6F030E83ECC8F0600098
:1075900028F314F160002CF315F1600020F2CAF01A
:1075A000600048F4CBF060004CF4CCF0020ECE6FDB
:1075B000CD6F100ED06FCF6F040E83ECC8F060005B
:1075C00028F312F160002CF313F16000A4F2CAF06A
:1075D000600040F4CBF0600044F4CCF0020ECE6FBB
:1075E000CD6F040ED06FCF6F050E83ECC8F0600036
:1075F00028F310F160002CF311F16000A0F2CAF042
:10760000600038F4CBF060003CF4CCF0020ECE6F9A
:10761000CD6F040ED06FCF6F060E83ECC8F0E8D0AC
:10762000AF0501E08AD0600078F5CAF0600060F430
:10763000CBF0600064F4CCF0020ECE6FCD6F040E80
:10764000D06FCF6F010E83ECC8F0600028F318F103
:1076500060002CF319F1600074F5CAF0600058F472
:10766000CBF060005CF4CCF0020ECE6FCD6F040E58
:10767000D06FCF6F020E83ECC8F0600028F316F1D4
:1076800060002CF317F1600070F5CAF0600050F450
:10769000CBF0600054F4CCF0020ECE6FCD6F040E30
:1076A000D06FCF6F030E83ECC8F0600028F314F1A5
:1076B00060002CF315F160006CF5CAF0600048F42E
:1076C000CBF060004CF4CCF0020ECE6FCD6F040E08
:1076D000D06FCF6F83ECC8F0600028F312F1600028
:1076E0002CF313F160002CF1CAF0600040F4CBF0F1
:1076F000600044F4CCF0020ECE6FCD6F040ED06F5C
:10770000CF6F050E83ECC8F0600028F310F1600025
:107710002CF311F160009CF2CAF0600038F4CBF059
:1077200060003CF4CCF0020ECE6FCD6F100ED06F27
:10773000CF6F060E83ECC8F05BD0020EAF192BE1C1
:1077400060002CF1CAF0600040F4CBF0600044F41B
:10775000CCF0020ECE6FCD6F040ED06FCF6F050E42
:1077600083ECC8F0600028F310F160002CF311F1F5
:1077700060009CF2CAF0600038F4CBF060003CF48A
:10778000CCF0020ECE6FCD6F100ED06FCF6F060E05
:1077900083ECC8F02DD0030EAF1930E160002CF15E
:1077A000CAF0600040F4CBF0600044F4CCF0020E6C
:1077B000CE6FCD6F040ED06FCF6F050E83ECC8F087
:1077C000600028F310F160002CF311F160009CF2CE
:1077D000CAF0600038F4CBF060003CF4CCF0020E4C
:1077E000CE6FCD6F040ED06FCF6F060E83ECC8F056
:1077F000600028F30EF160002CF30FF16000A8F296
:10780000CAF0600090FACBF0600094FACCF0020E5F
:10781000CE6FCD6F040ED06FCF6F0A0E83ECC8F021
:10782000600028F3A4F260002CF3A5F2600040F69B
:10783000CAF0600098FACBF060009CFACCF0020E1F
:10784000CE6FCD6F040ED06FCF6F080E83ECC8F0F3
:10785000600028F3A6F260002CF3A7F20101585152
:107860001DE10001C86B400EC76F26EC02F0CA6F25
:107870006000F0F1CBF06000F4F1CCF0020ECE6FBE
:10788000CD6F040ED06FCF6F070E83ECC8F0600091
:1078900028F37CF060002CF37DF01200600060F5AE
:1078A000CAF06000F0F1CBF06000F4F1CCF0020E11
:1078B0000001CE6FCD6F200ED06FCF6F070E83EC1F
:1078C000C8F0600028F37CF060002CF37DF012001B
:1078D000040EDA191CE1C86B400EC76F26EC02F0EB
:1078E000CA6F6000F0F1CBF06000F4F1CCF0020E52
:1078F000CE6FCD6F100ED06FCF6F070E83ECC8F038
:10790000600028F37CF060002CF37DF012006D0E17
:10791000A2191CE1C86B400EC76F26EC02F0CA6FBB
:107920006000F0F1CBF06000F4F1CCF0020ECE6F0D
:10793000CD6F040ED06FCF6F070E83ECC8F06000E0
:1079400028F37CF060002CF37DF01200780EA21971
:107950001CE1C86B400EC76F26EC02F0CA6F6000D6
:10796000F0F1CBF06000F4F1CCF0020ECE6FCD6FF1
:10797000040ED06FCF6F070E83ECC8F0600028F3C1
:107980007CF060002CF37DF01200700EA2191CE157
:10799000C86B400EC76F26EC02F0CA6F6000F0F1B2
:1079A000CBF06000F4F1CCF0020ECE6FCD6F040E80
:1079B000D06FCF6F070E83ECC8F0600028F37CF027
:1079C00060002CF37DF012006F0EA2191CE1C86B51
:1079D000400EC76F26EC02F0CA6F6000F0F1CBF0EA
:1079E0006000F4F1CCF0020ECE6FCD6F040ED06FBC
:1079F000CF6F070E83ECC8F0600028F37CF06000C6
:107A00002CF37DF012006E0EA2191CE1C86B400E23
:107A1000C76F26EC02F0CA6F6000F0F1CBF0600097
:107A2000F4F1CCF0020ECE6FCD6F040ED06FCF6F9D
:107A3000070E83ECC8F0600028F37CF060002CF3A4
:107A40007DF01200830EA2191CE1C86B400EC76FB7
:107A500026EC02F0CA6F6000F0F1CBF06000F4F1A8
:107A6000CCF0020ECE6FCD6F040ED06FCF6F070E2D
:107A700083ECC8F0600028F37CF060002CF37DF00C
:107A80001200650EA2191CE1C86B400EC76F26ECF0
:107A900002F0CA6F6000F0F1CBF06000F4F1CCF0BE
:107AA000020ECE6FCD6F040ED06FCF6F070E83EC3A
:107AB000C8F0600028F37CF060002CF37DF0120029
:107AC000640EA2191CE1C86B400EC76F26EC02F0D1
:107AD000CA6F6000F0F1CBF06000F4F1CCF0020E60
:107AE000CE6FCD6F040ED06FCF6F070E83ECC8F052
:107AF000600028F37CF060002CF37DF012000B0E88
:107B0000A2191CE1C86B400EC76F26EC02F0CA6FC9
:107B10006000F0F1CBF06000F4F1CCF0020ECE6F1B
:107B2000CD6F040ED06FCF6F070E83ECC8F06000EE
:107B300028F37CF060002CF37DF01200820EA21975
:107B40001CE1C86B400EC76F26EC02F0CA6F6000E4
:107B5000F0F1CBF06000F4F1CCF0020ECE6FCD6FFF
:107B6000040ED06FCF6F070E83ECC8F0600028F3CF
:107B70007CF060002CF37DF01200840EA219D8A4D2
:107B80001200C86B400EC76F26EC02F0CA6F60008F
:107B9000F0F1CBF06000F4F1CCF0020ECE6FCD6FBF
:107BA000040ED06FCF6F070E83ECC8F0600028F38F
:107BB0007CF060002CF37DF01200D805E26F6000CD
:107BC00058F3C0F060005CF3C1F0270EC36F100ED5
:107BD000C26F1DECFFF0C051100FDD6F270EBE6F9E
:107BE000100EBD6F600058F3BBF060005CF3BCF09A
:107BF000D0ECFFF06000ECF2C0F06000F0F2C1F0F9
:107C0000030EC36FE80EC26F1DECFFF0C051100FE2
:107C1000DE6F030EBE6FE80EBD6F600058F3BBF061
:107C200060005CF3BCF0D0ECFFF06000ECF2C0F060
:107C30006000F0F2C1F0C36B640EC26F1DECFFF088
:107C4000C051100FDF6FBE6B640EBD6F600058F344
:107C5000BBF060005CF3BCF0D0ECFFF06000ECF235
:107C6000C0F06000F0F2C1F0C36B0A0EC26F1DECF1
:107C7000FFF0C051100FE06F600058F3BBF06000E0
:107C80005CF3BCF0BE6B0A0EBD6FD0ECFFF0BB51D5
:107C9000100FE16F970503E0985101E0C5D1100E78
:107CA000D65D270ED75901E292D0630EBC6FE50E68
:107CB000BD6F070EBE6F020EBF6F600074F3C0F0A1
:107CC000600060F3C1F0600064F3C2F0600068F32C
:107CD000C3F060006CF3C4F0600070F3C5F0C66BD5
:107CE000C76B6000D8F3C8F0B3ECEAF0630EBC6F6A
:107CF000E50EBD6F070EBE6F020EBF6F600078F31A
:107D0000C0F0D851080FC16F600064F3C2F060008A
:107D100068F3C3F060006CF3C4F0600070F3C5F06A
:107D2000C66BC76B6000D8F3C8F0B3ECEAF0630E23
:107D3000BC6FE50EBD6F070EBE6F020EBF6F600019
:107D40007CF3C0F0D851100FC16F600064F3C2F033
:107D5000600068F3C3F060006CF3C4F0600070F37F
:107D6000C5F0C66BC76B6000D8F3C8F0B3ECEAF09F
:107D7000630EBC6FE50EBD6F070EBE6F020EBF6FC8
:107D8000600080F3C0F0D851180FC16F600064F339
:107D9000C2F0600068F3C3F060006CF3C4F06000F0
:107DA00070F3C5F0C66BC76B6000D8F3C8F0B3ECD6
:107DB000EAF0630EBC6FE50EBD6F070EBE6F020EDC
:107DC000BF6F600084F3C0F0D851200FB4D1E80E2B
:107DD000D65D030ED75971E3630EBC6FE50EBD6F20
:107DE000070EBE6F020EBF6F600078F3C0F0600038
:107DF00060F3C1F0600064F3C2F0600068F3C3F0A8
:107E000060006CF3C4F0600070F3C5F0C66BC76B24
:107E10006000D8F3C8F0B3ECEAF0630EBC6FE50E77
:107E2000BD6F070EBE6F020EBF6F60007CF3C0F027
:107E3000D851080FC16F600064F3C2F0600068F3AE
:107E4000C3F060006CF3C4F0600070F3C5F0C66B63
:107E5000C76B6000D8F3C8F0B3ECEAF0630EBC6FF8
:107E6000E50EBD6F070EBE6F020EBF6F600080F3A0
:107E7000C0F0D851100FC16F600064F3C2F0600011
:107E800068F3C3F060006CF3C4F0600070F3C5F0F9
:107E9000C66BC76B6000D8F3C8F0B3ECEAF0630EB2
:107EA000BC6FE50EBD6F070EBE6F020EBF6F6000A8
:107EB00084F3C0F0D851180F3ED1D75103E1640EBE
:107EC000D65D50E3630EBC6FE50EBD6F070EBE6F4F
:107ED000020EBF6F60007CF3C0F0600060F3C1F081
:107EE000600064F3C2F0600068F3C3F060006CF3FC
:107EF000C4F0600070F3C5F0C66BC76B6000D8F3C8
:107F0000C8F0B3ECEAF0630EBC6FE50EBD6F070E70
:107F1000BE6F020EBF6F600080F3C0F0D851080F33
:107F2000C16F600064F3C2F0600068F3C3F06000EA
:107F30006CF3C4F0600070F3C5F0C66BC76B6000F3
:107F4000D8F3C8F0B3ECEAF0630EBC6FE50EBD6F7A
:107F5000070EBE6F020EBF6F600084F3C0F0D851F1
:107F6000100FE9D0D75103E10A0ED65D2FE3630E5F
:107F7000BC6FE50EBD6F070EBE6F020EBF6F6000D7
:107F800080F3C0F0600060F3C1F0600064F3C2F001
:107F9000600068F3C3F060006CF3C4F0600070F33D
:107FA000C5F0C66BC76B6000D8F3C8F0B3ECEAF05D
:107FB000630EBC6FE50EBD6F070EBE6F020EBF6F86
:107FC000600084F3C0F0D851080FB5D0630EBC6FC9
:107FD000E50EBD6F070EBE6F020EBF6FC06BE251A4
:107FE000090FC16F600064F3C2F0600068F3C3F072
:107FF00060006CF3C4F0600070F3C5F0C66BC76B33
:108000006000D8F3C8F0B3ECEAF0630EBC6FE50E85
:10801000BD6F070EBE6F020EBF6F600084F3C0F02D
:10802000600060F3C1F088D0630EBC6FE50EBD6FD9
:10803000070EBE6F020EBF6FC06B600088F3C1F009
:10804000600064F3C2F0600068F3C3F060006CF39A
:10805000C4F0600070F3C5F0C66BC76B6000D8F366
:10806000C8F0B3ECEAF0630EBC6FE50EBD6F070E0F
:10807000BE6F020EBF6FC06BE251070FC16F600091
:1080800064F3C2F0600068F3C3F060006CF3C4F006
:10809000600070F3C5F0C66BC76B6000D8F3C8F022
:1080A000B3ECEAF0630EBC6FE50EBD6F070EBE6F5A
:1080B000020EBF6FC06BE2510E0FC16F600064F320
:1080C000C2F0600068F3C3F060006CF3C4F06000BD
:1080D00070F3C5F0C66BC76B6000D8F3C8F0B3ECA3
:1080E000EAF0630EBC6FE50EBD6F070EBE6F020EA9
:1080F000BF6FC06BE251150FC16F600064F3C2F037
:10810000600068F3C3F060006CF3C4F0600070F3CB
:10811000C5F0C66BC76B6000D8F3C8F0B3ECEAF0EB
:10812000630EBC6FE50EBD6F070EBE6F020EBF6F14
:10813000C06BE2511B0FC16F600064F3C2F06000BE
:1081400068F3C3F060006CF3C4F0600070F3C5F036
:10815000C66BC76B6000D8F3C8F0B3EFEAF06000FD
:1081600058F3C0F060005CF3C1F0270EC36F100E2F
:10817000C26F1DECFFF0C051100FDD6F270EBE6FF8
:10818000100EBD6F600058F3BBF060005CF3BCF0F4
:10819000D0ECFFF06000ECF2C0F06000F0F2C1F053
:1081A000030EC36FE80EC26F1DECFFF0C051100F3D
:1081B000DE6F030EBE6FE80EBD6F600058F3BBF0BC
:1081C00060005CF3BCF0D0ECFFF06000ECF2C0F0BB
:1081D0006000F0F2C1F0C36B640EC26F1DECFFF0E3
:1081E000C051100FDF6FBE6B640EBD6F600058F39F
:1081F000BBF060005CF3BCF0D0ECFFF06000ECF290
:10820000C0F06000F0F2C1F0C36B0A0EC26F1DEC4B
:10821000FFF0C051100FE06F600058F3BBF060003A
:108220005CF3BCF0BE6B0A0EBD6FD0ECFFF0BB512F
:10823000100FE16FB00EBC6FF50EBD6F050EBE6F77
:10824000010EBF6FC06B600060F3C1F0600064F3AB
:10825000C2F0600068F3C3F060006CF3C4F060002B
:1082600070F3C5F0C66BC76B6000D8F3C8F0B3EC11
:10827000EAF0B00EBC6FF50EBD6F050EBE6F010EBD
:10828000BF6FC06BD851060FC16F600064F3C2F0BE
:10829000600068F3C3F060006CF3C4F0600070F33A
:1082A000C5F0C66BC76B6000D8F3C8F0B3ECEAF05A
:1082B000B00EBC6FF50EBD6F050EBE6F010EBF6F29
:1082C000C06BD8510C0FC16F600064F3C2F0600046
:1082D00068F3C3F060006CF3C4F0600070F3C5F0A5
:1082E000C66BC76B6000D8F3C8F0B3ECEAF0B00E11
:1082F000BC6FF50EBD6F050EBE6F010EBF6FC06B7C
:10830000D851120FC16F600064F3C2F0600068F3CF
:10831000C3F060006CF3C4F0600070F3C5F0C66B8E
:10832000C76B6000D8F3C8F0B3ECEAF0B00EBC6FD6
:10833000F50EBD6F050EBE6F010EBF6FC06BD8513D
:10834000180FC16F600064F3C2F0600068F3C3F0FF
:1083500060006CF3C4F0600070F3C5F0C66BC76BCF
:108360006000D8F3C8F0B3ECEAF0100ED65D270E2B
:10837000D75901E292D0B00EBC6FF50EBD6F050E5D
:10838000BE6F010EBF6F600074F3C0F0600060F359
:10839000C1F0600064F3C2F0600068F3C3F06000F5
:1083A0006CF3C4F0600070F3C5F0C66BC76B60007F
:1083B000D8F3C8F0B3ECEAF0B00EBC6FF50EBD6FA9
:1083C000050EBE6F010EBF6F600078F3C0F0D8518C
:1083D000060FC16F600064F3C2F0600068F3C3F081
:1083E00060006CF3C4F0600070F3C5F0C66BC76B3F
:1083F0006000D8F3C8F0B3ECEAF0B00EBC6FF50E35
:10840000BD6F050EBE6F010EBF6F60007CF3C0F044
:10841000D8510C0FC16F600064F3C2F0600068F3C4
:10842000C3F060006CF3C4F0600070F3C5F0C66B7D
:10843000C76B6000D8F3C8F0B3ECEAF0B00EBC6FC5
:10844000F50EBD6F050EBE6F010EBF6F600080F3AD
:10845000C0F0D851120FC16F600064F3C2F0600029
:1084600068F3C3F060006CF3C4F0600070F3C5F013
:10847000C66BC76B6000D8F3C8F0B3ECEAF0B00E7F
:10848000BC6FF50EBD6F050EBE6F010EBF6F6000B5
:1084900084F3C0F0D851180FFED0E80ED65D030E5D
:1084A000D75971E3B00EBC6FF50EBD6F050EBE6FF0
:1084B000010EBF6F600078F3C0F0600060F3C1F0A0
:1084C000600064F3C2F0600068F3C3F060006CF316
:1084D000C4F0600070F3C5F0C66BC76B6000D8F3E2
:1084E000C8F0B3ECEAF0B00EBC6FF50EBD6F050E30
:1084F000BE6F010EBF6F60007CF3C0F0D851060F55
:10850000C16F600064F3C2F0600068F3C3F0600004
:108510006CF3C4F0600070F3C5F0C66BC76B60000D
:10852000D8F3C8F0B3ECEAF0B00EBC6FF50EBD6F37
:10853000050EBE6F010EBF6F600080F3C0F0D85112
:108540000C0FC16F600064F3C2F0600068F3C3F009
:1085500060006CF3C4F0600070F3C5F0C66BC76BCD
:108560006000D8F3C8F0B3ECEAF0B00EBC6FF50EC3
:10857000BD6F050EBE6F010EBF6F600084F3C0F0CB
:10858000D851120F88D0D75103E1640ED65D50E365
:10859000B00EBC6FF50EBD6F050EBE6F010EBF6F46
:1085A00060007CF3C0F0600060F3C1F0600064F331
:1085B000C2F0600068F3C3F060006CF3C4F06000C8
:1085C00070F3C5F0C66BC76B6000D8F3C8F0B3ECAE
:1085D000EAF0B00EBC6FF50EBD6F050EBE6F010E5A
:1085E000BF6F600080F3C0F0D851060FC16F60000C
:1085F00064F3C2F0600068F3C3F060006CF3C4F091
:10860000600070F3C5F0C66BC76B6000D8F3C8F0AC
:10861000B3ECEAF0B00EBC6FF50EBD6F050EBE6F89
:10862000010EBF6F600084F3C0F0D8510C0F33D03F
:10863000D75103E10A0ED65D30E3B00EBC6FF50EE4
:10864000BD6F050EBE6F010EBF6F600080F3C0F0FE
:10865000600060F3C1F0600064F3C2F0600068F392
:10866000C3F060006CF3C4F0600070F3C5F0C66B3B
:10867000C76B6000D8F3C8F0B3ECEAF0B00EBC6F83
:10868000F50EBD6F050EBE6F010EBF6F600084F367
:10869000C0F0D851060FC16F0ED0B00EBC6FF50EF2
:1086A000BD6F050EBE6F010EBF6F600084F3C0F09A
:1086B000600060F3C1F0600064F3C2F0600068F332
:1086C000C3F060006CF3C4F0600070F3C5F0C66BDB
:1086D000C76B6000D8F3C8F0B3EFEAF0D841E842C6
:1086E0003F0B030D6F00CCFFDFF0DA054FE16C0E9E
:1086F000BC6FFC0EBD6FDF516608BE6F010EBF6F11
:10870000C06B60007CF3C1F0600064F3C2F0C36B27
:10871000C46BC56FC66BC76B6000D8F3C8F0B3EC11
:10872000EAF06C0EBC6FFC0EBD6FDF516608BE6FC9
:10873000010EBF6FC06B60007CF3C1F0D929C26F1E
:10874000C36BC46B010EC56FC66BC76B6000D8F3FB
:10875000C8F0B3ECEAF06C0EBC6FFC0EBD6FDF51DD
:108760006608BE6F010EBF6FC06B60007CF3C1F086
:10877000D951020FC26FC36BC46B010EC56FC66BBC
:10878000C76B6000D8F3C8F0B3ECEAF0040ED75D15
:1087900004E3030ED76FD66906D0D651D71103E193
:1087A000D76B010ED66F600058F3C0F060005CF329
:1087B000C1F0030EC36FE80EC26F1DECFFF0C05195
:1087C000DB6F030EBE6FE80EBD6F600058F3BBF0A9
:1087D00060005CF3BCF0D0ECFFF06000ECF2C0F0A5
:1087E0006000F0F2C1F0C36B640EC26F1DECFFF0CD
:1087F000C051DC6FBE6B640EBD6F600058F3BBF000
:1088000060005CF3BCF0D0ECFFF06000ECF2C0F074
:108810006000F0F2C1F0C36B0A0EC26F1DECFFF0F6
:10882000C051DD6F600058F3BBF060005CF3BCF03A
:10883000BE6B0A0EBD6FD0ECFFF0BB51DE6F97052B
:1088400003E0985101E0B5D1E80ED65D030ED7598B
:1088500063E3450EBC6FF10EBD6F0A0EBE6F030ED3
:10886000BF6F60006CF3C0F0600060F3C1F06000A7
:1088700064F3C2F0C36BC46B600068F3C5F0C66BF1
:10888000C76B6000D8F3C8F0B3ECEAF0450EBC6FDC
:10889000F10EBD6F0A0EBE6F030EBF6F600070F366
:1088A000C0F0D8510D0FC16F600064F3C2F0C36B0C
:1088B000C46B600068F3C5F0C66BC76B6000D8F38B
:1088C000C8F0B3ECEAF0450EBC6FF10EBD6F0A0EB6
:1088D000BE6F030EBF6F600074F3C0F0D8511A0F63
:1088E000C16F600064F3C2F0C36BC46B600068F3D7
:1088F000C5F0C66BC76B6000D8F3C8F0B3ECEAF004
:10890000450EBC6FF10EBD6F0A0EBE6F030EBF6F3A
:10891000600078F3C0F083D0D75104E1640ED65DD7
:1089200001E280D0450EBC6FF10EBD6F0A0EBE6F26
:10893000030EBF6F140EC06F600060F3C1F06000E3
:1089400064F3C2F0C36BC46B600068F3C5F0C66B20
:10895000C76B6000D8F3C8F0B3ECEAF0450EBC6F0B
:10896000F10EBD6F0A0EBE6F030EBF6F600070F395
:10897000C0F0600060F3C1F0600064F3C2F0C36B4C
:10898000C46B600068F3C5F0C66BC76B6000D8F3BA
:10899000C8F0B3ECEAF0450EBC6FF10EBD6F0A0EE5
:1089A000BE6F030EBF6F600074F3C0F0D8510D0F9F
:1089B000C16F600064F3C2F0C36BC46B600068F306
:1089C000C5F0C66BC76B6000D8F3C8F0B3ECEAF033
:1089D000450EBC6FF10EBD6F0A0EBE6F030EBF6F6A
:1089E000600078F3C0F0D8511A0FC16F600064F3D3
:1089F000C2F0C36BC46B600068F3C5F0C66BC76B95
:108A00006000D8F3C8F0B3ECEAF0450EBC6FF10E8D
:108A1000BD6F0A0EBE6F030EBF6F140EC06FD8512C
:108A2000260F5BD0D75103E10A0ED65D60E3450EF9
:108A3000BC6FF10EBD6F0A0EBE6F030EBF6F140E3A
:108A4000C06F600060F3C1F0600064F3C2F0C36BFC
:108A5000C46B600068F3C5F0C66BC76B6000D8F3E9
:108A6000C8F0B3ECEAF0450EBC6FF10EBD6F0A0E14
:108A7000BE6F030EBF6F140EC06FD851260FC16FAB
:108A8000600064F3C2F0C36BC46B600068F3C5F0B0
:108A9000C66BC76B6000D8F3C8F0B3ECEAF0450EC4
:108AA000BC6FF10EBD6F0A0EBE6F030EBF6F60008C
:108AB00074F3C0F0D8510D0FC16F600064F3C2F0C1
:108AC000C36BC46B600068F3C5F0C66BC76B600016
:108AD000D8F3C8F0B3ECEAF05ED0C16F600064F385
:108AE000C2F0C36BC46B600068F3C5F0A8D0450E3C
:108AF000BC6FF10EBD6F0A0EBE6F030EBF6F140E7A
:108B0000C06F600060F3C1F0600064F3C2F0C36B3B
:108B1000C46B600068F3C5F0C66BC76B6000D8F328
:108B2000C8F0B3ECEAF0450EBC6FF10EBD6F0A0E53
:108B3000BE6F030EBF6F140EC06FD8510D0FC16F03
:108B4000600064F3C2F0C36BC46B600068F3C5F0EF
:108B5000C66BC76B6000D8F3C8F0B3ECEAF0450E03
:108B6000BC6FF10EBD6F0A0EBE6F030EBF6F140E09
:108B7000C06FD851260FC16F600064F3C2F0C36BA1
:108B8000C46B600068F3C5F0C66BC76B6000D8F3B8
:108B9000C8F0B3ECEAF0450EBC6FF10EBD6F0A0EE3
:108BA000BE6F030EBF6F600078F3C0F0D8511A0F8C
:108BB00094D76C0EBC6FFC0EBD6FD8516608BE6FAB
:108BC000010EBF6FC06B600060F3C1F0600064F322
:108BD000C2F0C36BC46BC56BC66BC76B6000D8F3C8
:108BE000C8F0B3ECEAF06C0EBC6FFC0EBD6FD85150
:108BF0006608BE6F010EBF6FC06B600060F3C1F00E
:108C0000D929C26FC36BC46BC56BC66BC76B6000E1
:108C1000D8F3C8F0B3ECEAF06C0EBC6FFC0EBD6F7D
:108C2000D8516608BE6F010EBF6FC06B600060F365
:108C3000C1F0D951020FC26FC36BC46BC56BC66B59
:108C4000C76B6000D8F3C8F0B3EFEAF000017651CB
:108C5000D61905E17751D71902E1DD6B08D07051C3
:108C6000D61905E17151D71902E1010EDD6F040E2D
:108C7000D75D04E3030ED76FD66906D0D651D7115E
:108C800003E1D76B010ED66F600058F3C0F06000AF
:108C90005CF3C1F0030EC36FE80EC26F1DECFFF072
:108CA000C051100FD86F030EBE6FE80EBD6F60008D
:108CB00058F3BBF060005CF3BCF0D0ECFFF0600058
:108CC000ECF2C0F06000F0F2C1F0C36B640EC26F52
:108CD0001DECFFF0C051100FD96FBE6B640EBD6F5D
:108CE000600058F3BBF060005CF3BCF0D0ECFFF028
:108CF0006000ECF2C0F06000F0F2C1F0C36B0A0E4D
:108D0000C26F1DECFFF0C051100FDA6F600058F316
:108D1000BBF060005CF3BCF0BE6B0A0EBD6FD0EC24
:108D2000FFF0BB51100FDB6F450404E001018551DA
:108D300001E081D100019A0501E07DD1E80ED65D08
:108D4000030ED7595FE3630EBC6FE50EBD6F070ED0
:108D5000BE6F020EBF6F600060F3C0F0C16BDD51EB
:108D6000020DF350030FC26FC36BC46BC56BC66BB0
:108D7000C76B6000D8F3C8F0B3ECEAF0630EBC6FC9
:108D8000E50EBD6F070EBE6F020EBF6F600064F38D
:108D9000C0F0090EC16FDD51020DF350030FC26F19
:108DA000C36BC46BC56BC66BC76B6000D8F3C8F0F0
:108DB000B3ECEAF0630EBC6FE50EBD6F070EBE6F3D
:108DC000020EBF6F600068F3C0F0120EC16FDD517C
:108DD000020DF350030FC26FC36BC46BC56BC66B40
:108DE000C76B6000D8F3C8F0B3ECEAF0630EBC6F59
:108DF000E50EBD6F070EBE6F020EBF6F60006CF315
:108E0000C0F070D1D75103E1640ED65D6DE3630EFF
:108E1000BC6FE50EBD6F070EBE6F020EBF6FC06B5D
:108E2000C16BDD51020DF350030FC26FC36BC46BF6
:108E3000C56BC66BC76B6000D8F3C8F0B3ECEAF043
:108E4000630EBC6FE50EBD6F070EBE6F020EBF6FE7
:108E5000600064F3C0F0C16BDD51020DF350030FED
:108E6000C26FC36BC46BC56BC66BC76B6000D8F3B6
:108E7000C8F0B3ECEAF0630EBC6FE50EBD6F070EF1
:108E8000BE6F020EBF6F600068F3C0F0090EC16FC5
:108E9000DD51020DF350030FC26FC36BC46BC56B82
:108EA000C66BC76B6000D8F3C8F0B3ECEAF0630E92
:108EB000BC6FE50EBD6F070EBE6F020EBF6F600088
:108EC0006CF3C0F0120EC16FDD51020DF350030FB1
:108ED000C26FC36BC46BC56BC66BC76B6000D8F346
:108EE000C8F0B3ECEAF0F5D0D75103E10A0ED65D35
:108EF00052E3630EBC6FE50EBD6F070EBE6F020E30
:108F0000BF6FC06BC16BDD51020DF350030FC26F19
:108F1000C36BC46BC56BC66BC76B6000D8F3C8F07E
:108F2000B3ECEAF0630EBC6FE50EBD6F070EBE6FCB
:108F3000020EBF6F600068F3C0F0090EC16FDD5113
:108F4000020DF350030FC26FC36BC46BC56BC66BCE
:108F5000C76B6000D8F3C8F0B3ECEAF0630EBC6FE7
:108F6000E50EBD6F070EBE6F020EBF6F60006CF3A3
:108F7000C0F0120EC16FDD51020DF350030FC26F2E
:108F8000C36BC46BC56BC66BC76B6000D8F3C8F00E
:108F9000B3ECEAF09ED0630EBC6FE50EBD6F070E1A
:108FA000BE6F020EBF6FC06BC16BDD51020DF3507F
:108FB000030FC26FC36BC46BC56BC66BC76B60001E
:108FC000D8F3C8F0B3ECEAF0630EBC6FE50EBD6FEA
:108FD000070EBE6F020EBF6FC06B090EC16FDD5171
:108FE000020DF350030FC26FC36BC46BC56BC66B2E
:108FF000C76B6000D8F3C8F0B3ECEAF0630EBC6F47
:10900000E50EBD6F070EBE6F020EBF6F60006CF302
:10901000C0F0120EC16FDD51020DF350030FC26F8D
:10902000C36BC46BC56BC66BC76B6000D8F3C8F06D
:10903000B3ECEAF04ED0630E0001BC6FE50EBD6FDD
:10904000070EBE6F020EBF6FC06BC16BDD51020D0C
:10905000F350030FC26FC36BC46BC56BC66BC76B9A
:109060006000D8F3C8F0B3ECEAF0630EBC6FE50E15
:10907000BD6F070EBE6F020EBF6FC06B090EC16FD2
:10908000DD51020DF350030FC26FC36BC46BC56B90
:10909000C66BC76B6000D8F3C8F0B3ECEAF0630EA0
:1090A000BC6FE50EBD6F070EBE6F020EBF6FC06BCB
:1090B000120EC16FDD51020DF350030FC26FC36B6F
:1090C000C46BC56BC66BC76B6000D8F3C8F0B3EC5C
:1090D000EAF0630EBC6FE50EBD6F070EBE6F020EA9
:1090E000BF6FC06B1A0EC16FDD51020DF350030F3D
:1090F000C26FC36BC46BC56BC66BC76B6000D8F324
:10910000C8F0B3EFEAF0D36F600030F3D4F0600042
:109110002CF3D5F0600040F3D6F060003CF3D7F0BC
:10912000600038F3D8F0600034F3D9F01ED2CA5191
:109130001DE1D451D8190AE0D851CEECFEF0C36F2E
:10914000050E42EC01F0600060F3D4F00001D5514F
:10915000D91901E129D2D951CEECFEF0C36F010E2D
:1091600042EC01F0600064F3D5F01ED2D451D61960
:109170000AE0D651CEECFEF0C36F050E42EC01F0D2
:10918000600058F3D4F00001D551D71901E10CD299
:10919000D751CEECFEF0C36F010E42EC01F060003F
:1091A0005CF3D5F001D2CA511AE1D451D8190AE0C2
:1091B000D851CEECFEF0C36F060E42EC01F0600019
:1091C00060F3D4F00001D551D91901E1EDD1D951A5
:1091D000CEECFEF0C36F020E42EC01F0C3D7D451C7
:1091E000D6190AE0D651CEECFEF0C36F060E42EC63
:1091F00001F0600058F3D4F00001D551D71901E116
:10920000D3D1D751CEECFEF0C36F020E42EC01F089
:10921000C6D7CA511AE1D451D8190AE0D851CEECB8
:10922000FEF0C36F070E42EC01F0600060F3D4F073
:109230000001D551D91901E1B7D1D951CEECFEF0D9
:10924000C36F030E42EC01F08DD7D451D6190AE05A
:10925000D651CEECFEF0C36F070E42EC01F0600079
:1092600058F3D4F00001D551D71901E19DD1D75160
:10927000CEECFEF0C36F030E42EC01F090D7CA5162
:109280001AE1D451D8190AE0D851CEECFEF0C36FE0
:10929000080E42EC01F0600060F3D4F00001D551FB
:1092A000D91901E181D1D951CEECFEF0C36F040E82
:1092B00042EC01F057D7D451D6190AE0D651CEEC82
:1092C000FEF0C36F080E42EC01F0600058F3D4F0DA
:1092D0000001D551D71901E167D1D751CEECFEF08D
:1092E000C36F040E42EC01F05AD7CA511AE1D451AF
:1092F000D8190AE0D851CEECFEF0C36F0B0E42EC49
:1093000001F0600060F3D4F00001D551D91901E1FA
:109310004BD1D951CEECFEF0C36F090E42EC01F0F7
:1093200021D7D451D6190AE0D651CEECFEF0C36F46
:109330000B0E42EC01F0600058F3D4F00001D5515F
:10934000D71901E131D1D751CEECFEF0C36F090E30
:1093500042EC01F024D7CA511AE1D451D8190AE0DD
:10936000D851CEECFEF0C36F0C0E42EC01F0600061
:1093700060F3D4F00001D551D91901E115D1D951CB
:10938000CEECFEF0C36F0A0E42EC01F0EBD6D451E6
:10939000D6190AE0D651CEECFEF0C36F0C0E42ECAB
:1093A00001F0600058F3D4F00001D551D71901E164
:1093B000FBD0D751CEECFEF0C36F0A0E42EC01F0A9
:1093C000EED6CA511AE1D451D8190AE0D851CEECE0
:1093D000FEF0C36F0F0E42EC01F0600060F3D4F0BA
:1093E0000001D551D91901E1DFD0D951CEECFEF001
:1093F000C36F0D0E42EC01F0B5D6D451D6190AE078
:10940000D651CEECFEF0C36F0F0E42EC01F06000BF
:1094100058F3D4F00001D551D71901E1C5D0D75187
:10942000CEECFEF0C36F0D0E42EC01F0B8D6CA517F
:109430001AE1D451D8190AE0D851CEECFEF0C36F2E
:10944000100E42EC01F0600060F3D4F00001D55141
:10945000D91901E1A9D0D951CEECFEF0C36F0E0E9F
:1094600042EC01F07FD6D451D6190AE0D651CEECA9
:10947000FEF0C36F100E42EC01F0600058F3D4F020
:109480000001D551D71901E18FD0D751CEECFEF0B4
:10949000C36F0E0E42EC01F082D6CA5119E1D451CD
:1094A000D8190AE0D851CEECFEF0C36F130E42EC8F
:1094B00001F0600060F3D4F00001D551D91974E0D7
:1094C000D951CEECFEF0C36F110E42EC01F04AD63A
:1094D000D451D6190AE0D651CEECFEF0C36F130E6C
:1094E00042EC01F0600058F3D4F00001D551D719D7
:1094F0005BE0D751CEECFEF0C36F110E42EC01F0F1
:109500004ED6CA5119E1D451D8190AE0D851CEEC3F
:10951000FEF0C36F140E42EC01F0600060F3D4F073
:109520000001D551D91940E0D951CEECFEF0C36FFE
:10953000120E42EC01F016D6D451D6190AE0D651DB
:10954000CEECFEF0C36F140E42EC01F0600058F355
:10955000D4F00001D551D71927E0D751CEECFEF059
:10956000C36F120E42EC01F01AD60001D351010A6A
:1095700001E1DDD5030A01E116D6010A01E149D670
:10958000070A01E17CD6010A01E1AFD6030A01E135
:10959000E2D6010A01E115D70F0A01E148D7010A15
:1095A00001E17BD7030AADE00001D451D16FD55161
:1095B000CA6F600044F3CBF012006C0EBC6FFC0E5F
:1095C000BD6F660EBE6F010EBF6FC06BD8512D0F01
:1095D000C16F600064F3C2F0C36BC46BC56BC66B34
:1095E000C76B6000D8F3C8F0B3ECEAF06C0EBC6F48
:1095F000FC0EBD6F660EBE6F010EBF6FC06BD85103
:109600002D0FC16FD929C26FC36BC46BC56BC66BFD
:10961000C76B6000D8F3C8F0B3ECEAF0DA0537E1C5
:109620006C0EBC6FFC0EBD6FD8513608BE6F010EBC
:10963000BF6FC06BD8512D0FC16F600064F3C2F0D3
:10964000C36BC46B600068F3C5F0C66BC76B60008A
:10965000D8F3C8F0B3ECEAF06C0EBC6FFC0EBD6F33
:10966000D8513608BE6F010EBF6FC06BD8512D0F99
:10967000C16FD929C26FC36BC46B600068F3C5F0BA
:10968000C66BC76B6000D8F3C8F0B3ECEAF0040E09
:10969000D75D03E3030ED76FD669300ED82760007D
:1096A00058F3C0F060005CF3C1F0030EC36FE80E26
:1096B000C26F1DECFFF0C051100FDB6F030EBE6FC9
:1096C000E80EBD6F600058F3BBF060005CF3BCF0C7
:1096D000D0ECFFF06000ECF2C0F06000F0F2C1F0FE
:1096E000C36B640EC26F1DECFFF0C051100FDC6F36
:1096F000BE6B640EBD6F600058F3BBF060005CF39E
:10970000BCF0D0ECFFF06000ECF2C0F06000F0F2D2
:10971000C1F0C36B0A0EC26F1DECFFF0C051100FF9
:10972000DD6F600058F3BBF060005CF3BCF0BE6B13
:109730000A0EBD6FD0ECFFF0BB51100FDE6F970526
:1097400003E09851D8A41200E80ED65D030ED75955
:1097500058E3630EBC6FE50EBD6F070EBE6F020EC1
:10976000BF6F60006CF3C0F0600060F3C1F0600098
:1097700064F3C2F0C36BC46B600068F3C5F0C66BE2
:10978000C76B6000D8F3C8F0B3ECEAF0630EBC6FAF
:10979000E50EBD6F070EBE6F020EBF6F600070F367
:1097A000C0F0D851080FC16F600064F3C2F0C36B02
:1097B000C46B600068F3C5F0C66BC76B6000D8F37C
:1097C000C8F0B3ECEAF0630EBC6FE50EBD6F070E98
:1097D000BE6F020EBF6F600074F3C0F0D851100F5F
:1097E000C16F600064F3C2F0C36BC46B600068F3C8
:1097F000C5F0C66BC76B6000D8F3C8F0B3ECEAF0F5
:1098000005D1D75103E1640ED65D56E3630EBC6FFC
:10981000E50EBD6F070EBE6F020EBF6FC06B60001E
:1098200060F3C1F0600064F3C2F0C36BC46B60000E
:1098300068F3C5F0C66BC76B6000D8F3C8F0B3EC33
:10984000EAF0630EBC6FE50EBD6F070EBE6F020E31
:10985000BF6F600070F3C0F0D851080FC16F600097
:1098600064F3C2F0C36BC46B600068F3C5F0C66BF1
:10987000C76B6000D8F3C8F0B3ECEAF0630EBC6FBE
:10988000E50EBD6F070EBE6F020EBF6F600074F372
:10989000C0F0D851100FC16F600064F3C2F0C36B09
:1098A000C46B600068F3C5F0C66BC76B6000D8F38B
:1098B000C8F0B3ECEAF0AAD0D75103E10A0ED65DA6
:1098C00054E3630EBC6FE50EBD6F070EBE6F020E54
:1098D000BF6FC06B600060F3C1F0600064F3C2F062
:1098E000C36BC46B600068F3C5F0C66BC76B6000E8
:1098F000D8F3C8F0B3ECEAF0630EBC6FE50EBD6FB1
:10990000070EBE6F020EBF6FC06BD851080FC16F3C
:10991000600064F3C2F0C36BC46B600068F3C5F011
:10992000C66BC76B6000D8F3C8F0B3ECEAF0630E07
:10993000BC6FE50EBD6F070EBE6F020EBF6F6000FD
:1099400074F3C0F0D851100FC16F600064F3C2F01F
:10995000C36BC46B600068F3C5F0C66BC76B600077
:10996000D8F3C8F0B3ECEAF051D0630EBC6FE50E4B
:10997000BD6F070EBE6F020EBF6FC06B600060F35D
:10998000C1F0600064F3C2F0C36BC46B600068F3A5
:10999000C5F0C66BC76B6000D8F3C8F0B3ECEAF053
:1099A000630EBC6FE50EBD6F070EBE6F020EBF6F7C
:1099B000C06BD851080FC16F600064F3C2F0C36B75
:1099C000C46B600068F3C5F0C66BC76B6000D8F36A
:1099D000C8F0B3ECEAF0630EBC6FE50EBD6F070E86
:1099E000BE6F020EBF6FC06BD851100FC16F600009
:1099F00064F3C2F0C36BC46B600068F3C5F0C66B60
:109A0000C76B6000D8F3C8F0B3ECEAF0630EBC6F2C
:109A1000E50EBD6F070EBE6F020EBF6F600078F3DC
:109A2000C0F0D851180FC16F600064F3C2F0C36B6F
:109A3000C46B600068F3C5F0C66BC76B6000D8F3F9
:109A4000C8F0B3EFEAF0040ED75D04E3030ED76F5E
:109A5000D66906D0D651D71103E1D76B010ED66F68
:109A6000600058F3C0F060005CF3C1F0030EC36FF8
:109A7000E80EC26F1DECFFF0C051D86F030EBE6F31
:109A8000E80EBD6F600058F3BBF060005CF3BCF003
:109A9000D0ECFFF06000ECF2C0F06000F0F2C1F03A
:109AA000C36B640EC26F1DECFFF0C051D96FBE6B6B
:109AB000640EBD6F600058F3BBF060005CF3BCF057
:109AC000D0ECFFF06000ECF2C0F06000F0F2C1F00A
:109AD000C36B0A0EC26F1DECFFF0C051DA6F60005D
:109AE00058F3BBF060005CF3BCF0BE6B0A0EBD6FB8
:109AF000D0ECFFF0BB51DB6F450404E00101855160
:109B000001E063D1E80E0001D65D030ED75955E39D
:109B1000450EBC6FF10EBD6F0A0EBE6F030EBF6F18
:109B2000600060F3C0F0C16BC26FC36BC46BC56BE8
:109B3000C66BC76B6000D8F3C8F0B3ECEAF0450E13
:109B4000BC6FF10EBD6F0A0EBE6F030EBF6F6000DB
:109B500064F3C0F00D0EC16F030EC26FC36BC46B14
:109B6000C56BC66BC76B6000D8F3C8F0B3ECEAF006
:109B7000450EBC6FF10EBD6F0A0EBE6F030EBF6FB8
:109B8000600068F3C0F01A0EC16F030EC26FC36BA2
:109B9000C46BC56BC66BC76B6000D8F3C8F0B3EC81
:109BA000EAF0450EBC6FF10EBD6F0A0EBE6F030EDC
:109BB000BF6F60006CF3C0F05AD1D75103E1640E5F
:109BC000D65D61E3450EBC6FF10EBD6F0A0EBE6F30
:109BD000030EBF6F140EC06FC16B030EC26FC36B59
:109BE000C46BC56BC66BC76B6000D8F3C8F0B3EC31
:109BF000EAF0450EBC6FF10EBD6F0A0EBE6F030E8C
:109C0000BF6F600064F3C0F0C16BC26FC36BC46B05
:109C1000C56BC66BC76B6000D8F3C8F0B3ECEAF055
:109C2000450EBC6FF10EBD6F0A0EBE6F030EBF6F07
:109C3000600068F3C0F00D0EC16F030EC26FC36BFE
:109C4000C46BC56BC66BC76B6000D8F3C8F0B3ECD0
:109C5000EAF0450EBC6FF10EBD6F0A0EBE6F030E2B
:109C6000BF6F60006CF3C0F01A0EC16F030EC26FBD
:109C7000C36BC46BC56BC66BC76B6000D8F3C8F011
:109C8000B3ECEAF0EAD0D75103E10A0ED65D49E31E
:109C9000450EBC6FF10EBD6F0A0EBE6F030EBF6F97
:109CA000140EC06FC16B030EC26FC36BC46BC56B68
:109CB000C66BC76B6000D8F3C8F0B3ECEAF0450E92
:109CC000BC6FF10EBD6F0A0EBE6F030EBF6F140E98
:109CD000C06F260EC16F030EC26FC36BC46BC56B22
:109CE000C66BC76B6000D8F3C8F0B3ECEAF0450E62
:109CF000BC6FF10EBD6F0A0EBE6F030EBF6F60002A
:109D000068F3C0F00D0EC16F030EC26FC36BC46B5E
:109D1000C56BC66BC76B6000D8F3C8F0B3ECEAF054
:109D200047D0450EBC6FF10EBD6F0A0EBE6F030E1D
:109D3000BF6F140EC06FC16B030EC26FC36BC46BD9
:109D4000C56BC66BC76B6000D8F3C8F0B3ECEAF024
:109D5000450EBC6FF10EBD6F0A0EBE6F030EBF6FD6
:109D6000140EC06F0D0EC16F030EC26FC36BC46BB8
:109D7000C56BC66BC76B6000D8F3C8F0B3ECEAF0F4
:109D8000450EBC6FF10EBD6F0A0EBE6F030EBF6FA6
:109D9000140EC06F260EC16F030EC26FC36BC46B6F
:109DA000C56BC66BC76B6000D8F3C8F0B3ECEAF0C4
:109DB000450EBC6FF10EBD6F0A0EBE6F030EBF6F76
:109DC00060006CF3C0F01A0E53D0450E0001BC6F5A
:109DD000F10EBD6F0A0EBE6F030EBF6F140EC06F83
:109DE000C16B030EC26FC36BC46BC56BC66BC76B15
:109DF0006000D8F3C8F0B3ECEAF0450EBC6FF10E8A
:109E0000BD6F0A0EBE6F030EBF6F140EC06F0D0E36
:109E1000C16F030EC26FC36BC46BC56BC66BC76BE0
:109E20006000D8F3C8F0B3ECEAF0450EBC6FF10E59
:109E3000BD6F0A0EBE6F030EBF6F140EC06F1A0EF9
:109E4000C16F030EC26FC36BC46BC56BC66BC76BB0
:109E50006000D8F3C8F0B3ECEAF0450EBC6FF10E29
:109E6000BD6F0A0EBE6F030EBF6F140EC06F260EBD
:109E7000C16F030EC26FC36BC46BC56BC66BC76B80
:109E80006000D8F3C8F0B3EFEAF0420E0001B46FFF
:109E9000010E0101B86F416E766F5A6A5B6A010E5E
:109EA000B96F00018D6F8F6B0101696B020E64EC5D
:109EB000EFF0AF6F0B0E476E0D0E926F92C07BF1FD
:109EC000010E01017A6F0001BC6BBB6F73EC03F0F4
:109ED0005A0A0AE10001BC6B020EBB6F73EC03F07F
:109EE0005B6E010E0101B96F0001BC6B030EBB6F0D
:109EF00073EC03F05A0A07E10001BC6B040EBB6F60
:109F000073EC03F05A6E0001BC6B050EBB6F73EC73
:109F100003F05A0A1BE10001BC6B060EBB6F73EC29
:109F200003F0000913E00001BC6B060EBB6F73EC7D
:109F300003F00001BD6F040EBD6108D0BC6B060EBE
:109F4000BB6F73EC03F064ECEFF0AF6F0001BC6B20
:109F5000070EBB6F73EC03F05A0A1EE10001BC6BE5
:109F6000080EBB6F73EC03F00001BD6F070EBD65FB
:109F700013D0BC6B080EBB6F73EC03F00001BD6F18
:109F8000130EBD6109D0BC6B080EBB6F73EC03F000
:109F90000001926F92C07BF10001BC6B090EBB6F98
:109FA00073EC03F05A0A02E10B0E476E0001BC6B22
:109FB0000B0EBB6F73EC03F05A0A15E10001BC6B8A
:109FC0000C0EBB6F73EC03F00001B16F010E0101C9
:109FD000B86F420E0001B16506D0470EB16103D0E3
:109FE000010E0101776F0001BC6B0D0EBB6F73ECAE
:109FF00003F05A0A0AE10001BC6B0E0EBB6F73EC52
:10A0000003F0416E010E0101766F0001BC6B0F0E73
:10A01000BB6F73EC03F05A0A28E10001BC6B100E11
:10A02000BB6F73EC03F00001C06FC0511F0B3F6E9C
:10A030006000FCF08FF0010E01016B6F0001C03970
:10A04000E842070B010BB76FB7C069F1C045E8469E
:10A05000030B010B0101626F62C1B6F00001B75141
:10A06000B61901016A6F010E686F0001BC6B110E19
:10A07000BB6F73EC03F05A0A41E10001BC6B120E96
:10A08000BB6F73EC03F00001C16FC151070B8E6F02
:10A090008EC08DF0010E0101676F0001C139E846E5
:10A0A0001F0B010B856F600014F23DF0010E0101E2
:10A0B000526F0001C1390F0B010B866F86C055F13D
:10A0C000010E0101546F0001C139E842070B010B79
:10A0D000876F87C05AF1010E0101596F0001870592
:10A0E00004E1010E0101576F586F0001C145E846B8
:10A0F000030B010B8B6FC145010B886F0001BC6B1B
:10A10000200EBB6F73EC03F05B0A21E10001BC6B16
:10A11000220EBB6F73EC03F00001BD6FBC6B210E10
:10A12000BB6F73EC03F00001BE6FBD51766F600032
:10A13000F8F277F0765177110AE07651335C775177
:10A14000345805E376C078F077C079F005D0000187
:10A15000776B3D0E766FF6D7BC6B230EBB6F73EC3F
:10A1600003F05B0A1FE10001BC6B250EBB6F73ECB3
:10A1700003F00001BD6FBC6B240EBB6F73EC03F0EA
:10A180000001BE6FBD51746F6000F8F275F074513C
:10A19000751105E07451335C7551345803E2756BE9
:10A1A0003D0E746F0001BC6B260EBB6F73EC03F0A9
:10A1B0005B0A1FE10001BC6B280EBB6F73EC03F060
:10A1C0000001BD6FBC6B270EBB6F73EC03F0000189
:10A1D000BE6FBD51376E6000F8F238F0375038105E
:10A1E00005E03750335C3850345803E2386A3D0E8E
:10A1F000376E0001BC6B290EBB6F73EC03F05B0A7A
:10A2000038E10001BC6B2B0EBB6F73EC03F0000157
:10A21000BD6FBC6B2A0EBB6F73EC03F00001BE6F09
:10A22000BD51706F6000F8F271F07051711118E05B
:10A23000705101010A5D0001715101010B5910E3D8
:10A2400070C072F071C073F000017851701903E1B1
:10A250007951711903E0010E9A6F0BD09A6B09D0F6
:10A260000001716B3D0E706F70C072F071C073F0C1
:10A27000F5D700018F51D8B41200010E01015A6FB9
:10A28000596F010CDA6F270E0001BE6F100EBD6F03
:10A29000600058F3BBF060005CF3BCF0D0ECFFF062
:10A2A0006000ECF2C0F06000F0F2C1F0030EC36F8A
:10A2B000E80EC26F1DECFFF0030EBE6FE80EBD6F1F
:10A2C000600058F3BBF060005CF3BCF0D0ECFFF032
:10A2D0006000ECF2C0F06000F0F2C1F0C36B640EFD
:10A2E000C26F1DECFFF0BE6B640EBD6F600058F3D3
:10A2F000BBF060005CF3BCF0D0ECFFF06000ECF26F
:10A30000C0F06000F0F2C1F0C36B0A0EC26F1DEC2A
:10A31000FFF0C051600FDB6F600058F3BBF06000CE
:10A320005CF3BCF0BE6B0A0EBD6FD0ECFFF0BB510E
:10A33000600FDC6F7AD1210EBC6FAF0EBD6F440E83
:10A34000BE6F050EBF6F020EC06F600060F3C1F0FC
:10A35000600064F3C2F0C36BC46B010EC56FC66BC3
:10A36000C76B6000D8F3C8F0B3ECEAF0630EBC6FC3
:10A37000E50EBD6F070EBE6F020EBF6F600070F37B
:10A38000C0F0D851190FC16FD951030FC26FC36B01
:10A39000C46B010EC56FC66BC76B6000D8F3C8F005
:10A3A000B3ECEAF035D1210EBC6FAF0EBD6F440E99
:10A3B000BE6F050EBF6F030EC06F600060F3C1F08B
:10A3C000600064F3C2F0C36BC46B010EC56FC66B53
:10A3D000C76B6000D8F3C8F0B3ECEAF0630EBC6F53
:10A3E000E50EBD6F070EBE6F020EBF6F60006CF30F
:10A3F000C0F0D851150FC16FD951030FC26FC36B95
:10A40000C46B010EC56FC66BC76B6000D8F3C8F094
:10A41000B3ECEAF0630EBC6FE50EBD6F070EBE6FC6
:10A42000020EBF6F600070F3C0F0D8511E0FC16FF5
:10A43000D951030FC26FC36BC46B010EC56FC66BDE
:10A44000C76B6000D8F3C8F0B3ECEAF0630EBC6FE2
:10A45000E50EBD6F070EBE6F020EBF6F6A0EC06FB6
:10A46000D851280F38D0210EBC6FAF0EBD6F440EEF
:10A47000BE6F050EBF6F040EC06F600060F3C1F0C9
:10A48000600064F3C2F0C36BC46B010EC56FC66B92
:10A49000C76B6000D8F3C8F0B3ECEAF0630EBC6F92
:10A4A000E50EBD6F070EBE6F020EBF6F600070F34A
:10A4B000C0F0D851190FC16FD951030FC26FC36BD0
:10A4C000C46B010EC56FC66BC76B6000D8F3C8F0D4
:10A4D000B3ECEAF09DD0C16FD951030FC26F09D020
:10A4E000210EBC6FAF0EBD6F440EBE6F050EBF6F69
:10A4F00050D0C36BC46B010EC56FC66BC76B6000D9
:10A50000D8F3C8F0B3EFEAF0210EBC6FAF0EBD6F09
:10A51000440EBE6F050EBF6F060E3BD0210EBC6F02
:10A52000AF0EBD6F440EBE6F050EBF6F070E31D06C
:10A53000210EBC6FAF0EBD6F440EBE6F050EBF6F18
:10A54000080E27D0210EBC6FAF0EBD6F440EBE6F3C
:10A55000050EBF6F090E1DD0210EBC6FAF0EBD6F73
:10A56000440EBE6F050EBF6F0A0E13D0210EBC6FD6
:10A57000AF0EBD6F440EBE6F050EBF6F0B0E09D040
:10A58000210EBC6FAF0EBD6F440EBE6F050EBF6FC8
:10A590000C0EC06F600060F3C1F0600064F3C2F0A5
:10A5A000A8D7210EBC6FAF0EBD6F440EBE6F050E57
:10A5B000BF6F0D0EC06F600060F3C1F0600064F308
:10A5C000C2F0C36BC46B010EC56FC66BC76B600076
:10A5D000D8F3C8F0B3ECEAF0630EBC6FE50EBD6FC4
:10A5E000070EBE6F020EBF6F600070F3C0F0D8514F
:10A5F000190FC16FD951030FC26FC36BC46B010E2A
:10A60000C56FC66BC76B6000D8F3C8F0B3ECEAF057
:10A61000630EBC6FE50EBD6F070EBE6F020EBF6FFF
:10A620006A0EC06FD851230F56D7DA51020A01E1E2
:10A6300082D6010A01E1B7D6070A01E114D7010A5F
:10A6400001E14ED7030A01E15FD7010A01E166D7B4
:10A650000F0A01E16DD7010A01E174D7030A01E194
:10A660007BD7010A83E0070A8BE0010A9AE0120017
:10A67000DC6F6C0E0001BC6FFC0EBD6F660EBE6F12
:10A68000010EBF6FC06BD6512D0FC16F60005CF320
:10A69000C2F0C36BC46BC56BC66BC76B6000D8F3ED
:10A6A000C8F0B3ECEAF06C0EBC6FFC0EBD6F660E2A
:10A6B000BE6F010EBF6FC06BD6512D0FC16FD72972
:10A6C000C26FC36BC46BC56BC66BC76B6000D8F33E
:10A6D000C8F0B3ECEAF0D80537E16C0EBC6FFC0EA5
:10A6E000BD6FD6513608BE6F010EBF6FC06BD6511D
:10A6F0002D0FC16F60005CF3C2F0C36BC46B6000D0
:10A7000060F3C5F0C66BC76B6000D8F3C8F0B3EC5C
:10A71000EAF06C0EBC6FFC0EBD6FD6513608BE6FF2
:10A72000010EBF6FC06BD6512D0FC16FD729C26FFD
:10A73000C36BC46B600060F3C5F0C66BC76B600091
:10A74000D8F3C8F0B3ECEAF0300ED627640EBF6F32
:10A75000DC517AEC01F0100FD96F0A0EBF6F640E56
:10A76000BB6FDC5166EC02F07AEC01F0100FDA6F8F
:10A770000A0EBB6FDC5166EC02F0100FDB6F970521
:10A7800003E09851D8A41200630EDC6564D0630E18
:10A79000BC6FE50EBD6F070EBE6F020EBF6F60008F
:10A7A00064F3C0F0D651080FC16F60005CF3C2F0D3
:10A7B000C36BC46B600060F3C5F0C66BC76B600011
:10A7C000D8F3C8F0B3ECEAF0630EBC6FE50EBD6FD2
:10A7D000070EBE6F020EBF6F600068F3C0F0D65167
:10A7E000100FC16F60005CF3C2F0C36BC46B6000FC
:10A7F00060F3C5F0C66BC76B6000D8F3C8F0B3EC6C
:10A80000EAF0630EBC6FE50EBD6F070EBE6F020E61
:10A81000BF6F60006CF3C0F0D651180FC16F6000BD
:10A820005CF3C2F0C36BC46B600060F3C5F0C66B31
:10A83000C76B6000D8F3C8F0B3ECEAF0630EBC6FEE
:10A84000E50EBD6F070EBE6F020EBF6FC06B6000DE
:10A8500058F3C1F057D0090EDC6563D0630EBC6FAE
:10A86000E50EBD6F070EBE6F020EBF6FC06B6000BE
:10A8700058F3C1F060005CF3C2F0C36BC46B6000BE
:10A8800060F3C5F0C66BC76B6000D8F3C8F0B3ECDB
:10A89000EAF0630EBC6FE50EBD6F070EBE6F020ED1
:10A8A000BF6FC06BD651080FC16F60005CF3C2F080
:10A8B000C36BC46B600060F3C5F0C66BC76B600010
:10A8C000D8F3C8F0B3ECEAF0630EBC6FE50EBD6FD1
:10A8D000070EBE6F020EBF6F600068F3C0F0D65166
:10A8E000100FC16F60005CF3C2F0C36BC46B6000FB
:10A8F00060F3C5F0C66BC76B6000D8F3C8F0B3EC6B
:10A90000EAF060D060005CF3C2F0C36BC46B60001F
:10A9100060F3C5F0C66BC76B6000D8F3C8F0B3EF47
:10A92000EAF0630EBC6FE50EBD6F070EBE6F020E40
:10A93000BF6FC06B600058F3C1F060005CF3C2F001
:10A94000C36BC46B600060F3C5F0C66BC76B60007F
:10A95000D8F3C8F0B3ECEAF0630EBC6FE50EBD6F40
:10A96000070EBE6F020EBF6FC06BD651080FC16FCE
:10A9700060005CF3C2F0C36BC46B600060F3C5F0B1
:10A98000C66BC76B6000D8F3C8F0B3ECEAF0630E97
:10A99000BC6FE50EBD6F070EBE6F020EBF6FC06BC2
:10A9A000D651100FC16F60005CF3C2F0C36BC46B73
:10A9B000600060F3C5F0C66BC76B6000D8F3C8F0E9
:10A9C000B3ECEAF0630EBC6FE50EBD6F070EBE6F11
:10A9D000020EBF6F60006CF3C0F0D651180FC16F4C
:10A9E00091D7E76BE86BE96B9ED1B00EBC6FF50EAB
:10A9F000BD6F050EBE6F010EBF6FE951D625E06F2A
:10AA0000000ED721E16F600083F3F6FF600087F34B
:10AA1000F7FF000EF86E1F0EF76403D00800F55024
:10AA200007D06F00DBFFE1FF6F00DFFFE2FFE750C1
:10AA3000E00F0001C06FE751FC0D6F00CCFFE2F0AA
:10AA4000E951060DF350E225E36FE851E35DD925A6
:10AA5000C16F600068F3C2F060006CF3C3F0600087
:10AA600070F3C4F0600074F3C5F0600078F3C6F0D2
:10AA700060007CF3C7F06000D8F3C8F0B3ECEAF0F4
:10AA8000E951D625E06F000ED721E16F600083F316
:10AA9000F6FF600087F3F7FF000EF86E1F0EF764F5
:10AAA00003D00800F55007D06F00DBFFE1FF6F0017
:10AAB000DFFFE2FFE750490A1EE00001E951D62519
:10AAC000E06F000ED721E16F600083F3F6FF6000B6
:10AAD00087F3F7FF000EF86E1F0EF76403D008002F
:10AAE000F55007D06F00DBFFE1FF6F00DFFFE2FFF3
:10AAF000E750690A02E10001E72B0001E951D62580
:10AB0000E06F000ED721E16F600083F3F6FF600075
:10AB100087F3F7FF000EF86E1F0EF76403D00800EE
:10AB2000F55007D06F00DBFFE1FF6F00DFFFE2FFB2
:10AB3000E7504B0A01E1F3D00001E951D625E06F5F
:10AB4000000ED721E16F600083F3F6FF600087F30A
:10AB5000F7FF000EF86E1F0EF76403D00800F550E3
:10AB600007D06F00DBFFE1FF6F00DFFFE2FFE75080
:10AB70004C0A01E1D4D00001E951D625E06F000E66
:10AB8000D721E16F600083F3F6FF600087F3F7FFE2
:10AB9000000EF86E1F0EF76403D00800F55007D0C2
:10ABA0006F00DBFFE1FF6F00DFFFE2FFE750530ABA
:10ABB00001E1B5D00001E951D625E06F000ED721A3
:10ABC000E16F600083F3F6FF600087F3F7FF000E8C
:10ABD000F86E1F0EF76403D00800F55007D06F0021
:10ABE000DBFFE1FF6F00DFFFE2FFE750660A01E1F4
:10ABF00096D00001E951D625E06F000ED721E16F14
:10AC0000600083F3F6FF600087F3F7FF000EF86E35
:10AC10001F0EF76403D00800F55007D06F00DBFF6C
:10AC2000E1FF6F00DFFFE2FFE7506B0A78E0000111
:10AC3000E951D625E06F000ED721E16F600083F364
:10AC4000F6FF600087F3F7FF000EF86E1F0EF76443
:10AC500003D00800F55007D06F00DBFFE1FF6F0065
:10AC6000DFFFE2FFE7506C0A5AE00001E951D62508
:10AC7000E06F000ED721E16F600083F3F6FF600004
:10AC800087F3F7FF000EF86E1F0EF76403D008007D
:10AC9000F55007D06F00DBFFE1FF6F00DFFFE2FF41
:10ACA000E750740A3CE00001E951D625E06F000E40
:10ACB000D721E16F600083F3F6FF600087F3F7FFB1
:10ACC000000EF86E1F0EF76403D00800F55007D091
:10ACD0006F00DBFFE1FF6F00DFFFE2FFE7502E0AAE
:10ACE0001EE00001E951D625E06F000ED721E16F8B
:10ACF000600083F3F6FF600087F3F7FF000EF86E45
:10AD00001F0EF76403D00800F55007D06F00DBFF7B
:10AD1000E1FF6F00DFFFE2FFE7502C0A02E10001D4
:10AD2000E82B0001E92BE069E169D851E26FE36BA0
:10AD3000E051E227E151E323E951E46FE56BE25191
:10AD4000E45DE551800AE66FE351800AE65901E2CD
:10AD50004CD61200C96F0001CA6BCE6B606B616B81
:10AD6000626B636B646B656BC70507E1600074FB26
:10AD7000CBF0600078FBCCF092D1020EC71901E055
:10AD80008ED1600010FACBF0600014FACCF087D1BD
:10AD9000795103E1790E785DD8B055D10101615147
:10ADA00001E051D10001B70503E1040ED06F01D0DD
:10ADB000D06B200E3F6008D03F38E842F80BD0132C
:10ADC000870502E1070ED017600040F361F0CB5118
:10ADD000FC0BD01901E061838E510408D06F8E51B5
:10ADE00002E1030ED06F8B0501E1D0878A0501E1F6
:10ADF000D089880501E1D08B030EAF1909E18605E2
:10AE000004E1D08D010ECD6F06D0CD6BD09D03D067
:10AE1000890501E1D08D600040F362F0600030F3FD
:10AE2000C8F07B0EC817D0517B0BC81901E06181B7
:10AE30006295795103E13E0E785D06E37851030F88
:10AE4000BF0BD06F628509D07851791103E13E0EB6
:10AE5000D06F03D06000E0F1D0F0CD0501E1D08DDE
:10AE6000600040F360F0735112E13E0E725D0FE23C
:10AE700072513F0B636F01016A0504E100016351E8
:10AE80004009636F00019A0504E1638F02D03E0E12
:10AE9000636F030E0101E617E62BE651030B030A6D
:10AEA00001E1E66BAB051AE13F0E000160170101FD
:10AEB000015106E13E0E005D03E200C163F006D0E1
:10AEC0000051030F3F0B0001636F608D1F0E0001E7
:10AED0006217628F0101E689040E556EAA0503E030
:10AEE0000001AB0528E1010E0001CE6F6F5103E1B7
:10AEF0004E0E6E5D01E3CE6B6000B8F1C0F06000F5
:10AF0000BCF1C1F0C36B0A0EC26F1DECFFF0C05163
:10AF1000D06FD051060DF3506E25CF6FCFB7CE6BEB
:10AF2000AB0509E16B5106E1E70E6A5D03E26A5188
:10AF30006B1101E1CE6BCE0501E08DD00101AA05B8
:10AF400036E16000B8F1C0F06000BCF1C1F0000172
:10AF5000C36B0A0EC26F1DECFFF0C051D06FD05111
:10AF6000060DF3506E25CF6F040E6217628F6000DE
:10AF70003CF3C8F0070EC817D890C837D890C83728
:10AF8000D890C835D06FD0516213CF390F0B030B57
:10AF9000D06FD0516213CF51400BD06FD05162139C
:10AFA000400E636F0101E68B040E546E54D0000115
:10AFB000AB051EE14D501CE1010E616F040E6217DE
:10AFC0006000A8F1C0F06000ACF1C1F0C36B3C0EB2
:10AFD000C26F1DECFFF0C05103086213628B725107
:10AFE0003F0B636F0F0E0101E617040E536E33D053
:10AFF000AB0531E16000A8F1C0F06000ACF1C1F038
:10B00000C36B3C0EC26F1DECFFF0C051D06F6000EF
:10B01000A8F1BBF06000ACF1BCF0BE6B3C0EBD6FA4
:10B02000D0ECFFF0BB51CF6F040E6217A00E62137D
:10B03000D0510308622760003CF363F0638F639D87
:10B040000101E68DD2D700016295010E0101B26FB8
:10B05000616F0F0EE617E6C164F03B0411E1BE8498
:10B060000001905102E1010E816F810505E10101AE
:10B070004B5102E1080E01D0020E0001D06F0AD040
:10B0800001014B0505E1010E0001D06FBE9402D015
:10B090000001D06BD0516513060ECA6F05D0C9519F
:10B0A000230A01E175D60B0ACA511200CE6F600067
:10B0B00028F3CFF05FD1CB5106E1C86B010EC76F0B
:10B0C00026EC02F021D1CC510BE1C86B010EC76F09
:10B0D00070EC00F0E80601E086D1CA51010A14D1F3
:10B0E000C86B010EC76F8FEC00F0E806F6E07BD16D
:10B0F000CB5106E1C86B020EC76F26EC02F004D1FB
:10B10000CC5106E1C86B020EC76F70EC00F0EDD7B2
:10B11000C86B020EC76F8FEC00F0E7D7CB5106E18A
:10B12000C86B040EC76F26EC02F0EED0CC5106E1DE
:10B13000C86B040EC76F70EC00F0D7D7C86B040E55
:10B14000C76F8FEC00F0D1D7CB5106E1C86B080E6A
:10B15000C76F26EC02F0D8D0CC5106E1C86B080EC0
:10B16000C76F70EC00F0C1D7C86B080EC76F8FECCB
:10B1700000F0BBD7AA0501E036D1CB519EE0CC51FF
:10B1800006E1C86B010EC76F70EC00F0AED7C86B5C
:10B19000010EC76F8FEC00F0A8D7AA0501E023D1FC
:10B1A000CB51A8E0CC5106E1C86B020EC76F70EC22
:10B1B00000F09BD7C86B020EC76F8FEC00F095D7DD
:10B1C000AA0501E010D1CB51ABE0CC5106E1C86B30
:10B1D000040EC76F70EC00F088D7C86B040EC76F01
:10B1E0008FEC00F082D7AA0501E0FDD0CB51AEE094
:10B1F000CC5106E1C86B080EC76F70EC00F075D734
:10B20000C86B080EC76F8FEC00F06FD7CB0501E05D
:10B21000EAD0CC5106E1C86B400EC76F70EC00F06D
:10B2200064D7C86B400EC76F8FEC00F05ED7CB5170
:10B2300006E1C86B100EC76F26EC02F065D0CC514A
:10B2400006E1C86B100EC76F70EC00F04ED7C86BEC
:10B25000100EC76F8FEC00F048D7CB5106E1C86BDA
:10B26000200EC76F26EC02F04FD0CC5106E1C86B20
:10B27000200EC76F70EC00F038D7C86B200EC76F78
:10B280008FEC00F032D7AA0501E0ADD0CB51D1E070
:10B29000CC5106E1C86B100EC76F70EC00F025D7DB
:10B2A000C86B100EC76F8FEC00F01FD7AA0501E026
:10B2B0009AD0CB51D4E0CC5106E1C86B200EC76FB9
:10B2C00070EC00F012D7C86B200EC76F8FEC00F047
:10B2D0000CD7CB0501E087D0CC5106E1020EC86F38
:10B2E000C76B70EC00F001D7020EC86FC76B8FEC14
:10B2F00000F0FBD6CB5177E1C86B080EC76F70EC3E
:10B3000000F0E80603E1010ECF6F6DD0CF6B6BD07C
:10B31000CB5169E1C86B040EC76F70EC00F0E80612
:10B32000F2E0F4D7CB515FE1C86B010EC76F70EC50
:10B3300000F0F5D7CB5157E1C86B020EC76F70EC28
:10B3400000F0EDD7CB514FE1C86B800EC76F26ECF4
:10B3500002F0E5D7CB0547E1CC5106E1C86B800E82
:10B36000C76F70EC00F0C1D6C86B800EC76F8FEC52
:10B3700000F0BBD60001CE51010A01E19CD6030AC0
:10B3800001E1B6D6010A01E1C9D6070A01E1DCD61E
:10B39000010A01E1EFD6030A01E1FFD6010A01E14A
:10B3A0000FD70F0A01E11FD7010A01E12FD7030AC6
:10B3B00001E13DD7010A01E150D7070A01E163D756
:10B3C000010A01E173D7030A84E0010A93E01F0A2E
:10B3D0009FE0010A08E0030AA5E0010AABE0070AC2
:10B3E000B1E0020AB7E0CF511200CC51800BD56F0B
:10B3F000CC51CC25DB6FCBBFDB81DB5108E0DB29F7
:10B4000004E1C96BCA6BCB6BCC6BCB8F04D0C96B1F
:10B41000CA6BCB6BCC6BD051800BD51BD051D025D8
:10B42000D66FCFBFD681D65108E0D62904E1CD6BC7
:10B43000CE6BCF6BD06BCF8F04D0CD6BCE6BCF6B81
:10B44000D06BD65102E0DB5105E1C96BCA6BCB6B07
:10B45000CC6B1200CF51C9036F00CCFFE0F06F003E
:10B46000D0FFE1F0E051D76FD86BD96BDA6BE151C7
:10B47000DC6FDD6BDE6BDF6BCE51CA036F00CCFF80
:10B48000E0F06F00D0FFE1F0E051D727000ED823A5
:10B49000D923DA23E151DC27000EDD23DE23DF236D
:10B4A000CD51CB036F00CCFFE0F06F00D0FFE1F097
:10B4B000E051D727000ED823D923DA23E151DC2726
:10B4C000000EDD23DE23DF23600064F3DAF060008A
:10B4D00060F3D9F060005CF3D8F0D76BCD51CA03AC
:10B4E0006F00CCFFE0F06F00D0FFE1F0E051D72714
:10B4F000E151D823000ED923DA23CE51C9036F00BE
:10B50000CCFFE0F06F00D0FFE1F0E051D727E15130
:10B51000D823000ED923DA23600064F3DAF0600048
:10B5200060F3D9F060005CF3D8F0D76BCD51C9035C
:10B530006F00CCFFE0F06F00D0FFE1F0E051D727C3
:10B54000E151D823000ED923DA23CF51CA036F006B
:10B55000CCFFE0F06F00D0FFE1F0E051DC27E151DB
:10B56000DD23000EDE23DF23CE51CB036F00CCFFA3
:10B57000E0F06F00D0FFE1F0E051DC27E151DD2386
:10B58000000EDE23DF23CF51CB036F00CCFFE0F0B2
:10B590006F00D0FFE1F0E051D16FE151D26FD36B7A
:10B5A000D46B60004CF3D4F0600048F3D3F060003B
:10B5B00044F3D2F0D16BD151DC27D251DD23D351EA
:10B5C000DE23D451DF23DA51DC27000EDD23DE2316
:10B5D000DF23600064F3DAF0600060F3D9F060000C
:10B5E0005CF3D8F0D76BD65160006CF3D1F0D26B1E
:10B5F000D127000ED223820ED125E06FFF0ED2217B
:10B60000E16F0FD0D890DC37DD37DE37DF37DABFB8
:10B61000DC81D890D737D837D937DA37E007D8A0C8
:10B62000E107DEAFEFD7D66BDAAF13D0D751D16FCA
:10B63000D851D26FD951D36F7F0EDA15D46FD15153
:10B64000D211D311D41103E0010ED66F02D0DCB1B8
:10B65000FBD7D6510EE0DC2B000EDD23DE23DF23EB
:10B66000DFA107D0DF35DF33DE33DD33DC33E04B02
:10B67000E12BE1BF0AD0E15102E1E02906E3DC6BF6
:10B68000DD6B800EDE6F7F0E16D0E1BF04D0E1517E
:10B6900008E1E00506E2DC6BDD6BDE6BDF6BD56B92
:10B6A0000BD0600080F3DBF07F0EDE17DF6BDBB1C9
:10B6B000DE8FD890DB31DF6FD551DF13600070F380
:10B6C000C9F0600074F3CAF0600078F3CBF060005A
:10B6D0007CF3CCF01200030E0001C36F010E42ECAC
:10B6E00001F0000E0001C06F020EBF6F63ECFDF0B1
:10B6F0000B0E0001C86F640EC76FB40EE82EFED7A4
:10B70000C72FFCD7C82FFAD700F0030E0001C36F74
:10B71000020E42EC01F0000E0001C06F040EBF6F7C
:10B7200063ECFDF00B0E0001C86F640EC76FB40E22
:10B73000E82EFED7C72FFCD7C82FFAD700F0030E8C
:10B740000001C36F42EC01F0000E0001C06F060E55
:10B75000BF6F63ECFDF00B0E0001C86F640EC76F86
:10B76000B40EE82EFED7C72FFCD7C82FFAD700F0AB
:10B77000030E0001C36F040E42EC01F0000E000145
:10B78000C06F080EBF6F63ECFDF00B0E0001C86FB9
:10B79000640EC76FB40EE82EFED7C72FFCD7C82F94
:10B7A000FAD700F0030E0001C36F050E42EC01F062
:10B7B000000E0001C06F0A0EBF6F63ECFDF00B0EB0
:10B7C0000001C86F640EC76FB40EE82EFED7C72FF6
:10B7D000FCD7C82FFAD700F0030E0001C36F060E86
:10B7E00042EC01F0000E0001C06F0C0EBF6F63EC65
:10B7F000FDF00B0E0001C86F640EC76FB40EE82E8B
:10B80000FED7C72FFCD7C82FFAD700F0030E0001D0
:10B81000C36F070E42EC01F0000E0001C06F0E0E68
:10B82000BF6F63ECFDF00B0E0001C86F640EC76FB5
:10B83000B40EE82EFED7C72FFCD7C82FFAD700F0DA
:10B84000030E0001C36F080E42EC01F0000E000170
:10B85000C06F100EBF6F63ECFDF0000E0001C06FF3
:10B86000120EBF6F63ECFDF02A0E0001C86F8F0E41
:10B87000C76FD80EE82EFED7C72FFCD7C82FFAD730
:10B8800000F0020E0001C36F040E42EC01F0020E44
:10B890000001C36F080E42EC01F0000E0001C06F02
:10B8A000140EBF6F63ECFDF0000E0001C06F160EAA
:10B8B000BF6F63ECFDF0000E0001C06F180EBF6F8C
:10B8C00063ECFDF0000E0001C06F1A0EBF6F63EC59
:10B8D000FDF0150E0001C86FC80EC76F6B0EE82E85
:10B8E000FED7C72FFCD7C82FFAD7000E0001C06FB4
:10B8F000210EBF6F63ECFDF0020E0001C36F030E5B
:10B9000042EC01F0020E0001C36F070E42EC01F0A1
:10B91000150E0001C86FC80EC76F6B0EE82EFED75C
:10B92000C72FFCD7C82FFAD7000E0001C06F240E16
:10B93000BF6F63ECFDF0000E0001C06F270EBF6FFC
:10B9400063ECFDF0020E0001C36F42EC01F0020E49
:10B950000001C36F060E42EC01F0150E0001C86F26
:10B96000C80EC76F6B0EE82EFED7C72FFCD7C82FA7
:10B97000FAD7000E0001C06F2A0EBF6F63ECFDF016
:10B98000020E0001C36F010E42EC01F0020E000135
:10B99000C36F050E42EC01F0010C0001C86B010EF3
:10B9A000C76F70EC00F0E80607E0C86B010EC76FC8
:10B9B0008FEC00F0E8060EE160002CF2CAF06000A7
:10B9C000A4F6CBF0600074F6CCF0CD6B010E56EC13
:10B9D000D8F08B6FC86B020EC76F70EC00F0E806F2
:10B9E00007E0C86B020EC76F8FEC00F0E8060EE1AF
:10B9F000600028F2CAF06000A0F6CBF0600070F69C
:10BA0000CCF0CD6B020E56ECD8F08A6FC86B040EEA
:10BA1000C76F70EC00F0E80607E0C86B040EC76F54
:10BA20008FEC00F0E8060EE1600024F2CAF060003E
:10BA30009CF6CBF060006CF6CCF0CD6B030E56ECB0
:10BA4000D8F0896FC86B080EC76F70EC00F0E8067D
:10BA500007E0C86B080EC76F8FEC00F0E8060EE138
:10BA6000600020F2CAF0600098F6CBF0600068F643
:10BA7000CCF0CD6B040E56ECD8F0886FB00579E1B0
:10BA8000C86B010EC76F70EC00F0E80607E0C86BEA
:10BA9000010EC76F8FEC00F0E8060FE1600078F54B
:10BAA000CAF0600094F6CBF0600064F6CCF0CD6B89
:10BAB000050E56ECD8F001015E6F0001C86B020E56
:10BAC000C76F70EC00F0E80607E0C86B020EC76FA6
:10BAD0008FEC00F0E8060FE1600074F5CAF060003A
:10BAE00090F6CBF0600060F6CCF0CD6B060E56EC15
:10BAF000D8F001015D6F0001C86B040EC76F70ECD8
:10BB000000F0E80607E0C86B040EC76F8FEC00F08A
:10BB1000E8060FE1600070F5CAF060008CF6CBF02B
:10BB200060005CF6CCF0CD6B070E56ECD8F001014E
:10BB30005C6F0001C86B080EC76F70EC00F0E80680
:10BB400008E0C86B080EC76F8FEC00F0E806D8A4B9
:10BB5000120060006CF5CAF0600088F6CBF060005F
:10BB600058F6CCF0CD6B080E56ECD8F001015B6FA7
:10BB70001200C86B010EC76F70EC00F0E80607E01A
:10BB8000C86B010EC76F8FEC00F0E8060EE1600095
:10BB90002CF2CAF06000A4F6CBF0600074F6CCF092
:10BBA000CD6B050E56ECD8F08B6FC86B020EC76FCD
:10BBB00070EC00F0E80607E0C86B020EC76F8FEC70
:10BBC00000F0E8060EE1600028F2CAF06000A0F67E
:10BBD000CBF0600070F6CCF0CD6B060E56ECD8F0D2
:10BBE0008A6FC86B040EC76F70EC00F0E80607E0C0
:10BBF000C86B040EC76F8FEC00F0E8060EE1600022
:10BC000024F2CAF060009CF6CBF060006CF6CCF039
:10BC1000CD6B070E56ECD8F0896FC86B080EC76F56
:10BC200070EC00F0E80608E0C86B080EC76F8FECF8
:10BC300000F0E806D8A41200600020F2CAF060000C
:10BC400098F6CBF0600068F6CCF0CD6B080E56ECA1
:10BC5000D8F0886F12000001CA6FCB6BAC0504E00E
:10BC6000B30502E0010ECB6FC95119E1010ECE6F91
:10BC7000CD6B010ECC6F9251FE0F01017E6F000162
:10BC80009251FE0F01017D6F0001920501017C6F51
:10BC9000010E0001C36F170E25EC01F012D1640EE6
:10BCA000C9190FE1010ECE6FCD6FCC6F92C07EF13E
:10BCB00092C07DF192C07CF1C36F170E25EC01F0AC
:10BCC00000D15A0EC91914E1020ECE6FCB51010EEC
:10BCD000D8B4050ECD6F010ECC6F92C07EF192C02C
:10BCE0007DF192C07CF1C36F170E25EC01F0E9D015
:10BCF000500EC91918E1020ECE6F050ECD6F020E5F
:10BD0000CC6F920501017E6F0001920501017D6FEC
:10BD10000001920501017C6F010E0001C36F170E37
:10BD200025EC01F0CED04B0EC91919E1020ECE6FF1
:10BD3000050ECD6F020ECC6F920501017E6F0001E2
:10BD40009251FE0F01017D6F0001920501017C6F90
:10BD5000010E0001C36F170E25EC01F0B2D0400EAA
:10BD6000C9191AE1030ECE6F050ECD6F020ECC6F0E
:10BD7000920501017E6F00019251FE0F01017D6F5E
:10BD800000019251FE0F01017C6F010E0001C36F93
:10BD9000170E25EC01F095D0320EC9191AE1020EEA
:10BDA000CE6F040ECD6F010ECC6F920501017E6F38
:10BDB00000019251FE0F01017D6F00019251FE0FB3
:10BDC00001017C6F010E0001C36F170E25EC01F01D
:10BDD00078D0300EC9191AE1020ECE6F030ECD6F66
:10BDE000010ECC6F920501017E6F00019251FD0F93
:10BDF00001017D6F00019251FD0F01017C6F010E69
:10BE00000001C36F170E25EC01F05BD0200EC9199D
:10BE10001BE1010ECE6F030ECD6F010ECC6F925160
:10BE2000FE0F01017E6F00019251FD0F01017D6F38
:10BE300000019251FD0F01017C6F030E0001C36FE1
:10BE4000170E25EC01F03DD0190EC9191EE1010EA7
:10BE5000CE6FCB51020ED8B4030ECD6F010ECC6F56
:10BE60009251FE0F01017E6F00019251FD0F010101
:10BE70007D6F00019251FD0F01017C6F030E0001E7
:10BE8000C36F170E25EC01F01CD0010ECE6FCB5105
:10BE9000010ED8B4020ECD6FCC6B9251FE0F010192
:10BEA0007E6F00019251FD0F01017D6F00019251E3
:10BEB000FD0F01017C6F020E0001C36F170E25EC10
:10BEC00001F0020E0001CA190AE1CE51050FC76F39
:10BED000CE51F6ECFEF001017E51AFEF01F0030E02
:10BEE000CA1908E1C76BCC29F6ECFEF001017C51C0
:10BEF000AFEF01F0CD51020FC76F000EF6ECFEF070
:10BF000001017D51AFEF01F00001D26F20D1040E8D
:10BF10000201406502D045B345D041513F0B0001BD
:10BF2000D46FD45103E03E0ED41906E17A6B7B6BDB
:10BF3000010E0101B26F0FD0020143A505D000012F
:10BF4000D4514009FD0FD46F600050F37AF0000126
:10BF50007B6B0101B26B030E0001AF190BE1020113
:10BF60004351400BE80604E1010E0101566F02D077
:10BF70000101566B020144513F0B0001D36F0201D6
:10BF800044BF02D00001D36B0001D35109E09A05F0
:10BF900007E16000C8F135F06000CCF136F002D066
:10BFA000356A366A040E02014065040C45C2B5F0DC
:10BFB0006000D4F2D1F0030E0001D1170101E65167
:10BFC000030B0001D11901E0A3D0B5A929D0B5AF69
:10BFD0001CD0556A0101AB6B030EE61700C102F1DC
:10BFE00001C103F1010E566E040E0201DE173E0E72
:10BFF000DF6F0F0EE017566ADEC2C9F2DFC2CAF267
:10C00000E0C2CBF20001626B0BD0556A0101AB6B51
:10C01000030EE61778C07AF079C07BF0026B036BF1
:10C020000001B5AB3DD0B5AF34D06AC09AF26BC059
:10C030009BF26EC09CF26FC09DF20101AA6B0001E1
:10C04000AB0525E14D5023E1040E536E546A010EF9
:10C05000C76F230EAAECD6F0010E566E60C0DCF25C
:10C0600061C0DDF262C0DEF263C0DFF264C0E0F204
:10C07000566A60C0C7F261C0C8F262C0C9F263C04C
:10C08000CAF264C0CBF2020E4C6E010E4D6E546AC1
:10C0900007D002019D6B0A0E9C6F0101AA6BF7D7B6
:10C0A0000001AB0523E14C5021E14D041FE1010EDD
:10C0B000C76F230EAAECD6F0010E566E60C0DCF2FC
:10C0C00061C0DDF262C0DEF263C0DFF264C0E0F2A4
:10C0D000536E566A60C0C7F261C0C8F262C0C9F24E
:10C0E00063C0CAF264C0CBF2020E536EB5AD10D07D
:10C0F000B5AF07D06AC09AF26BC09BF24D6A536A23
:10C1000006D002019A6B9B6B4D6A536A0001AB6BC0
:10C11000600018F9D4F0D4A308D03B5004E1010E1C
:10C120000101496F486B010E3B6E0001D4B307D08B
:10C130003B0404E10101496B010E486F3B6A0001B9
:10C14000D4A503D0010E816F010C816B1200000198
:10C15000D251230A01E1DBD60B0A1200EE6F0C0E5E
:10C160000001EB6502D00D0EEB6F020EED6F6C0E51
:10C17000BC6FFC0EBD6F0C0EBE6F010EBF6FC06BAF
:10C180005A0EC16F6000B4F3C2F0C36BC46BC56BD1
:10C19000C66BC76B6000D8F3C8F0B3ECEAF0ED2BC8
:10C1A000070EED65E4D76C0EBC6FFC0EBD6F660E1E
:10C1B000BE6F010EBF6FC06BC16B6000B8F3C2F001
:10C1C000C36BC46BC56BC66BC76B6000D8F3C8F09C
:10C1D000B3ECEAF06C0EBC6FFC0EBD6F660EBE6F6A
:10C1E000010EBF6FC06BC16BEE29C26FC36BC46B16
:10C1F000C56BC66BC76B6000D8F3C8F0B3ECEAF050
:10C20000020EEE6518D0500EBC6FFA0EBD6F0B0E0D
:10C21000BE6F010EBF6F1B0EC06F5B0EC16FEE05D0
:10C22000C26FC36BC46BC56BC66BC76B6000D8F3C2
:10C23000C8F0B3ECEAF0060EEE6119D0500EBC6FF8
:10C24000FA0EBD6F0B0EBE6F010EBF6F1C0EC06FDE
:10C250005B0EC16FEE51020FC26FC36BC46BC56B37
:10C26000C66BC76B6000D8F3C8F0B3ECEAF0020EFF
:10C27000BC6FBD6B6000B8F3BEF06000D8F3BFF0D8
:10C28000660EB2ECF3F0EC0541E16C0EBC6FFC0EF7
:10C29000BD6F660EBE6F010EBF6FC06BC16B6000DD
:10C2A000B8F3C2F0C36BC46BC56FC66BC76B6000DD
:10C2B000D8F3C8F0B3ECEAF06C0EBC6FFC0EBD6FA7
:10C2C000660EBE6F010EBF6FC06BC16BEE29C26FF1
:10C2D000C36BC46B010EC56FC66BC76B6000D8F330
:10C2E000C8F0B3ECEAF06000A4F3D6F06000A8F365
:10C2F000D7F06000ACF3D8F0030ED96F6000B8F34C
:10C30000DAF0DB6BDC6B010EDD6F12D06000A4F3A2
:10C31000D6F06000A8F3D7F06000ACF3D8F0030EBD
:10C32000D96F6000B8F3DAF0010EDB6FDC6FDD6B04
:10C33000DE6BDF6B68EFF1F00001DD6F600068F32A
:10C34000DEF0010EC86FC76B70EC00F0E8064CE140
:10C35000010ECA6F6000E4F0CBF06000E8F0CCF0B2
:10C36000020ECE6FCD6F040ED06FCF6F090E83EC2F
:10C37000C8F0600028F339F060002CF33AF0DD05D6
:10C3800027E1810531E180512FE1030EA26F010EFB
:10C390009F6F0101326B336B010E0001806F6000F3
:10C3A00000F2CAF06000E4F0CBF06000E8F0CCF0FE
:10C3B000040ECE6FCD6F100ED06FCF6F090E83ECD1
:10C3C000C8F0600028F339F060002CF33AF00CD08C
:10C3D000DA0506E1DE6BA1C0A2F0010E9F6F04D06A
:10C3E000A2C0A1F0010EDE6F010EC86FC76B26EC74
:10C3F00002F0E80630E1800534E1010E0101CE6F64
:10C400000001DD5106E0400E0101325D010E33599D
:10C4100028E30101CE6B326B336B0001806BDE6B66
